:100000000C94E00C0C94FD0C0C94FD0C0C94FD0C69
:100010000C94FD0C0C94020F0C9427110C94FD0C05
:100020000C94FD0C0C94FD0C0C94FD0C0C94FD0C2C
:100030000C94FD0C0C94FD0C0C94B5220C94FD0C4E
:100040000C9449140C9438120C94120F0C94C90E91
:100050000C94FD0C0C94CA1D0C94FD0C0C94FD0C1E
:100060000C94FD0C0C94FD0C0C94FD0C0C94FD0CEC
:100070000C94FD0C0C945D230C943B110C94E91032
:100080000C94FD0C0C944B590C94FD0CC0538C54E7
:10009000F552C953A05427534353EE54EE54EE5433
:1000A0006153EE54EE54EE54EE54DD536C546C54E4
:1000B0008854215421541F541D541B54EE54EE54A3
:1000C000EE54EE54EE54EE54EE54B053EE54EE545F
:1000D000EE54EE54EE54EE54EE54EE54EE54EE5410
:1000E000EE54EE54EE54EE54EE54EE54EE54EE5400
:1000F000EE54EE54EE54EE54EE54EE54EE54EE54F0
:10010000EE54EE54EE54EE54EE54DF54D154BF543A
:10011000A45445617379436F6E74726F6C00204D07
:100120004300696E636F6D70617469626C6520482D
:100130005700312E342E30005F03AF01D7006B0023
:10014000470035001A0011000102031304050611CF
:10015000070809120A000B0C100F0E0D0101010512
:100160000D1F0C04040E1F04041F0E041F1F1F008C
:100170001F1F1F001F1F1F001F111F001F111F0027
:100180001F1F1F001F111F001F111F00000609174E
:1001900017090600000609121412090603070F1EAC
:1001A0001C18100003050912141810000707070790
:1001B0000707070707050505050505071C1018179C
:1001C000150705071C101817110202021C1018123F
:1001D000140605021C101817140601061C10181529
:1001E000150701011C101816110201061C10181623
:1001F000110204071C10181216020207040A110A41
:100200000A0E00000C17141714170C001C101810FD
:10021000160505051F0A0A0A0A0A1F000E11111FFA
:100220001B1B1F0002060F1F0F060200080C1E1FDB
:100230001E0C08000E0E0E0E1F0E0400040E1F0EE4
:100240000E0E0E0000030C0F30333C3FC0C3CCCF6A
:10025000F0F3FCFFC303F333CF0FFF3FAAC080309E
:10026000F0B020E0A00CCC8C3CFCBC2CECAC08C862
:100270008838F8B828E8A803C38333F3B323E3A38B
:100280000FCF8F3FFFBF2FEFAF0BCB8B3BFBBB2BBA
:10029000EBAB02C28232F2B222E2A20ECE8E3EFE60
:1002A000BE2EEEAE0ACA8A3AFABA2AEA004060972F
:1002B0007048685878446454744C6C5C7C42625258
:1002C000724A6A5A7A466656764E6E5E7E41615131
:1002D000714969597945659F754D6D5D7D436353DE
:1002E000734B6B5B7B476757774F6F5F7F101814BB
:1002F0001C121A161E1119151D131B171FD0D8D446
:10030000DCD2DAD6DED1D9D5DDD3DBD7DF90989435
:100310009C929A969E9199959D939B5055040605A3
:1003200007C4C6C5C78486858734363537F4F6F5E5
:10033000F7B4B6B5B724262527E4E6E5E7A4A6A5D5
:10034000A701C18131F1B121E1A10DCD8D3DFDBDEF
:100350002DEDAD09C98939F9B929E9A92020202055
:1003600020200000204D4D4920200000204D4D014F
:100370002020000020444343202000002053544FFD
:100380005020000053484F52542100002048414C57
:100390005420000000000000000000002050524FD8
:1003A0004720000052455345542000007E0E0E0E9B
:1003B0000E1B1B1C0E1B1B7E0E0E0E0E232D004152
:1003C00044523A20256C6420202020202020202028
:1003D00020002D2D2D2D202000252D3564002533C6
:1003E0006400202001022020202020202000252D34
:1003F000356400252D31312E313173000002060A9B
:100400000F13181D22262B3035393F43484C5156C7
:100410005B5F64696E72777B7F0002060A0F1318B8
:100420001D22262B3035393F43484C51565B5F64C3
:10043000696E73797F00020A131D263039434C56CA
:100440005F69727F2530386C75005741524E494EB6
:10045000473A20004552524F523A200062616420D0
:10046000706172616D657465722076616C7565008E
:10047000706F776572206973204F666600747572BD
:100480006E6F75742071756575652066756C6C008E
:10049000636F6D6D616E642071756575652066753D
:1004A0006C6C006E6F2064617461006E6F20736C01
:1004B0006F7420617661696C61626C65006C6F6B52
:1004C000206275737900696C6C6567616C20747566
:1004D000726E6F757420616472657373004D432092
:1004E000696E2048414C54004D4320696E2053549E
:1004F0004F50004C207B4C6F6B232C205B5370655E
:1005000065645D2C205B464C5D2C205B4469725D0C
:100510002C205B46315D2C205B46325D2C205B46F7
:10052000335D2C205B46345D7D0054207B54726E1D
:1005300074232C205B436F6C6F725D2C205B5374B3
:10054000617475735D7D0046207B4C6F6B232C209E
:100550005B46315D2C205B46325D2C205B46335D73
:100560002C205B46345D2C205B46355D2C205B46A1
:10057000365D2C205B46375D2C205B46385D7D0068
:10058000484C2048656C7020666F72206C6F6B2041
:10059000636F6D6D616E64730D0048462048656C35
:1005A0007020666F722066756E6374696F6E20636B
:1005B0006F6D6D616E64730D0048542048656C70FA
:1005C00020666F72207475726E6F757420636F6D24
:1005D0006D616E647300507772206F6666004861CB
:1005E0006C7465642100507772206F6E0044434341
:1005F0002070726F6772616D005245534554004818
:10060000616C746564210D5D004C20257520257595
:100610002025632025632025632025632025632072
:10062000256300756E75736564004D6F746F726F2E
:100630006C61204F6C64004D6F746F726F6C612041
:100640004E657700444343004620257520256320EE
:10065000256320256320256320256320256320252D
:1006600063202563004658202575202563202563D7
:100670002025632025632025632025630054202541
:1006800064202563202564004D43205265766973FC
:10069000696F6E2000312E342E30000D5365724E7E
:1006A000722E2025386C75004D5420256420256459
:1006B000005352202564004D6F64756C652023251E
:1006C000642028696E70757420312E2E3820262003
:1006D000392E2E313629203D200053452025640037
:1006E0003537363030002575000D5D002564005A21
:1006F0007A4100556E6B6E6F776E20636F6D6D6122
:100700006E64000D5D003132000032340000343878
:1007100000003936000031343400313932003338CA
:100720003400353736004142434445464748494A3C
:100730004B4C4D4E4F505152535455565758595A91
:10074000303132333435363738392E2C3A2D2B238D
:100750002F3D3C7C3E20004D4D204920203134204F
:10076000004D4D20492020323761004D4D20492059
:1007700020323762004D4D20012020313420004DC1
:100780004D20012020323761004D4D2001202032C4
:100790003762004443432020203134200044434347
:1007A000202020323820004443432020313238209A
:1007B000004C6F636D656E75000000000000000066
:1007C000004443432D70726F6772616D6D2E00009F
:1007D000004D6F64656C6261616E7369742E000018
:1007E00000496E7374656C6C696E67656E0000001D
:1007F00000536F667477617265205570646174652B
:10080000004C4344207665726C69636874696E6756
:10081000004D6173746572436F6E74726F6C00008B
:10082000004578697400000000000000000000002E
:10083000004B69657A656E20000000000000000032
:100840000044617461666F726D61740000000000A5
:10085000004E61616D20202020202000000000005B
:1008600000496E766F657220202020000000000095
:1008700000435620286279746529000000000000BA
:10088000004356202862697429000000000000001F
:100890000042617369736164726573000000000057
:1008A000004C616E67206164726573000000000097
:1008B00000526567697374657200000000000000F3
:1008C00000506167652D4D6F6465000000000000F9
:1008D00000486F6F666473706F6F720000000000F5
:1008E000007338382D696E7374656C6C696E67655A
:1008F0006E436F6E666967757261746965000000AA
:1009000000426F6F73746572636F6E666967000093
:1009100000496E74657266616365204261756400AA
:100920000057697373656C636F6E666967000000DA
:10093000004C6F63666F726D617400000000000010
:10094000004D4D207369676E61616C7061757A65E9
:10095000007338382D6D6F64756C65000000000001
:10096000007338382D6D6F64756C65746573740031
:10097000004B6F7274736C2E20706F6C2E00000031
:10098000004B6F7274736C2E206765762E0000002A
:100990000057697373656C666F726D617400000057
:1009A000004D696E2E20736368616B656C74696AB3
:1009B000644D61782E20736368616B656C74696A3D
:1009C000644D656E75204C6F636F00000000000081
:1009D0000050726F6772616D2E2044434300000027
:1009E0000045746174205265736561752E000000C6
:1009F000005265676C6167657300000000000000CD
:100A0000004D414A206C6F67696369656C000000A6
:100A1000004C756D696E6F736974650000000000AD
:100A2000004D6173746572436F6E74726F6C000079
:100A3000004578697400000000000000000000001C
:100A40000053656C656374696F6E200000000000E0
:100A500000466F726D617420646F6E6E6565730021
:100A6000004E6F6D2020202020202000000000007C
:100A70000053616973696520202020000000000098
:100A800000435620286279746529000000000000A8
:100A9000004356202862697429000000000000000D
:100AA00000416472657373652064652062617365DB
:100AB0000041647265737365206C6F6E67756500C5
:100AC00000526567697374657200000000000000E1
:100AD00000506167652D4D6F6465000000000000E7
:100AE00000566F6965207072696E636970616C652C
:100AF000005265676C61676520733838000000003C
:100B000000436F6E66696775726174696F6E00008D
:100B100000436F6E6669672E20426F6F7374657253
:100B200000496E7465726661636520426175640098
:100B300000436F6E662E2041696775696C6C612E8B
:100B400000466F726D6174206C6F636F000000006F
:100B5000005061757365207369676E616C204D4D3F
:100B6000004D6F64756C65732073383800000000A9
:100B70000054657374206D6F64756C65207338382C
:100B800000506F6C2E6372742D63697263756974A3
:100B90000053656E732E206372742D6369726374E3
:100BA00000466F726D61742061696775696C6C2EA7
:100BB00000547073206D696E2E696D70756C732EA4
:100BC00000547073206D61782E696D70756C732E92
:100BD000004C6F6B204D656EFC00000000000000B3
:100BE000004443432D50726F6772616D6D672E0034
:100BF00000416E6C6167656E7A757374616E640036
:100C00000045696E7374656C6C756E67656E000087
:100C100000536F6674776172652055706461746506
:100C2000004C43442042656C6575636874756E675B
:100C3000004D6173746572436F6E74726F6C000067
:100C4000004578697400000000000000000000000A
:100C50000041757377E4686C656E20000000000049
:100C600000446174656E666F726D6174000000000F
:100C7000004E616D65202020202020000000000033
:100C80000045696E7472616720202000000000003A
:100C90000043562028627974652900000000000096
:100CA00000435620286269742900000000000000FB
:100CB0000042617369732D4164726573736500004E
:100CC000006C616E67652041647265737365000036
:100CD00000526567697374657200000000000000CF
:100CE00000506167652D4D6F6465000000000000D5
:100CF000004861757074676C6569730000000000DE
:100D0000007338382D45696E7374656C6C756E6749
:100D1000004B6F6E66696775726174696F6E000073
:100D200000426F6F737465726B6F6E6669672E0039
:100D300000496E7465726661636520426175640086
:100D4000005765696368656E6B6F6E6669672E0034
:100D5000004C6F6B666F726D6174000000000000E4
:100D6000004D4D2D5369676E616C20506175736540
:100D7000007338382D4D6F64756C650000000000FD
:100D8000007338382D4D6F64756C74657374000092
:100D9000004B75727A7363686C2E2D506F6C2E0049
:100DA000004B75727A7363686C2E2D456D70662EDC
:100DB000005765696368656E666F726D61740000E7
:100DC000006D696E2E20536368616C747A65697476
:100DD000006D61782E20536368616C747A65697464
:100DE00000547261696E206D656E75000000000030
:100DF000004443432070726F6772616D6D696E6766
:100E0000004C61796F7574206D6F6475730000001C
:100E10000053657474696E67730000000000000081
:100E200000536F66747761726520557064617465F4
:100E3000004C4344206C69676874696E6700000069
:100E4000004D6173746572436F6E74726F6C000055
:100E500000457869740000000000000000000000F8
:100E60000073656C656374200000000000000000E2
:100E7000006461746120666F726D6174000000002F
:100E8000004E616D65202020202020000000000021
:100E900000456E74727920202020200000000000A0
:100EA0000043562028627974652900000000000084
:100EB00000435620286269742900000000000000E9
:100EC000004261736963206164726573730000009E
:100ED000004C6F6E672061647265737300000000E0
:100EE00000526567697374657200000000000000BD
:100EF00000506167652D4D6F6465000000000000C3
:100F0000004D61696E20747261636B000000000027
:100F1000007338382073657474696E67730000005D
:100F200000436F6E66696775726174696F6E000069
:100F300000426F6F7374657220436F6E6669672E2F
:100F400000496E7465726661636520426175640074
:100F500000506F696E747320436F6E6669672E0070
:100F600000547261696E20666F726D6174000000DA
:100F7000004D4D207369676E616C207061757365FB
:100F800000733838206D6F64756C65730000000065
:100F900000733838206D6F64756C652074657374E8
:100FA0000073686F727420706F6C6172697479007D
:100FB0000073686F72742073656E73697469762E3E
:100FC00000706F696E747320666F726D61740000DB
:100FD000006D696E2E20737769746368696E6700AF
:100FE000006D61782E20737769746368696E67009D
:100FF00000202D2D2D2D0025357500536F6674773B
:101000002E205600312E342E30005365724E722E33
:101010002025386C75003A2000253575002533648D
:10102000002534643A20002D2D2D00253364002046
:101030004F4B202020200020202020202020004373
:10104000563A20202020204269743A203D20004357
:10105000563A253464204269743A25643D00202DB7
:101060002D2D0025346400202D2D2D2D2D0025360D
:1010700064002533642C256473002534646D73008B
:101080003030204261756400446F776E6C6F61642C
:10109000202E2E2E002564206D7300202532640042
:1010A0004E723A2025326420200073686F727420DB
:1010B00028312E356D73292000006C6F6E67202853
:1010C000342E3032356D732900004D6F746F726F9E
:1010D0006C61000000000000000044434320202019
:1010E00020200000000000000000706F7369746928
:1010F000766520284D4D290000006E656761746992
:101100007665202844434329000020726573746F7C
:101110007265202020202020000020736176652049
:10112000202020202020202000004B6F72722028D9
:10113000312E356D7329202000004C616E67202808
:10114000342E3032356D732900004D6F746F726F1D
:101150006C61000000000000000044434320202098
:1011600020200000000000000000506F73697469C7
:10117000656620284D4D290000004E656761746941
:101180006566202844434329000020486572737433
:10119000656C6C656E2020200000204F70736C61C0
:1011A000616E2020202020200000436F7572742083
:1011B00028312E356D73292000004C6F6E67202872
:1011C000342E3032356D732900004D6F746F726F9D
:1011D0006C61000000000000000044434320202018
:1011E00020200000000000000000706F7369746927
:1011F000766520284D4D290000006E656761746991
:1012000076652028444343290000205265737461A9
:1012100075726174696F6E20000020456E7265679B
:10122000697374726520202000004B75727A202843
:10123000312E356D7329202000004C616E67202807
:10124000342E3032356D732900004D6F746F726F1C
:101250006C61000000000000000044434320202097
:1012600020200000000000000000706F73697469A6
:101270007620284D4D29000000006E656761746975
:10128000762028444343290000002077696564657F
:101290007268657273742E20000020737065696334
:1012A0006865726E202020200000696E636F6D708B
:1012B00061742E20466F726D617400496E636F6DAC
:1012C000702E20466F726D6174202000466F726D23
:1012D000617420696E636F6D7061742E00696E6B4E
:1012E0006F6D7061742E20466F726D6174002E2ECA
:1012F0002E2077616974696E67202E2E2E200023C0
:101300003D64656C6574650000000000000000002D
:10131000286E6F20656E747279290000000000004D
:10132000002E2E2E2064656C6574696E67202E2E4B
:101330002E00206661756C74000000000000000043
:1013400000000020444343206F6E6C7921000000B0
:10135000000000002A3D446973636F6E742E200004
:1013600000000000002070726F6772616D696E6727
:101370000000000000002D73686F727420636972B2
:10138000637569742D20002A726561642000000075
:1013900000000000000000002A77726974650000F8
:1013A0000000000000000000002E2E2E2077726941
:1013B00074696E67202E2E2E20002E2E2E20726530
:1013C0006164696E67202E2E2E2000212121206667
:1013D00061756C742021212120202000204F4B209A
:1013E000202020202020202020202020002E2E2EF3
:1013F00020736176696E67202E2E2E2020002E2EFF
:1014000020726573746F72696E67202E2E20002320
:101410003D64656C657465202A3D646973632E00C4
:10142000233D796573202A3D646973636F6E742E62
:10143000002064656C657465202020202020202019
:1014400000004F46460000000000000000000000C1
:101450000000002A2A2A206E6F20547261696E20D3
:101460002A2A2A002A2073686F72742063697263C3
:1014700075697420002A2A2A2074696D65206F75A9
:1014800074202A2A2A00506F696E74202025346443
:101490002F2534640000002E2E2E2077616368749F
:1014A000656E202E2E2E2020233D77697373656E86
:1014B000000000000000000000286765656E2069DC
:1014C0006E766F65722900000000202E2E2E207788
:1014D000697373656E202E2E2E000020666F757462
:1014E00000000000000000000000000020416C6CC3
:1014F00065656E204443432100000000002A3D2022
:1015000041666272656B656E00000000000020504D
:10151000726F6772616D6D6572656E000000002DFF
:101520002D4B6F7274736C756974696E672D2D0025
:101530002A4C657A656E0000000000000000000083
:10154000002A536368726900000000000000000078
:1015500000002E2E2073636872696A76656E202EF5
:101560002E00002E2E2E206C657A656E202E2E2EDB
:10157000202000002021212120466F757420212188
:101580002120200000204F4B202020202020202040
:101590002020202000002E2E2E204F70736C6161C1
:1015A0006E202E2E2E00004865727374656C6C657B
:1015B0006E20202020200000233D77697373656E24
:1015C000202A3D616662720000233D4A41202A3D87
:1015D000616662722E202020000020776973736597
:1015E0006E2020202020202020200055495400007B
:1015F0000000000000000000000000002A2A2A204D
:101600006765656E204C6F63202A2A2A002A2A6BA0
:101610006F7274736C756974696E672A2A002A2068
:1016200054696A646F766572736368722E2A005714
:10163000697373656C732534642F2534640000006E
:1016400050617469656E74657A00000000000000E6
:1016500000233D7375707072696D65720000000043
:1016600000007669646500000000000000000000D2
:101670000000005375707072657373696F6E0000BF
:1016800000000000204572726575720000000000C5
:1016900000000000002044434320756E69717565A9
:1016A0006D656E7400002A3D4162616E646F6E204C
:1016B000200000000000002050726F6772616D6DA5
:1016C0006174696F6E0000002D436F7572742D6335
:1016D0006972637569742D20002A4C6563742E004D
:1016E000000000000000000000002A4563726974D9
:1016F00000000000000000000000002E2E2E2045FB
:1017000063726974757265202E2E2E002E2E2E2087
:101710004C656374757265202E2E2E2000212121C8
:101720002045727265757220212121202000204FF2
:101730004B2020202020202020202020202000209E
:10174000456E72656769737472656D656E742000AD
:1017500020526573746175726174696F6E20202008
:1017600000233D5375707072202A3D4162616E64A2
:101770002E00233D4F7569202A3D4162616E646FE2
:101780006E2000205375707072696D657220202084
:1017900020202000496E616374696620202020208B
:1017A00020202020002A20506173206465206C6F67
:1017B000636F202A20002A20436F7572742D63699D
:1017C000726375697420002A2054656D70732064FB
:1017D000657061737365200041696775696C2E25BA
:1017E00034642F2534640000002E2E2E2077617281
:1017F00074656E202E2E2E202000233D4CF6736340
:1018000068656E0000000000000000286B65696ECE
:101810002045696E7472616729000000202E2E2E0B
:10182000206CF673636865202E2E2E2000204665FE
:10183000686C657200000000000000000000206E6F
:1018400075722066FC722044434321000000002A88
:10185000203D204162627275636800000000000054
:101860002050726F6772616D6D696572756E670089
:10187000002D2D204B75727A7363686C75DF202DF7
:101880002D002A6C6573656E0000000000000000EA
:101890000000002A736368722E0000000000000040
:1018A000000000002E2E2073636872656962656E09
:1018B000202E2E00002E2E2E206C6573656E202E9D
:1018C0002E2E20200000212121204665686C6572A3
:1018D00020212121200000204F4B202020202020EB
:1018E00020202020202000002E2E207370656963A8
:1018F0006865726E202E2E000077696564657268D7
:1019000065727374656C6C656E00233D4CF6736391
:1019100068656E202A3D4162627200233D4A612063
:101920002A3D41626272756368000000206CF673A4
:101930006368656E20202020202020200041555320
:1019400000000000000000000000000000002A2A43
:10195000206B65696E65204C6F6B202A2A20002A57
:101960002A204B75727A7363686C75DF202A2A000F
:101970002A205A656974FC626572736368722E2A44
:1019800000576569636865202534642F2534640039
:1019900000005B6E6F206D6573736167655D005B52
:1019A000756E6B6E6F776E206572726F725D005B25
:1019B000756E6B6E6F776E207374617475735D00F6
:1019C00011241FBECFEFD0E1DEBFCDBF12E0A0E0FB
:1019D000B1E0E0EDF0ED00E00BBF02C007900D922A
:1019E000A63AB107D9F71DE0A6EAB2E001C01D9200
:1019F000AD34B107E1F70C94690D0C94000081E05F
:101A00008093A7020895982F8091A602891731F03C
:101A1000863021F0853029F4963019F080E090E08E
:101A200008959093A602892F8250823058F40E9424
:101A3000271D1092F0068091A602823051F40E9478
:101A4000C42707C0943019F40E944A1D02C00E94A6
:101A5000361D8091A602863011F40E94B551809106
:101A6000A602813019F482E00E94FF6146EA52E04A
:101A700063E08FEF0E946A520E94FF0C81E090E0C9
:101A8000089508958091A6029927089580E00E9404
:101A900030192FEF8F3F920719F0682F80E009C0AF
:101AA00081E00E9430192FEF8F3F920721F0682FBD
:101AB00081E00E94C33C0E9480520E94CF600E943D
:101AC000882B8091A702882311F40E941018A895F2
:101AD0000895CFEFD0E1DEBFCDBF0E94824F0E94BC
:101AE000470E0E9403240E94A45F0E94781D0E945A
:101AF000C24F21E04EE468E00E94740E21E04EE403
:101B000068E087E00E948D100E942B1278940E945A
:101B1000F9130E94BA4FFC0184810E94791862E196
:101B200071E082E00E94AE180E940550813059F0A9
:101B300060E081E00E94261762E271E082E00E948C
:101B4000AE18A895FECF6EE171E082E00E94AE185B
:101B500060E081E00E94261766E582E00E947E1820
:101B600062E371E082E00E94AE180E94BA4F8C01DD
:101B700081E00E941116882319F081E00E94BD4F78
:101B800082E00E941116882319F080E00E94BD4F68
:101B900083E00E941116882319F082E00E94BD4F55
:101BA00084E00E941116882319F083E00E94BD4F43
:101BB00080E00E94030D80E00E941116882319F036
:101BC00084E10E944E4E0E94A95C40E050E060E239
:101BD0008FEF0E946A5280E00E94A73C81E00E9441
:101BE000A73C8091F2069091F306A091F406B09183
:101BF000F506805D9740A040B04078F40E94460D05
:101C00008091F2069091F306A091F406B091F5064A
:101C1000805D9740A040B04088F3F80181859285AF
:101C2000892BC9F00E940C28EC0144969E01215F8B
:101C30003F4FAC01B901F801818592850E94BB5BE1
:101C4000BC01892B29F0F801818592858A8B9B8BB9
:101C50006115710519F4F801628173818FEF0E949B
:101C6000255181E011C00E94A32B0E94D316FFEFE3
:101C70008F3F9F07C1F70E94460D8091A7028823DE
:101C8000A1F31092A70280E00E948D29EECF8FE78A
:101C90008ABB1BBA80E187BB18BA80EF84BB8FEF89
:101CA00085BB8BEB81BB8CEC82BB86E082B987EF76
:101CB00083B98093610081EF809362008FE180930C
:101CC000640089E1809365000E94425910926A0085
:101CD0001ABE8AB78A608ABF0E946A15A89588E1F1
:101CE00081BD8CE081BD0895E82F1092C4068091DB
:101CF000C4068093C3068091C3068093E606809154
:101D0000E6068093E50691E09093EF068C9A119A8F
:101D100082B18E7E82B9199A83B18E7E83B982E0B8
:101D20008BB99498E83008F0E92FFF27EE0FFF1FDA
:101D3000E85CFE4FA591B491653010F465E003C0F6
:101D4000693008F068E04F7D6550660F453411F446
:101D5000606203C04F3409F46063223008F06860A9
:101D60008B2F992787FD9A958F7080939000A9B942
:101D70006093950088EB8AB980E090E00895909197
:101D8000E5068091E606981711F00C9B559A089588
:101D900008951F920F920FB60F9211248F939F9365
:101DA000EF93FF939091E5068091E606981761F016
:101DB00088B7806188BF0C9B09C089B7806189BFE3
:101DC0008091EF0680FF02C0559813C08091E6060F
:101DD000E82FFF27ED53F94F84A18CB98091E606D7
:101DE0008F5F8093E6068091E606883010F01092AF
:101DF000E606FF91EF919F918F910F900FBE0F908C
:101E00001F9018951F920F920FB60F9211248F9367
:101E100089B78F7E89BF559A8F910F900FBE0F9013
:101E20001F9018951F920F920FB60F9211242F93A7
:101E30003F934F935F936F937F938F939F93AF9352
:101E4000BF93EF93FF938091C306282F3327809190
:101E5000C406992701972817390741F08091C306D6
:101E60008F3179F48091C406882359F48091C40697
:101E70008F5F8093C4068091C406803210F0109268
:101E8000C4069BB18091C306E82FFF27ED53F94F9D
:101E90008CB18283228194FD0CC08091C3068F5F38
:101EA0008093C3068091C3068032A8F01092C306C7
:101EB00012C0222381F42093C4068091C40680932B
:101EC000C3069498822F0E94A73C21E04EE468E06C
:101ED000822F0E94740E8091C306282F3327809191
:101EE000C406281B310937FF02C0205E3F4F213155
:101EF00031050CF0949AFF91EF91BF91AF919F91B2
:101F00008F917F916F915F914F913F912F910F90A2
:101F10000FBE0F901F90189550E060E070E027E032
:101F2000813D920708F051E02FE0813A920708F0D6
:101F300052E023E28932920708F053E026E3813B26
:101F4000920708F054E026E48135920708F055E046
:101F500028E8893B920708F056E0895D964D08F025
:101F600057E078948BB1992726E0969587952A9526
:101F7000E1F79C012170307080FFB9016F5F7F4FE6
:101F8000A89587E26031780768F321E04EE468E0C5
:101F9000852F0E94740E089589B1282F33278091D0
:101FA00090009927982F8827282B392B60E040E054
:101FB00050E0FA01E85CFE4F8591949182179307F7
:101FC00029F06F5F4E5F5F4F683098F3862F992737
:101FD0008330910509F1843091054CF481309105ED
:101FE000A9F082309105ACF4892B69F024C08530CA
:101FF0009105C1F08530910594F086309105A9F0E6
:102000000797B1F018C080EB94E0089580E699E05E
:10201000089580EC92E1089580E895E2089580E4C7
:1020200098E3089580E09BE4089580E096E90895A0
:1020300080E091EE089580E090E008950895482FA3
:1020400007C08091E606882391F4559A7894A89564
:102050008091E506282F33278091E606992701977E
:102060002817390791F38091E506873051F3809165
:10207000E506E82FFF27ED53F94F44A38091E506CD
:102080008F5F8093E5068091E506883010F010920E
:10209000E506559A80E090E008958091C306282FC8
:1020A00033278091C406281B310937FF02C0205E08
:1020B0003F4F203131050CF494989091C3068091E4
:1020C000C406981719F48FEF9FEF08958091C40606
:1020D000E82FFF27ED53F94F8281282F3327809176
:1020E000C4068F5F8093C4068091C406803210F0CE
:1020F0001092C406C90108950895882331F0809193
:10210000EF0681608093EF0608958091EF068E7F41
:102110008093EF06559A08950895E82F1092970638
:102120008091970680939606809196068093B906D3
:102130008091B9068093B80691E09093C20681B36E
:10214000886281BB8A981598939A92981D9882E02C
:1021500080939B009598E83008F0E92FFF27EE0F59
:10216000FF1FE85CFE4FA591B491653010F465E067
:1021700003C0693008F068E04F7D6550660F8B2F13
:10218000992787FD9A958F7080939800A093990066
:10219000453411F4606203C04F3409F460632230A7
:1021A00008F0686060939D0088EB80939A0080E05F
:1021B00090E008959091B8068091B906981739F08B
:1021C0000D9905C080919A00806280939A000895CD
:1021D00008951F920F920FB60F9211248F939F9321
:1021E000EF93FF939091B8068091B906981761F02C
:1021F00088B7806288BF0D9B0DC089B7806289BF98
:102200008091C20680FF06C080919A008F7D8093E6
:102210009A0014C08091B906E82FFF27EA56F94FBB
:1022200084A180939C008091B9068F5F8093B9064A
:102230008091B906883010F01092B906FF91EF91A5
:102240009F918F910F900FBE0F901F9018951F9226
:102250000F920FB60F9211248F9389B78F7D89BF8C
:1022600080919A00806280939A008F910F900FBEA8
:102270000F901F9018951F920F920FB60F92112476
:102280002F933F934F935F936F937F938F939F937E
:10229000AF93BF93EF93FF9380919606282F332738
:1022A00080919706992701972817390741F0809167
:1022B00096068F3179F480919706882359F480919E
:1022C00097068F5F8093970680919706803210F073
:1022D0001092970690919B0080919606E82FFF2719
:1022E000EA56F94F80919C008283828194FD0CC054
:1022F000809196068F5F8093960680919606803235
:1023000078F0109296060CC0882351F480939706BB
:102310008091970680939606959881E00E94A73C4D
:1023200080919606282F332780919706281B310924
:1023300037FF02C0205E3F4F213131050CF0959AE6
:10234000FF91EF91BF91AF919F918F917F916F918D
:102350005F914F913F912F910F900FBE0F901F9063
:102360001895482F0BC08091B9068823B1F480914D
:102370009A00806280939A007894A8958091B8061C
:10238000282F33278091B9069927019728173907F5
:1023900071F38091B806873031F38091B806E82F49
:1023A000FF27EA56F94F44A38091B8068F5F8093C8
:1023B000B8068091B806883010F01092B806809167
:1023C0009A00806280939A0080E090E00895809166
:1023D0009606282F332780919706281B310937FF4F
:1023E00002C0205E3F4F203131050CF4959890914A
:1023F000960680919706981719F48FEF9FEF08952E
:1024000080919706E82FFF27EA56F94F8281282FFF
:102410003327809197068F5F809397068091970668
:10242000803210F010929706C9010895089588230C
:1024300031F08091C20681608093C2060895809138
:10244000C2068E7F8093C20680919A00806280933C
:102450009A000895089587B3876087BBBB9888B3B7
:10246000896088BB1DB88EB18FB187E78DB908959B
:102470001F920F920FB60F9211242F938F939F9359
:10248000EF93FF932FB18091A802E82FFF27E85523
:10249000FD4F22838F5F8093A802883110F0109245
:1024A000A8029091C302E92FFF27E855FD4F248D24
:1024B00027FDC09A8091C202981759F0C098892FC1
:1024C0008F5F8093C302883110F01092C3022FB93E
:1024D00002C0C09A6F98FF91EF919F918F912F91B9
:1024E0000F900FBE0F901F9018958091C302282F58
:1024F00033278091C202281B3109C90147968831D0
:10250000910514F0C901019708950895282F6F9936
:1025100019C0C0988FB16F9A8091C2029091C30286
:10252000891711F42FB91CC0E92FFF27E855FD4F7B
:10253000848D8FB9892F8F5F8093C302883110F00B
:102540001092C3028091C202E82FFF27E855FD4F89
:10255000248F8F5F8093C202883110F01092C202E4
:1025600080E090E008958091A8022091A90282174E
:1025700019F48FEF9FEF0895E22FFF27E855FD4FE5
:102580008281482F5527822F8F5F8093A90288313F
:1025900010F01092A902CA0190700895089588233E
:1025A00011F0DD9A0895DD98089508950F931F9313
:1025B000CF93282FDE9B63C0882309F060C08091F1
:1025C000DE029091DF0253E0969587955A95E1F7E8
:1025D000182FC091DE02C770022FCF9901E09BB384
:1025E000892F8F7A8BBB94FF02C081E001C0822FBC
:1025F0000E94CF12A091DE02B091DF02412F552739
:102600006C2F7727C091890A002399F0FA01E55FC2
:10261000F44F20E830E002C0359527956A95E2F73F
:102620008081822B8083FA01E553F54F8081822BD4
:102630000EC0FA01E55FF44F80E890E002C0959586
:1026400087956A95E2F7982F9095808189238083FA
:102650009D012F5F3F4F3093DF022093DE028C2FCE
:10266000992744E0880F991F4A95E1F72817390701
:1026700058F0DC9A1092DF021092DE0205C022238D
:1026800011F0DE9A01C0DE98CF911F910F9108954D
:1026900000000000000000000895882341F08091B0
:1026A00065008460809365000E94481308958091BE
:1026B00065008B7F80936500089508959B01AC01B0
:1026C0008091F2069091F306A091F406B091F50680
:1026D00082179307A407B507A0F08091F2069091A6
:1026E000F306A091F406B091F506821B930BA40BA0
:1026F000B50B80509041A040B040A0F080E090E049
:1027000008958091F2069091F306A091F406B0919D
:10271000F506281B390B4A0B5B0B2050304F4F4FEF
:102720005F4F18F081E090E0089580E090E0089518
:102730000895EF92FF920F931F93AA27BB27E09073
:10274000F206F090F3060091F4061091F506E80EFB
:10275000F91E0A1F1B1F01C0A895C801B7010E94DE
:102760005E138823C9F31F910F91FF90EF90089596
:102770000F931F93CF93C82F162F042F80916500BE
:102780008D7F8093650080E00E944D138AB38F6037
:102790008ABB8BB3807F9C2F92959F70892B8BBBBC
:1027A000112321F080916500816003C08091650054
:1027B0008E7F8093650081E00E944D1380E00E942F
:1027C0004D13002329F088E090E00E9499130DC07A
:1027D0008BB3807FCF708C2B8BBB0E94481381E022
:1027E0000E944D13802F0E944D13CF911F910F9186
:1027F000089588E290E00E94991341E060E080E350
:102800000E94B81341E060E080E30E94B81341E009
:1028100060E080E30E94B81341E060E080E20E9443
:10282000B81388E20E941C1788E00E941C1781E000
:102830000E941C1786E00E941C178CE00E941C1747
:102840006CE372E080E00E94551864E172E081E080
:102850000E9455186CE172E082E00E94551864E015
:1028600072E083E00E94551864EF71E084E00E94FA
:1028700055186CEE71E085E00E94551864EE71E029
:1028800086E00E9455186CED71E087E00E945518B3
:1028900008951F920F920FB60F9211241F932F933A
:1028A0003F934F935F936F937F938F939F93AF93D8
:1028B000BF93EF93FF938091DC028F5F8093DC02E4
:1028C000282F237009F0F4C0869586958770992784
:1028D0008330910509F47CC0843091054CF481303B
:1028E000910551F182309105DCF5892B89F0E0C02A
:1028F0008530910509F4A2C0853091050CF49CC087
:102900008630910509F4CEC0079709F4CFC0D0C036
:102910008091F2069091F306A091F406B091F5062D
:102920000196A11DB11D8093F2069093F306A0932A
:10293000F406B093F50680C08091F2069091F306FC
:10294000A091F406B091F50681709070A070B070FF
:10295000892B19F00E942416ABC00E94E515A8C06F
:1029600081E00E94D6120E94420D833009F0A0C07F
:102970000E94831D2091F0063091F1068823E9F032
:102980002E5F3F4F3093F1062093F0060E94BA4F1E
:10299000FC019681992309F48BC08AE0989F9001ED
:1029A00011248091F0069091F1068217930708F4A4
:1029B0007FC081E00E94030D7BC02115310509F421
:1029C00077C0215030403093F1062093F00670C05C
:1029D0008091DD02882309F46BC08AB3807F8ABBB3
:1029E000822F0E944D138091650082608093650064
:1029F000809165008E7F809365000000000081E07B
:102A00000E944D1319B380E00E944D131295107F60
:102A10000E94481381E00E944D1389B38F70182BD8
:102A200080E00E944D13812F992787FD909588277C
:102A3000990F881F992733C0822F35C06091DD021E
:102A40006623B1F59091F6068091F706981789F004
:102A50001091F706E12FFF27EA50F94F82811F5F9F
:102A6000103108F0162F803891F48091F606811706
:102A700019F480E090E013C0E12FFF27EA50F94FEE
:102A800082811F5F103108F0162F462F02C0462F9B
:102A900061E00E94B8131093F70681E090E0809304
:102AA000DD0206C081E00E94D61202C00E94B91663
:102AB000FF91EF91BF91AF919F918F917F916F9116
:102AC0005F914F913F912F911F910F900FBE0F90EB
:102AD0001F90189510927D0017BE11BE89E683BF26
:102AE00087B7816087BF82EF8FBD3AE13EBD4FEC73
:102AF00050E057BD46BD85EB90E09BBD8ABD99BDBA
:102B000088BD22EC20938B0030938A005093810083
:102B10004093800090938700809386000E94BA4F74
:102B2000FC0180858093890A0895EF92FF920F93AC
:102B30001F93AA27BB27E090F206F090F3060091BE
:102B4000F4061091F506E80EF91E0A1F1B1F02C0BD
:102B50000E94460DC801B7010E945E138823C1F38D
:102B60001F910F91FF90EF900895282F220F611170
:102B70002160822F83708150823028F424FF02C0AC
:102B80002E6001C0217F822F992708959091E20243
:102B9000E92FFF27EE51FD4F8283892F8F5F8093AE
:102BA000E202883010F01092E2029091E3028091EC
:102BB000E202981741F4892F8F5F8093E3028830F7
:102BC00010F01092E302089508950F931F9311B12E
:102BD000812F8074682F8091E0020E94B515082F24
:102BE0008093E0021078612F8091E1020E94B51578
:102BF0008093E102007C807C003829F4882339F03E
:102C0000803C61F408C0003449F4803C11F484E154
:102C100003C0882319F485E10E94C6151F910F9106
:102C20000895843118F080E090E0089520E030E0CD
:102C3000E82FFF27E451FD4F8081882311F021E028
:102C400030E0C90108950895FF920F931F93CF9329
:102C500080910503E82FFF27E050FD4F008113B35B
:102C60001083FF2480910503E82FFF27EE0FFF1F3D
:102C7000EE0FFF1FEF0DF11DE85BFE4FC49110FD3D
:102C800042C000FF14C0C23129F481E10E94111634
:102C9000882331F48C2F0E94C615C43108F054C02B
:102CA000EC2FFF27E451FD4F81E080834DC0C431FC
:102CB00008F04AC0EC2FFF27DF01A451BD4F9C91C3
:102CC0009F5F9C93992311F49F5F9C93E131F105E1
:102CD000DCF1E331F1056CF07397B1F58091FF02FF
:102CE000853690F18CE10E94C61581E08093FF0249
:102CF0002BC08091FD02893738F18091FE0289371F
:102D000018F185E01FC0C43128F4EC2FFF27E451EF
:102D1000FD4F108200FD18C08C2F80680E94C615E0
:102D20000E94420D853081F4C13121F482E10E947C
:102D3000111605C0C23141F481E10E9411168823A9
:102D400019F486E00E94030D16950695F39483E02E
:102D50008F1508F087CF809105038F5F809305035F
:102D6000853010F010920503CF911F910F91FF90C5
:102D7000089590910503943029F485B3806F85BB45
:102D800097980895979A85B38F7020E130E002C03C
:102D9000220F331F9A95E2F7922F9095907F892BFF
:102DA00085BB089508958091E2022091E302821785
:102DB00019F48FEF9FEF0895E22FFF27EE51FD4F9B
:102DC0008281482F5527822F8F5F8093E3028830BE
:102DD00010F01092E302CA0108950895CF93C82F0E
:102DE00006C08091F706882389F40E948052809162
:102DF000F606282F33278091F70699270197281781
:102E0000390799F38091F6068F3059F3F894809141
:102E1000F606E82FFF27EA50F94FC2838091F606A5
:102E20008F5F8093F6068091F606803110F0109245
:102E3000F6067894CF9108951F93182F80E80E948A
:102E4000EE16812F0E94EE161F9108958295880F2D
:102E5000880F807C860F80680E941C1708950E944E
:102E600026178EE00E941C1708958CE00E941C1704
:102E70000895FF920F931F93CF93F82E6091190737
:102E8000809118070E942617C0E008E017E08091A3
:102E90001A07C81778F4FF2021F0F80161918F011B
:102EA00001C060E282E00E947E18CF5F80911A0725
:102EB000C81788F3CF911F910F91FF9008959093B9
:102EC000230780932207892B89F170932107609350
:102ED0002007CB01AA27BB272091F2063091F306E9
:102EE0004091F4065091F506280F391F4A1F5B1FC9
:102EF00020931C0730931D0740931E0750931F0714
:102F000080911B078E7F80931B072115310541059A
:102F1000510561F42F5F3F4F4F4F5F4F20931C07C8
:102F200030931D0740931E0750931F07089508957F
:102F3000AF92BF92CF92DF92EF92FF920F931F93C7
:102F4000CF93DF93D82EC62EEA0188E0E82E87E0E3
:102F5000F82E109223071092220781E08D1568F158
:102F6000EFE0E61750F14115510539F1FA010190F2
:102F70000020E9F731970E2F041B013108F000E122
:102F80006C2D8D2D0E9426175701002361F0102F04
:102F90008881F50181935F018991682F82E00E9409
:102FA0007E181150A9F7F701D08AC18A028B64EF0D
:102FB00071E089E397E10E945F17DF91CF911F9144
:102FC0000F91FF90EF90DF90CF90BF90AF9008955A
:102FD000CF93DF93CDB7DEB7A0970FB6F894DEBFDF
:102FE0000FBECDBF282FDE01119690E0FA014F5F92
:102FF0005F4F8491882321F08D939F5F9F31B0F3C1
:103000001C92AE014F5F5F4F822F0E949817A096CF
:103010000FB6F894DEBF0FBECDBFDF91CF910895FC
:103020008091220790912307892BA9F160911C07B9
:1030300070911D0780911E0790911F070E945E13DB
:10304000882349F180911B07E0912207F091230723
:103050008170099580911B0791E0892780931B0758
:1030600080912007909121079C014427552780914A
:10307000F2069091F306A091F406B091F506820F46
:10308000931FA41FB51F80931C0790931D07A09347
:103090001E07B0931F0708950895109223071092FA
:1030A000220781E00E941C1708950F931F93CF936E
:1030B000DF93EB018830C0F4992723E0880F991F34
:1030C0002A95E1F780640E941C1707E010E0FE01DA
:1030D000219684910E94EE160150104017FFF7CF01
:1030E00060E0862F0E942617DF91CF911F910F91EC
:1030F0000895813308F080E381BF089599278130D6
:10310000910539F1823091051CF4892BF1F0089575
:10311000029711F567FF15C0643E31F0663F41F03C
:103120006C3F51F0643C11F461EE0BC0663D11F44C
:103130006FEE07C06C3D11F465EF03C06F3D09F4FD
:1031400062EE862F0E94EE160895862F0E941F10B1
:103150000895862F0E94B111089508951F93CF936B
:10316000DF93182FEB01FB016491662349F0812F57
:103170000E947E182196FE018491682F8823B9F75A
:10318000DF91CF911F9108951F93CF93DF93182F55
:10319000EB018881882341F08991682F812F0E945B
:1031A0007E1888818823C1F7DF91CF911F91089500
:1031B0001F93CF93DF93CDB7DEB7C055D0400FB686
:1031C000F894DEBF0FBECDBF67961FAD67976996B7
:1031D0008EAD9FAD6997AE01475A5F4FBC01CE01DE
:1031E00001960E941267BE016F5F7F4F812F0E9480
:1031F000C418C05BDF4F0FB6F894DEBF0FBECDBF63
:10320000DF91CF911F9108951F93CF93DF93CDB797
:10321000DEB7C055D0400FB6F894DEBF0FBECDBFAD
:1032200067961FAD679769968EAD9FAD6997AE01A2
:10323000475A5F4FBC01CE0101960E943B67BE0119
:103240006F5F7F4F812F0E94C418C05BDF4F0FB6A6
:10325000F894DEBF0FBECDBFDF91CF911F910895CF
:1032600099278130910571F0823091051CF4892BEA
:1032700031F00BC0029749F40E94D31608950E94C2
:103280004D1008950E94E71108958FEF9FEF089564
:103290000895FC018F3F910519F010F0E0E0F0E097
:1032A000E45AFD4F84919927089590E08F3010F0F3
:1032B0008EE001C081118F5F442311F028E001C02E
:1032C000242F77276230710581F06330710524F473
:1032D0006130710541F00EC06330710541F064301A
:1032E000710539F007C0236005C0246003C0266063
:1032F00001C02760281729F4442311F02AE001C0F7
:1033000025E043E050E0990F990F80FD926020FD89
:103310009160869526954150504057FFF4CF892FF4
:10332000992708959C01FB018F37910528F48F7729
:10333000808388E090E00895832F9927806C8183B3
:10334000208380E190E008950895FC014081242FBE
:1033500033278181992701972817390729F04F30A2
:1033600031F48181882319F481E090E0089580E0B0
:1033700090E0089508951F9384E297E00E94A519B4
:10338000182F86E997E00E94A519182B812F9927FD
:103390001F910895AF92BF92CF92DF92EF920F9359
:1033A0001F93CF93DF93EC016B015A01122F809191
:1033B0003803882369F40B3059F00C3049F0CB0105
:1033C0000E948F25992783709070892B09F452C031
:1033D000CE010E94A519282F882319F080E090E0E3
:1033E0004BC088819927FC0173E0EE0FFF1F7A958F
:1033F000E1F7E81BF90BEC0FFD1FC282D382888135
:103400009927FC0163E0EE0FFF1F6A95E1F7E81BC7
:10341000F90BEC0FFD1FA482B58288819927FC016E
:1034200053E0EE0FFF1F5A95E1F7E81BF90BEC0F85
:10343000FD1F178388819927FC0143E0EE0FFF1FD2
:103440004A95E1F7E81BF90BEC0FFD1F0683888115
:103450009927FC0133E0EE0FFF1F3A95E1F7E81BD7
:10346000F90BEC0FFD1FE08688818F5F8883803128
:1034700008F0288381E090E0DF91CF911F910F91B8
:10348000EF90DF90CF90BF90AF9008959F92AF9252
:10349000BF92CF92DF92EF92FF920F931F93CF9341
:1034A000DF93EC015B016A01922EF02E1E2D0E942B
:1034B000420D8250833048F5209761F4E12E0F2DA4
:1034C000292DA601B50186E997E00E94461AC4E2BB
:1034D000D7E0EDCF80913803882321F087E0C6390B
:1034E000D80799F0F894E12E0F2D292DA601B501EA
:1034F000CE010E94CA197894882329F485E090E0CF
:103500000E949913EFCF10923B03DF91CF911F914F
:103510000F91FF90EF90DF90CF90BF90AF909F9072
:103520000895EF920F93CF93DF93EC01E62E0E9464
:103530004B24FC01892B89F080859927837090703A
:10354000039711F423E001C026E001E040E050E0E1
:10355000BE0184E297E00E94461A81E090E0DF918C
:10356000CF910F91EF900895EF920F93CF93DF9348
:10357000EC010E944B24FC01892BA9F0808599273E
:1035800083709070039731F486818F67E82E01E095
:1035900024E003C0EE2402E02BE040E050E0BE0156
:1035A000CA010E94461A81E090E0DF91CF910F910D
:1035B000EF900895EF920F93CF93DF93EC010E9469
:1035C0004B24FC01892B81F08085992783709070B2
:1035D0000197029748F4EE2402E02BE040E050E02F
:1035E000BE01CA010E94461A81E090E0DF91CF91AE
:1035F0000F91EF900895EF920F93CF93DF93EC012B
:103600000E944B24FC01892B79F0808599278370D7
:103610009070019749F4EE240AE024E040E050E085
:10362000BE01CA010E94461A81E090E0DF91CF916D
:103630000F91EF900895AF92BF92CF92DF92EF92E9
:103640000F93CF93DF935C016B010E944B24EC013D
:10365000892B09F451C08885992783709070823036
:10366000910571F5D7FE05C06E81888199810E9410
:10367000911AC0FE09C0EE8006E024E040E050E070
:10368000B501CA010E94461AC1FE09C0EE8007E0DA
:1036900024E040E050E0B501CA010E94461AC2FE93
:1036A00009C0EE8008E024E040E050E0B501CA0126
:1036B0000E94461AC3FE20C0EE8009E024E016C036
:1036C0000397D1F4C6018F709078892B49F0EE24CE
:1036D00003E024E040E050E0B501CA010E94461A30
:1036E0008C2D807F49F0EE2404E0202F40E050E054
:1036F000B501CA010E94461A81E090E0DF91CF91A6
:103700000F91EF90DF90CF90BF90AF900895EF9220
:103710000F931F93CF93DF93EC01162F0E948F25F9
:1037200083708150823050F4EE2402E0212F40E07B
:1037300050E0BE0184E297E00E94461A81E090E0EA
:10374000DF91CF911F910F91EF900895EF920F931A
:10375000E62E662319F0EE240CE001C00BE024E015
:1037600040E050E0BC01CA010E94461A81E090E0AE
:103770000F91EF900895EF920F93262FEE240DE016
:1037800040E050E0BC01CA010E94461A81E090E08E
:103790000F91EF900895EF920F93EE240EE0282FF3
:1037A00040E050E0BA01CA010E94461A81E090E070
:1037B0000F91EF900895EF920F93FC0180913803E1
:1037C000882319F480E090E013C06770862F806F23
:1037D000442311F0862F886FE82E01E121E040E0BC
:1037E00050E0BF0184E297E00E94461A81E090E039
:1037F0000F91EF900895EF920F93FC0180913803A1
:10380000882319F480E090E013C06770862F806EE3
:10381000442311F0862F886EE82E01E121E040E07C
:1038200050E0BF0184E297E00E94461A81E090E0F8
:103830000F91EF900895EF920F93FC01E62E809187
:103840003803882319F480E090E00BC002E121E006
:1038500040E050E0BF0184E297E00E94461A81E018
:1038600090E00F91EF900895EF920F93FC01E62EF8
:1038700080913803882319F480E090E00BC003E1C5
:1038800021E040E050E0BF0184E297E00E94461A48
:1038900081E090E00F91EF900895EF920F93FC017B
:1038A000E62E80913803882319F480E090E00BC065
:1038B0000FE021E040E050E0BF0184E297E00E9489
:1038C000461A81E090E00F91EF900895EF920F93E8
:1038D000FC01E62E80913803882319F480E090E003
:1038E0000BC000E121E040E050E0BF0184E297E03E
:1038F0000E94461A81E090E00F91EF900895EF92B8
:103900000F93FC01E42E04E124E0AB01BF0180E051
:1039100090E00E94461A81E090E00F91EF900895A8
:10392000982F882391F01092250780912507809386
:10393000240781E080933A0380913A03809338030F
:10394000BD9A87B7846087BF089587B78B7F87BF8D
:1039500090933803BD98C59808950895EF920F93FA
:10396000E0903803EE2069F5882359F1E0922507AD
:10397000809125078093240788E1E8E0F3E0119225
:103980008A95E9F70EE022E040E050E0BA0184E2D7
:1039900097E00E94461A81E080933A038BE390E01F
:1039A00099BD88BD88B599B59BBD8ABD87E790E074
:1039B00097BD86BD1DBC1CBC87B7846087BFBE9AFF
:1039C00005C0BE98C69887B78B7F87BF0F91EF90D1
:1039D0000895EF920F93E0903803EE2071F588235D
:1039E00061F1E0929707809197078093960788E1AD
:1039F000E0E2F3E011928A95E9F70EE022E040E080
:103A000050E0BA0186E997E00E94461A8BE390E005
:103A1000909387008093860087E790E090938100E1
:103A200080938000109289001092880080917D0020
:103A3000846080937D00139A07C013981B9880912F
:103A40007D008B7F80937D000F91EF90089580E043
:103A50000E94901C81E00E94AE1C81E00E94E91C43
:103A600080916200846080936200089580E00E94EB
:103A7000901C809162008B7F8093620080E00E94A6
:103A8000AE1C80E00E94E91C10923A0381E00E9483
:103A9000FF61089580E00E94AE1C80E00E94E91C56
:103AA00081E00E94FF61809162008B7F80936200C1
:103AB00088E1E8E0F3E011928A95E9F783E08093EA
:103AC0001A038FEF809308038BE390E099BD88BDC4
:103AD00088B599B59BBD8ABD87E790E097BD86BD47
:103AE00081E00E94901C82E090E00E94951508956C
:103AF0000E94BA4FFC01808182FF02C0C79A0895DC
:103B0000C798089508950E94BA4FFC01808182FFF2
:103B100007C080E090E0B79907C081E090E0089589
:103B200086B3992780789070089508950E94420D79
:103B3000833021F00E94420D843021F480913B03B8
:103B40009927089581E090E00895089580913903C0
:103B50009927089510923903089590935003809304
:103B60004F03089580914D0390914E03089580E195
:103B7000ECE3F3E011928A95E9F710924C0310926E
:103B80004E0310924D038FEF9FE790935003809365
:103B90004F03089578941F920F920FB60F9211243D
:103BA0002F933F934F938F939F93EF93FF93809126
:103BB0004C03883010F010924C0380914C03E82F96
:103BC000FF27EE0FFF1FE45CFC4F24B135B12083CB
:103BD00031838F5F80934C0310924E0310924D03FC
:103BE00020E030E047E0ECE3F3E081919191280F91
:103BF000391F415047FFF9CF30934E0320934D03B7
:103C000080914F0390915003821793071CF481E039
:103C100080933903FF91EF919F918F914F913F9145
:103C20002F910F900FBE0F901F9018956F927F925B
:103C30008F929F92AF92BF92CF92DF92EF92FF92BC
:103C40000F931F93CF93DF93EC015B018824665998
:103C5000774011F471E0872EF501908181819817EA
:103C600009F08AC0882019F481E080933B03809199
:103C70003803882339F0EE240DE021E040E050E0E5
:103C8000BA0177C0882019F00E94752502C00E94F1
:103C90001A256C01009731F4EE2401E022E0AC011A
:103CA000BC0167C0FC0180859927837090708230C9
:103CB000910581F0833091051CF4019721F05CC0DF
:103CC0000397D1F159C0F601E68001E022E040E01F
:103CD00050E04DC0F6011681E12E01E022E040E007
:103CE00050E060817181C5010E94CA190E941625A9
:103CF0008370482F55274130510591F042305105CE
:103D000024F44115510541F037C04230510559F0B6
:103D10004330510571F030C0E12E06E022E026C0AC
:103D2000E12E07E002C0E12E08E022E040E050E092
:103D30001DC0E12E09E0F9CFF601E68001E0202F59
:103D400040E050E060817181C5010E94CA190E9463
:103D500016259927AC014170507080FF04C0EE24F5
:103D600003E021E0E3CFEE2404E021E0F6016081EE
:103D70007181C5010E94CA19F50181819927FC0151
:103D800063E0EE0FFF1F6A95E1F7E81BF90BEA0D00
:103D9000FB1DE280F380F50181819927FC0153E04E
:103DA000EE0FFF1F5A95E1F7E81BF90BEA0DFB1D1B
:103DB00064807580F50181819927FC0143E0EE0F55
:103DC000FF1F4A95E1F7E81BF90BEA0DFB1D068181
:103DD000F50181819927FC0133E0EE0FFF1F3A9531
:103DE000E1F7E81BF90BEA0DFB1D9084F5018181D9
:103DF0009927FC0123E0EE0FFF1F2A95E1F7E81B4E
:103E0000F90BEA0DFB1D2781215027832223B1F4F2
:103E1000F50181819927FC0113E0EE0FFF1F1A9530
:103E2000E1F7E81BF90BEA0DFB1D2683F501818103
:103E30008F5F81838181803108F02183802F8B50B7
:103E4000823070F40E94BA4FFC01808181FF03C070
:103E5000B3E0BB2E02C0A1E0BA2ECC24DD2408C002
:103E600010913803112331F0CC24DD24F3E0BF2E70
:103E700010E014C0C7010E944B246C01009731F080
:103E8000192DFC01B084F3E0BF2206C0E1E0BE2E94
:103E90000E3011F473E0B72E811010788B2D992716
:103EA000813091050CF442C28330910524F00397D0
:103EB00009F406C13BC2C7010E944919982F829597
:103EC0008695869583708A83292F220F220F298356
:103ED00061E0A62EAA8A82E1888B82E0898BC114D8
:103EE000D10449F1F6018481958197FF02C02360D6
:103EF0002983812F99278F779070892BE1F0F60124
:103F000080850E9403280F97B4F01F5FF60180851B
:103F10000E941124892B29F410FF03C089818A256E
:103F20008983212F2078812F99278F719070959503
:103F30008795122F182B802F99278730910509F428
:103F40008FC0883091059CF48230910509F47DC0C2
:103F50008330910524F4019709F43FC0E7C1833011
:103F6000910509F43AC0069709F474C0DFC18A309C
:103F7000910509F48BC08B30910544F4883091058C
:103F800009F478C0099709F47BC0D0C10D970CF0F3
:103F9000CDC1C70143E0969587954A95E1F79070AA
:103FA00001960E944919982F82958695869583706F
:103FB0008A83990F990F99830B3011F418820AC0E4
:103FC000F7E0EF22FF2484E592E0E80EF91EF70106
:103FD0008491888382E08A8B3AC081E090E017FD6B
:103FE000892F212F2F702F3010F02EE001C02111CA
:103FF0002F5FF1E0BF1661F443E050E0990F990F95
:1040000020FD936026954150504057FFF7CF1BC0CD
:10401000882331F0283010F085E007C08DE005C01E
:10402000283010F48AE001C082E043E050E0990FAC
:10403000990F20FD926080FD9160269586954150F4
:10404000504057FFF4CF988371C180EC888384E09F
:10405000898B6CC1F60184818170482F61E005C0B5
:10406000F60184818270482F62E0812F8F770E9451
:10407000551924C0F60184818470482F63E0F5CF80
:10408000F60184818870482F64E0EFCFC7010E9459
:104090004919982F82958695869583708A83990F02
:1040A000990F9360998382E08A8BF60184819581D0
:1040B0008F7090708C5B9D4FFC018491888336C11A
:1040C00083E08A8B31E0B32EB98A88E1888B802F18
:1040D00099278D30910509F4D5C08E309105BCF437
:1040E0008430910509F4B6C08530910544F48130DF
:1040F000910509F43DC0039709F496C009C18530C4
:10410000910509F4B4C00B970CF402C10FC08231C1
:10411000910524F40F970CF0C5C0BFC08431910500
:104120000CF4D8C0449709F4E4C0F2C088E090E0F1
:10413000E80EF91EC70123E0969587952A95E1F7C9
:104140008F7380688A83C7018095909515E0969556
:1041500087951A95E1F7282F207720688E2D877094
:10416000282B29830C3009F0D3C028602983D0C0C4
:10417000F601808599278C7090700897B9F48FE3C9
:104180008A83812F99278F779070009731F08F372E
:10419000910511F4117801C01F5F1983CE010396B8
:1041A000BC01C7010E949219885EB1C017FF02C00E
:1041B00080E601C080E48983F60180850E9403289F
:1041C000212F3327BE016E5F7F4F0F97B4F0C901D7
:1041D0008F779070009731F08F37910511F412E0CE
:1041E00001C01D5F812F86958F709981982B9983CF
:1041F00010FF2BC09061998328C0C9018F77907000
:10420000009731F08F37910511F411E001C01F5F65
:104210001F702981212B2983F6018481958197FFC5
:1042200014C02061298311C080E88983F6012481AC
:104230002F70822F806889838481958197FF02C0C7
:1042400020692983CE010296BC01C7010E94921900
:10425000805F5DC080EA8983F60184819581B4E046
:1042600096958795BA95E1F78F70806B09C080EAC3
:104270008983F60184819581892F99278F70806ABF
:104280008983E0CF1982CE010296BC01C7010E944A
:104290009219805F888BB98A3BC08FEF8A8319821D
:1042A00081E025C0013111F488E707C0003111F425
:1042B00084E703C00F3011F48CE78B838F2D99278F
:1042C000982F93708B81892B8B83EA82998280E26D
:1042D000888B0CC080E78A83023111F488E78A83D7
:1042E0008E2D87709A81982B9A8399828AE0898B88
:1042F0000FC0872D992783708C6E8B836A82998279
:10430000CE010496BC01C7010E949219805E888B81
:1043100020E09889969596959695915031F0FE01FA
:10432000E90FF11D80812827F8CF28838A898330FF
:1043300011F010923A03DF91CF911F910F91FF90EE
:10434000EF90DF90CF90BF90AF909F908F907F9035
:104350006F900895CF93DF93DC01FC01848988235B
:1043600019F42589222361F021E0882321F081506E
:10437000FD01848B21C0FD0185898150858B1CC086
:10438000FD018289833019F487898823A9F4FD010E
:104390009389892F869586958695E80FF11D8081F2
:1043A000282F3327892F99278770907002C0359561
:1043B00027958A95E2F72170FD013289832F99278D
:1043C0008230910531F083309105CCF0039721F0D4
:1043D00016C0CBE6D0E015C0222319F0C7E7D0E025
:1043E00002C0CEECD0E0FD018389882351F4868998
:1043F000882339F482E0858B81E0868B2BC0C7ED62
:10440000D0E0FD018389882329F58589882311F56A
:104410008189882399F480913A038823D9F4809183
:1044200038038823B9F481E00E94DB4F882319F018
:10443000C35BDF4E0FC0CD5ED94F0CC0832F9927D1
:104440008130910529F0029729F4C857DD4F02C049
:10445000C05FDA4FCE01DF91CF910895DC01FC01FE
:104460008489882319F48589882311F021E02BC0E1
:10447000FD013389932F9150938B8289833069F4A6
:104480002789222351F4892F9927877090700797E5
:1044900021F481E0878B338B16C0FD01178A938945
:1044A000892F869586958695E80FF11D8081282FA6
:1044B0003327892F99278770907002C035952795EB
:1044C0008A95E2F72170FD01828999278230910552
:1044D00049F0833091051CF4019761F01BC00397EC
:1044E00089F018C0222319F08DE590E008958CE042
:1044F00090E00895222319F08CEB90E008958AE172
:1045000090E00895222319F08BE390E0089587E668
:1045100090E008958BE390E008950895FC01808970
:10452000838B8189823010F482E0818B8289992784
:1045300081309105B4F0833091051CF0039761F050
:1045400010C081E00E94DB4F882319F08DE490E1D8
:10455000089583E196E0089580E1848B82E390E002
:10456000089582E390E0089508951F920F920FB688
:104570000F9211241F932F933F934F935F936F9349
:104580007F938F939F93AF93BF93CF93DF93EF93DB
:10459000FF9380913803882331F00E94A61D882361
:1045A00011F010921903809106038823A1F08091E5
:1045B0003A03882329F08BE390E099BD88BD02C0BF
:1045C00019BC18BC8BE390E09BBD8ABD87E790E0E7
:1045D00097BD86BD5EC0C8E0D3E0CE010E94AA218F
:1045E000AC019C01255030408CB59DB582179307D6
:1045F00018F457BD46BD0EC08CB59DB5C29697BD8B
:1046000086BDCE010E948E222CB53DB5280F391FE4
:1046100037BD26BD80911B03882381F510911D03B2
:10462000112361F580911903882381F481E080933F
:10463000060386B7846086BF789464E277E088E0FA
:1046400093E00E94161EF8941092060380911903BD
:104650008150898B809118038B8B80911A03833052
:1046600049F480913803882311F084E101C080E18E
:104670008C8B01C01C8B1D8A1F8A1E8A88E093E0E8
:104680000E942E2299279BBD8ABD8AB59BB599BDF4
:1046900088BDFF91EF91DF91CF91BF91AF919F9135
:1046A0008F917F916F915F914F913F912F911F91CA
:1046B0000F900FBE0F901F9018951F920F920FB67C
:1046C0000F9211241F932F933F934F935F936F93F8
:1046D0007F938F939F93AF93BF93CF93DF93EF938A
:1046E000FF93809107038823B1F080913A038823D8
:1046F00039F08BE390E0909387008093860004C0AC
:10470000109287001092860087E790E090938100D6
:104710008093800064C0C0E2D3E0CE010E94AA2151
:10472000AC019C0125503040809188009091890017
:104730008217930728F4509381004093800016C09D
:104740008091880090918900C29690938100809317
:104750008000CE010E948E22209188003091890035
:10476000280F391F309381002093800080913303FC
:10477000882361F510913503112341F580913103B0
:10478000882391F481E08093070380917C0084600A
:1047900080937C00789466E977E080E293E00E9461
:1047A000161EF89410920703809131038150898B73
:1047B000809130038B8B80913203833019F480E138
:1047C0008C8B01C01C8B1D8A1F8A1E8A80E293E09D
:1047D0000E942E2299279093870080938600FF9154
:1047E000EF91DF91CF91BF91AF919F918F917F9189
:1047F0006F915F914F913F912F911F910F900FBE3D
:104800000F901F90189580E892E0E8E0F8E0119290
:104810000197E9F710925203109251031092880AFF
:1048200008958F7020E030E08550823010F421E050
:1048300030E0C90108950F931F93CF93DF93CDB755
:10484000DEB724970FB6F894DEBF0FBECDBF8FEF53
:104850009FEFAFEFBFEF89839A83AB83BC8300E206
:1048600010E044E050E0B801CE0101960E9486625B
:104870000E94460D0C5F1F4F8FE00D3F180788F315
:1048800024960FB6F894DEBF0FBECDBFDF91CF9157
:104890001F910F9108959C01009741F408958AE0BB
:1048A000A89FC0011124885F974F0895A0E0B091A0
:1048B000880AAB17A0F440E050E0BA01FA01E60F15
:1048C000F71FE85FF74F808191818217930739F3D3
:1048D000AF5F6F5F7F4F475F5F4FAB1778F380E04D
:1048E00090E008950895CF92DF92EF92FF920F9398
:1048F0001F93CF93DF93CDB7DEB723970FB6F8940E
:10490000DEBF0FBECDBF7C016C010894C108D10889
:104910008FEFC81687E2D806A0F5C7010E944B2486
:104920008C01892B09F072C02091880A203450F440
:104930008AE0289F80011124085F174F2F5F209382
:10494000880A22C008E018E0B80120E030E0A901A0
:10495000AFE3F901E40FF51FE85FF74F9185F80128
:104960008185891708F48B01A1504F5F5F4F275F46
:104970003F4F665F7F4FA7FFECCFF801818588230B
:1049800019F480E090E043C0F801E082F182FFEF8B
:10499000CF16F7E2DF06E0F480E2E82EF12CA895CE
:1049A00043E050E0B701CE0101960E946A6229817E
:1049B0003A81F8018081918128173907C9F084E094
:1049C00090E0E80EF91E9DEFE9169FE0F90638F336
:1049D000F801808191818F3F910519F010F083E0FB
:1049E0000BC088E00E94DB4F882321F083E003C0E6
:1049F0008B8101C082E0F801808780E8F80186831E
:104A0000148215821282138211861782C80123969E
:104A10000FB6F894DEBF0FBECDBFDF91CF911F91CF
:104A20000F91FF90EF90DF90CF9008958091530306
:104A300099270895EF92FF921F93CF93DF93909160
:104A4000880A992319F480E090E049C080915103CD
:104A50008F5F80935103891738F0809153038F5FE4
:104A60008093530310925103909151038AE0989FD1
:104A7000E0011124C85FD74F8091530399278770B5
:104A80009070892BA9F41E81E12EFF24C7018F7736
:104A90009070892B69F088850E941124892B41F040
:104AA000E0FC06C01F5F612F888199810E94911AE6
:104AB00080915303992787709070049751F48885EB
:104AC000992783709070019721F4888199810E94C1
:104AD000FB1A89858F3F11F08F5F8987CE01DF91A7
:104AE000CF911F91FF90EF9008959091880A99239C
:104AF00019F480E090E00895809152038F5F8093D5
:104B00005203891710F010925203909152038AE0D9
:104B1000989FC0011124885F974F089508950E94BF
:104B20004B24FC01009709F4089580859927089586
:104B300008950E944B24FC01009709F40895868192
:104B40009927089508950E944B24FC01009709F4C9
:104B500008958481958108950895BF92CF92DF9240
:104B6000EF92FF920F931F93CF93DF93CDB7DEB7F2
:104B700023970FB6F894DEBF0FBECDBF7C01B62ED3
:104B80000E947324FC01892BB1F180858B1599F16A
:104B9000B08611869FEFC92ED92E00E210E0A895AD
:104BA00043E050E0B801CE0101960E946A6289811B
:104BB0009A818E159F0511F468010DC0D7FE05C0BE
:104BC00028E28030920708F068010C5F1F4F2FE049
:104BD0000D3F120720F38E159F0511F0D7FC0BC077
:104BE000BB82E982FA82A89544E050E0B601CE018A
:104BF00001960E94866223960FB6F894DEBF0FBE20
:104C0000CDBFDF91CF911F910F91FF90EF90DF907B
:104C1000CF90BF900895CF92DF92FF920F931F9392
:104C2000CF93DF93EC01F62E142F892B09F47BC070
:104C300088850E940328482F5885752F73708F2D03
:104C400099278F779070242F3327281739071CF462
:104C500020E8F222F42A6E816F1509F464C01986E7
:104C6000112319F08F8181608F838F2D9927807890
:104C70009070C62EDD24960120783070821793073D
:104C800071F1C6018F779070009711F020E8F22241
:104C90007330B1F4892BD1F4852F99278C709070E3
:104CA0000897E9F48F2D99278F779070892BB9F4A5
:104CB0008F2D8160682F888199810E94911A0FC081
:104CC000892B49F0888199810E94911A8881998164
:104CD0000E94B41A04C0888199810E94DA1AFE8267
:104CE0000F2D1127C8018F779070892BB9F0888517
:104CF0000E941124892B91F000FD03C08F2D8F5F3E
:104D000008C00894C108D1080C151D0539F48F2D71
:104D10008150682F888199810E94911A6F2D888116
:104D200099810E94911ADF91CF911F910F91FF906D
:104D3000DF90CF900895FF920F931F93CF93DF934F
:104D4000EC01162FF42E0E94420D833009F01078EA
:104D5000CE010E947324EC010E814F2D612F0E9421
:104D60000B268A819B810097B1F00E947324EC018D
:104D70008E81282F332720783070802F99278078D4
:104D800090702817390711F080E818274F2D612FF0
:104D9000CE010E940B26DF91CF911F910F91FF90C2
:104DA0000895EF92FF920F931F93CF93DF93EC013F
:104DB0007B01892BE1F10C811D8106171707B9F1E1
:104DC0001986442319F08F8181608F83EC82FD82E4
:104DD00088859927837090708130910531F08130FA
:104DE00091052CF104971CF51BC0980120703078B8
:104DF000C701807090782817390729F06E81888163
:104E000099810E94911A0F7010708FE0E822FF24A0
:104E10000E151F0561F0888199810E94FB1A07C059
:104E20000E251F25B801888199810E941B1BDF91E7
:104E3000CF911F910F91FF90EF900895FF920F93E4
:104E40001F93CF93DF938B01F42E0E947324EC0108
:104E5000892B49F18A819B81892B01F1C8018F70CF
:104E60009F7B4F2DBC01CE010E94D1268A819B8160
:104E70000E947324EC01892BB1F0C80180709074FA
:104E8000880F991F007F107024E0169507952A95CA
:104E9000E1F7802B912B4F2DBC0102C04F2DB801A3
:104EA000CE010E94D126DF91CF911F910F91FF90EB
:104EB0000895EF92FF920F931F93CF93DF937C019E
:104EC0008B010E947324EC01892B61F0C8010E94C0
:104ED0007324FC01892B31F00A831B831986E2823B
:104EE000F3821186DF91CF911F910F91FF90EF9088
:104EF0000895009759F00E947324FC01892B31F02A
:104F000082819381128213821186F3CF08950895CE
:104F1000EF92FF920F931F93CF93DF93CDB7DEB73E
:104F200026970FB6F894DEBF0FBECDBF7C010E945E
:104F30004B248C01892BD9F0B701CE0101960E9438
:104F4000E751F801448155816681CE0101960E94A6
:104F5000CA51AE014F5F5F4F6AE08FEF0E946A5205
:104F6000F801448155816681C7010E947428269604
:104F70000FB6F894DEBF0FBECDBFDF91CF911F916A
:104F80000F91FF90EF9008951F93CF93DF9310E060
:104F9000C8E0D8E09091880A1917F0F48985899FB4
:104FA000C00111248035910534F08E8199278F77C7
:104FB0009070892B59F08E8180788E8388819981B9
:104FC0000E94B41A888199810E9488271F5F2A96BF
:104FD0009091880A191710F3DF91CF911F910895CE
:104FE0000F931F938C01C8010E947F1C84E00E94D4
:104FF000CB1B61E0C8010E94BB1B8AE00E94CB1B57
:105000001F910F910895E82FFF27EF70F070E4557E
:10501000FC4F84919927089584E593E00895809149
:10502000620382FF05C08091560390915703089553
:1050300080915403909155030895089580916203DF
:1050400082608093620308950F931F93CF93DF9341
:10505000C4E5D3E08091620399278C010170107040
:1050600080FF03C080E090E021C060915A037091FE
:105070005B0380915C0390915D036115710581056F
:10508000910531F00E945E13882311F4C8010EC00F
:105090001A821B821A8A1B8A10925503109254039B
:1050A0001E861C8A0E94FF0C81E090E0DF91CF9168
:1050B0001F910F9108959C01809156039091570381
:1050C000892B11F4C90108952F703F7B77FD30645F
:1050D000CB018F70907044E0880F991F4A95E1F7DB
:1050E000822B932B08950895FC0180915403909195
:1050F00055032091560330915703E817F907F9F447
:1051000060936403232BB1F080915803909159036D
:10511000F4E096958795FA95E1F7BC016F70707091
:10512000892F99278695869580FD7068CA010E940F
:105130005B280FC050935903409358030EC0E217E9
:10514000F30759F4BA0180915803909159030E94D2
:105150005B2890935903809358030E94FF0C089595
:105160009C01892B69F41092620310925A031092E9
:105170005B0310925C0310925D030E942428089543
:105180006093640350935903409358038091F2064F
:105190009091F306A091F406B091F50688519C4FCA
:1051A000AF4FBF4F816080935A0390935B03A093EE
:1051B0005C03B0935D038091620382FF10C0816045
:1051C0008B7F809362033093570320935603B9017A
:1051D00080915403909155030E94592707C08E7FF8
:1051E0008093620330935503209354030E94FF0C75
:1051F00008950895209162032B7F2160209362031C
:1052000090935703809356038091580390915903CC
:105210000E945B2890935903809358030E94FF0CCF
:105220000895809363030E940328809365030E947E
:10523000FF0C0895CF93C82F882319F064ED71E017
:1052400002C064EF71E084E00E945518CC2319F08D
:105250006CEC71E002C06CEE71E085E00E945518C4
:10526000CC2319F064EC71E002C064EE71E086E0DA
:105270000E945518CC2319F06CEB71E002C06CED64
:1052800071E087E00E945518CF910895CF93DF9386
:10529000C82FDD27C4FF02C083E001C085EA0E9459
:1052A000EE16C0FF02C084E001C085EA0E94EE163F
:1052B000C1FF02C085E001C085EA0E94EE16C2FF70
:1052C00002C086E001C085EA0E94EE16C3FF02C05C
:1052D00087E001C085EA0E94EE16DF91CF91089524
:1052E000809374030E94FF0C0895882319F06CE9E1
:1052F00071E002C064EA71E082E00E9455180895EE
:105300000895882319F06CEA71E002C064EB71E043
:1053100081E00E945518089508950F931F93CF932D
:1053200004E513E0C0917403CC2399F060E081E0C0
:105330000E9426178C2F81500E94DD4EBC0182E016
:105340000E94AE181092740388EE93E00E949515A7
:1053500002C0882319F00E944D1803C0682F0E94D4
:1053600026178091540390915503892BF9F00E94E0
:10537000BA4FFC01828193814091540350915503AF
:105380008417950749F421853285809166039091B1
:1053900067032817390751F04283538380916603CE
:1053A00090916703818792870E94414F2091540317
:1053B000309155032115310529F4F80124833583F3
:1053C000108A17868091620382FD0DC080915E0372
:1053D00090915F03A0916003B09161030097A105D4
:1053E000B10519F105C06CEB73E082E00E94AE18C4
:1053F00080915E0390915F03A0916003B09161037F
:10540000BF93AF939F938F938FEB93E09F938F9373
:1054100082E08F930E9404198DB79EB707960FB64E
:10542000F8949EBF0FBE8DBF43C02115310531F4E6
:1054300062ED73E082E00E94AE1818C03F932F9394
:1054400089ED93E09F938F93C2E0CF930E9404195C
:10545000809162030F900F900F900F900F9080FF3C
:1054600002C08C2F01C080E20E94EE16C09163033F
:105470000E94420D853010F085E00EC0833061F44B
:105480008C2F99278370907023E0880F991F2A959D
:10549000E1F7845A9C4F08C0992703E0880F991FB1
:1054A0000A95E1F784589C4FBC0182E00E94AE1837
:1054B0006CE080E00E9426178091640399278F7723
:1054C00090709F938F938EED93E09F938F9382E0E4
:1054D0008F930E94041980916303992783709070C1
:1054E0000F900F900F900F900F90019781F483E130
:1054F0000E941116882339F064E671E080E00E9472
:10550000551880E001C080E20E94EE160FC080E0D6
:105510000E94EE168091640387FF03C06CE372E083
:1055200002C064E372E080E00E9455180E94420DC0
:10553000C82F813049F488E00E94A84EAC0160E099
:105540008C2F0E94E817E0C040E050E060E0862F1A
:105550000E949817C0E08AE00E941116882371F01B
:105560008091560390915703892B39F480916303FE
:10557000992783709070039709F4C1E060E081E09F
:105580000E94261780915E0390915F03A0916003B3
:10559000B09161030097A105B10509F442C08DE007
:1055A0000E941116882329F48EE00E941116882388
:1055B00081F182EE93E09F938F93C2E0CF930E949C
:1055C00004198DE00E9411160F900F900F90882300
:1055D00079F06CEA71E081E00E94551864EA71E0AC
:1055E0008C2F0E9455186CE271E081E899E20EC0A0
:1055F00064EB71E081E00E9455186CE971E08C2F3A
:105600000E9455186CE271E085E799E20E945F17ED
:105610007BC086E00E94A84EBC0182E00E94AE18CA
:1056200044C08091560390915703009769F19F936E
:105630008F938EEE93E09F938F9382E08F930E94DF
:105640000419809158039091590314E09695879519
:105650001A95E1F7282F2F70892F9927869586951F
:105660000F900F900F900F900F9080FD2061822F70
:105670000E944629CC2321F08CE30E94EE1615C02F
:1056800080E20E94EE162CC088E693E09F938F93F1
:1056900083EF93E09F938F9382E08F930E9404198E
:1056A0000F900F900F900F900F90CC23C9F0809126
:1056B000560390915703892B99F480915803909148
:1056C0005903A4E096958795AA95E1F78F708061BC
:1056D0000E94462981E00E941A296CEF71E011C0F6
:1056E000209158032F70809158039091590397FD92
:1056F0002061822F0E94462980E00E941A2964E0DE
:1057000072E083E00E945518CF911F910F91089588
:1057100060915A0370915B0380915C0390915D03EB
:10572000611571058105910561F00E945E13882362
:1057300041F010925A0310925B0310925C03109296
:105740005D0308950895EF92FF920F931F93CF93F7
:10575000DF93EC01E4E5EE2EE3E0FE2E81319105CE
:10576000CCF48F3091050CF0D5C08A30910509F446
:10577000F9C18B30910534F4009709F410C197FDFD
:1057800000C220C18C30910509F462C00D970CF065
:105790007EC049C185319105D9F18631910574F4F6
:1057A0008231910509F4D6C0823191050CF4E9C02B
:1057B00083319105D1F14497B1F0E3C18F38910560
:1057C0006CF48D3891050CF062C08C31910509F4B0
:1057D000B9C08A38910509F4D2C1D3C18339910582
:1057E00009F4CDC1CEC18091640399278F77907061
:1057F000209165033327821793070CF0C2C10E94E2
:10580000420D833009F0BDC1809164038F5F1DC0DC
:1058100020916403822F99278F779070892B09F448
:10582000B0C1215020936403AAC1809163039927DA
:1058300083709070019729F464E671E080E00E9423
:10584000551880916403809580788093640397C194
:105850008AE00E941116882399F080915603909156
:105860005703892B69F0809158039091590320E0E8
:1058700030E48227932790935903809358037FC184
:10588000809158039091590320E030E855C08091F1
:105890005E0390915F03A0916003B0916103009754
:1058A000A105B105A9F120915E0330915F0321505C
:1058B0003040220F331FCE018F7790700E9709F47E
:1058C0002160C7FF20C060E0C9010E94F05F8091A5
:1058D0005E0390915F0301970E94056260E070E0B3
:1058E000CB010E945F1764E172E081E00E945518CD
:1058F0006CE172E082E00E945518F701128613866F
:10590000148615863CC161E0C9010E94F05F37C171
:10591000C7FD35C11C2F1D508AE00E941116811150
:105920001C5F21E030E002C0220F331F1A95E2F71E
:10593000809158039091590382279327F70184831C
:1059400095831DC16CE380915403909155030E948F
:10595000871B15C1F89483E00E94030D882319F07A
:1059600084E00E94FF6183E10E941116882339F0D0
:105970006BE480915403909155030E94871B7894A7
:10598000FEC08AE00E941116811182E00E94030D80
:10599000882309F4F4C084E00E94FF61F0C0809184
:1059A0005E0390915F03A0916003B0916103009743
:1059B000A105B10539F48FEF0E944E4E81E00E949F
:1059C0008D29DFC080915E0390915F03A0916003F9
:1059D000B09161039C01AD0163E0220F331F441FAE
:1059E000551F6A95D1F7280F391F4A1F5B1F280FD3
:1059F000391F4A1F5B1FCE01AA2797FDA095BA2F1A
:105A0000280F391F4A1F5B1F2030F8E23F07F0E0E4
:105A10004F07F0E05F070CF0B4C0F701228733872F
:105A200044875587ACC0C4E5D3E020915E03309134
:105A30005F03409160035091610360915603709140
:105A40005703211531054105510509F47FC0611542
:105A5000710519F10091540310915503C801AA274B
:105A6000BB2782179307A407B50741F0CB01AA27EC
:105A7000BB2782179307A407B50779F480916203C7
:105A80008E7FF7018687C8010E947927F70112826D
:105A900013821092550310925403809154039091F5
:105AA00055039C014427552780915E0390915F0325
:105AB000A0916003B09161036091620328173907D8
:105AC0004A075B0729F481E068276B7F6E8745C032
:105AD0006C7F6E871A8A1B8A1C8A6091680381E03A
:105AE0000E94261780E00E94A84EBC0182E00E941E
:105AF000AE1880916203992796958795969587951C
:105B00009C012170307080FD11C02A833B832C835F
:105B10003D8330935503209354031F8660915E03A9
:105B200070915F038FEF0E9425510BC040915E037F
:105B300050915F0360915403709155038FEF0E9461
:105B40004151809162038B7F8E8707C0672B29F4B8
:105B5000809162038460F70186871A861B861C8603
:105B60001D860DC010925E0310925F0310926003B9
:105B700010926103809162038B7F809362030E9485
:105B8000FF0CDF91CF911F910F91FF90EF9008953F
:105B9000FC01EC5BFF4F8081E454F040882319F452
:105BA00080E090E00895E95BFF4F8081E754F0408A
:105BB000882329F48481883511F0883719F481E02D
:105BC00090E0089580E090E008950895CF93DF93EA
:105BD000EC010E94C82D882319F480E090E01FC0DA
:105BE000FE01E95BFF4F8081882351F4CC5BDF4FDE
:105BF0008881C454D040823018F481E090E00FC016
:105C00008081882311F08C8101C08D81992787FDC7
:105C10009095809590958827990F881F9927DF91F7
:105C2000CF910895CF93C82FCF7719F480E090E0FB
:105C300029C0862F0E940328282F33272B313105B6
:105C400089F02C31310524F42E30310529F017C0AC
:105C50002C31310569F013C0EC2FFF27EB5CFB4FB3
:105C600084910BC0EC2FFF27E75EFB4F849105C0AA
:105C7000EC2FFF27E450FC4F8491992703C0CF5F9E
:105C80008C2F9927CF910895CF93C82FCF7719F4F0
:105C900080E090E02EC0C150862F0E940328282F5C
:105CA00033272B31310579F02C31310524F42E3096
:105CB000310529F01CC02C31310569F018C08C2F3A
:105CC000992708960DC083E0C89FC00111240B9648
:105CD0006EE070E007C08C2F9927880F991F0796F8
:105CE00069E070E00E94CD67CB01992702C08C2F3C
:105CF0009927CF910895019791F40E94BA4FFC0122
:105D00008181882311F484E608C0843011F485E68B
:105D100004C08150843008F08150992708958FEF96
:105D20009FEF089508951F93CF93C82FFB01142F61
:105D30008181282F332782819927982F8827282B24
:105D4000392BC90101978F5F974210F062E010C0B4
:105D5000112321F0C9010E94732403C0C9010E94CC
:105D60004B24009751F4112311F06BE001C06AE05D
:105D70008C2F0E947E1880E090E0CF911F910895B3
:105D8000EF92FF920F931F93CF93DF93EB01E42EDB
:105D900041E00E94932E8C01892B19F48FEF90E043
:105DA00064C00E94BB19882319F088E090E05DC0B0
:105DB000FB80EE2051F021E0F21639F4F82EF801C4
:105DC000808191810E94B41A08C0EE2031F0F80160
:105DD00060858B810E94442EF82E6C81862F992736
:105DE00085FF02C0F0E8FF2AF801C481D581DF7782
:105DF00084FDD06867FF05C0C07F8F709070C82B8E
:105E0000D92B2F2D332720783070F8016681862F0B
:105E10009927807890702817390731F0607840E032
:105E2000808191810E949B2640E06F2DF801808146
:105E300091810E949B2640E0BE01F8018081918102
:105E40000E941E27F801808191810E9488270E946C
:105E5000420D833019F480E090E007C0823019F4DD
:105E600081E490E002C082E490E0DF91CF911F9145
:105E70000F91FF90EF90089541E00E94C02E992766
:105E8000089540E00E94C02E992708951F93CF9354
:105E9000DF93182F40E0812F0E94932EEC01892B75
:105EA000C1F060E0812F0E947E1868858E810E947B
:105EB000122E682F812F0E947E186C816F708C814A
:105EC0009D8197FD60618E8187FD6062812F0E94B8
:105ED0007E188FEF90E0DF91CF911F9108951F936F
:105EE000CF93DF93182F40E0812F0E94932EEC0177
:105EF000892BC9F060E0812F0E947E18888583700D
:105F0000682F812F0E947E1888850E940328682FA1
:105F1000812F0E947E186FEF812F0E947E186FEFF5
:105F2000812F0E947E188FEF90E0DF91CF911F911B
:105F300008950F931F93CF93DF938B0141E00E944D
:105F4000932EEC01892B19F48FEF90E014C08C8113
:105F50009D818070F80123813327822B932B40E0B1
:105F6000BC01888199810E941E27888199810E94A5
:105F7000882780E090E0DF91CF911F910F910895E5
:105F80000F931F93CF93DF938B0141E00E94932ED9
:105F9000EC01892B19F48FEF90E018C02C813D8122
:105FA000307CF801838199278F739070982F882710
:105FB000282B392B40E0B901888199810E941E2746
:105FC000888199810E94882780E090E0DF91CF91BD
:105FD0001F910F9108951F93CF93DF93182F40E0E7
:105FE000812F0E94932EEC01892B41F060E0812FDC
:105FF0000E947E186C81812F0E947E188FEF90E0A6
:10600000DF91CF911F9108951F93CF93DF93182FA6
:1060100040E0812F0E94932EEC01892B69F060E013
:10602000812F0E947E188C819D81892F99278F73E3
:10603000682F812F0E947E188FEF90E0DF91CF9123
:106040001F910895DF92EF92FF920F931F93CF93CA
:10605000DF93982F8B01823008F064C088E4989F0A
:106060007001112485E793E0E80EF91EFB018181A0
:10607000C82FDD278281992787709070982F8827F5
:10608000C82BD92B2197F7E0C83FDF0718F082E033
:1060900090E04AC00E94BA4FFC01808181FD07C098
:1060A00023E0CD3FD20718F08EE090E03DC00E9483
:1060B000420D833039F00E94420D823019F086E0A3
:1060C00090E032C0CC0FDD1FF801628167FFC16034
:1060D000862F9927E6E096958795EA95E1F771E096
:1060E000D72ED82287010B5B1F4FF8018081918149
:1060F000FFEF8F3F9F0741F060E00E94F05F8FEF5E
:106100009FEFF801808391836D2DCE010E94F05F97
:10611000882319F487E090E007C0DD2019F0F8012A
:10612000C083D18380E090E0DF91CF911F910F91E8
:10613000FF90EF90DF900895FF920F931F93CF93FE
:10614000F82EFB018181082F112782819927877002
:106150009070982F8827082B192B87E0083F180785
:1061600018F082E090E022C0C8010E94B85F873634
:1061700011F0873411F4C4E001C0C0E00E94BA4FAE
:10618000FC01808181FF02C0C16006C00C5F13402A
:1061900018F08EE090E00AC060E08F2D0E947E181B
:1061A0006C2F8F2D0E947E188FEF90E0CF911F9162
:1061B0000F91FF9008951F93CF93182FFB01C1817A
:1061C000CC2319F482E090E00FC060E00E947E18BA
:1061D000EC2FFF27E65BF44F80818095682F812F9D
:1061E0000E947E188FEF90E0CF911F9108951F932A
:1061F000CF93182FFB01C181C150C03218F082E04B
:1062000090E015C060E00E947E1860E08C2F0E9434
:106210002059682F812F0E947E1861E08C2F0E94E8
:106220002059682F812F0E947E188FEF90E0CF9128
:106230001F9108950E943B5980E090E008951F93BC
:10624000CF93182FFB0181819927009719F00397AD
:1062500029F008C0C091890ACC0F07C0C0918A0AF2
:10626000C17003C082E090E00AC060E0812F0E940C
:106270007E186C2F812F0E947E188FEF90E0CF91B7
:106280001F910895FB0181819281282F33272115C9
:10629000310521F02330310559F014C0913490F4C8
:1062A000892F99270196959587958093890A0DC026
:1062B00080918A0A992311F0816001C08E7F8093BA
:1062C0008A0A03C082E090E0089580E090E008959B
:1062D0000895EF92FF920F931F93CF93DF93CDB763
:1062E000DEB760970FB6F894DEBF0FBECDBFF82EB5
:1062F00063E00E947E1861E08F2D0E947E1864E0AA
:106300008F2D0E947E1860E08F2D0E947E1864E021
:106310008F2D0E947E180E94F74FDC01CB01BF93A6
:10632000AF939F938F9384E494E09F938F938E0118
:106330000F5F1F4F1F930F930E94A2628DB79EB7EE
:1063400008960FB6F8949EBF0FBE8DBF33E0E32EC4
:10635000F80191919295907F81918F018053982BB4
:10636000692F8F2D0E947E18EA94E7FEF1CF80E01E
:1063700090E060960FB6F894DEBF0FBECDBFDF9100
:10638000CF911F910F91FF90EF9008951F93CF939E
:10639000182FC0E00E94420D982F8250823008F4DE
:1063A000C8E0923009F4C0616C2F812F0E947E18E2
:1063B0008FEF90E0CF911F9108951F93CF93DF93BC
:1063C000182FFB018181282F332782819927982F4D
:1063D0008827822B932B0E947B2EEC0197FF03C012
:1063E00082E090E00AC060E0812F0E947E186C2F4E
:1063F000812F0E947E188FEF90E0DF91CF911F9147
:10640000089560E00E947E1882E00E94030D8FEFE5
:1064100090E0089580E00E94030D80E090E00895F0
:1064200083E00E94030D80E090E0089580E090E01A
:1064300008951F93CF93DF93182F0E949A61EC0168
:1064400060E084E0989F812D9927112480FD61E010
:10645000CE01892F992782958695877080FD64608B
:10646000C0FD6860D7FD6062CE7FDF71209709F0C4
:106470006068812F0E947E18209791F060E0C1FD36
:1064800061E0C2FD6064C97F209709F06068812FD8
:106490000E947E18CD2B21F060E0812F0E947E1893
:1064A0008FEF90E0DF91CF911F9108950F931F938D
:1064B000CF93DF93182FC8E0D8E000E08091880ADE
:1064C000081778F58F8180FF29C068858E810E942A
:1064D000122E682F812F0E947E186C81812F0E94BE
:1064E0007E186881812F0E947E1888819981892F6A
:1064F0009927682F6F738C819D8197FD60648E81D1
:1065000087FD6068812F0E947E188E818F77682FAB
:10651000812F0E947E188F818E7F8F830F5F2A9636
:10652000CDCF80E890E0DF91CF911F910F9108953A
:10653000AF92BF92CF92DF92EF92FF920F931F9391
:10654000CF93DF93CDB7DEB7C254D0400FB6F894E7
:10655000DEBF0FBECDBFC82E21E030E010E0512FCE
:1065600041E07E01E20EF31E5701E52FFF27BF0138
:10657000655B734FDB018C91882319F4295F3F4FD2
:106580001DC08423C9F0D7012D937D01832F992746
:10659000982F97709C93E55BF44F8081842311F4CE
:1065A00090689C930894E11CF11C1F5F942F9095B8
:1065B000FB01808189238083440F11F45F5F41E0F8
:1065C0002F5F3F4FF7E0293F3F0710F4103268F28A
:1065D000612F8C2D0E947E18DD247501012F11275B
:1065E0000115110581F0D7018D917D01682F8C2D4A
:1065F0000E947E18D3942D2D3327C801800F911F40
:106600002817390784F38FEF90E0CE5BDF4F0FB68A
:10661000F894DEBF0FBECDBFDF91CF911F910F91D8
:10662000FF90EF90DF90CF90BF90AF900895CF9202
:10663000DF92EF92FF920F931F93CF93DF93D82EA9
:10664000CC248091890A882309F454C0F8948C2DB5
:10665000992787FD9095880F991F9C01255F344FDE
:106660008C010553154FEC01C557D54F4881942F28
:106670009095D8018C918923F901E080E82A59810D
:10668000952F9095F80181818923F901F180F82AED
:106690002E2D332727FD3095842F9927281739076A
:1066A00049F42F2D332727FD3095852F992728175B
:1066B000390799F08C2D8F5F682F8D2D0E947E18E1
:1066C0006E2D8D2D0E947E186F2D8D2D0E947E18AF
:1066D000E882F982F801118210827894C3942C2DFB
:1066E000332727FD30958091890A99272817390784
:1066F0000CF4ACCF60E08D2D0E947E188FEF90E0FF
:10670000DF91CF911F910F91FF90EF90DF90CF908D
:1067100008951F93CF93C82F162F603418F06AE4A2
:1067200074E002C064E574E08C2F0E94AE18812FE3
:1067300099278A30910589F18B3091057CF4863058
:10674000910511F1873091051CF40297D1F039C001
:1067500087309105E1F00897E9F033C08E3091055C
:1067600029F18F30910534F48B309105C9F00D97E4
:10677000D1F027C081349105E1F082349105E1F038
:1067800020C06CE574E01AC060E774E017C06DE7E4
:1067900074E014C060E974E011C063EA74E00EC0F4
:1067A0006BEA74E00BC06DEB74E008C066EC74E05B
:1067B00005C06DED74E002C068EE74E08C2F0E949D
:1067C000AE18103420F06DE08C2F0E947E1881E00E
:1067D00090E0CF911F9108950F931F93D8018A30B5
:1067E000C0F48617B0F49927FC0164E0EE0FFF1F98
:1067F0006A95E1F7E81BF90BEB5FFB4F8685882371
:1068000041F0008111810417150718F02017310796
:1068100008F48D01C8011F910F91089563EF74E092
:106820000E94AE1881E090E008956AE275E00E944F
:10683000AE1881E090E0089567E475E00E94AE181C
:1068400081E090E008951F93182F60E875E00E94A2
:10685000AE186AE975E0812F0E94AE1869EB75E009
:10686000812F0E94AE1881E090E01F910895CF9390
:10687000C82F0E94420D992783309105A1F08430E2
:1068800091052CF4009749F0029751F017C084301D
:10689000910561F0079794F40CC066ED75E00BC0AC
:1068A0006EED75E008C066EE75E005C06DEE75E052
:1068B00002C069EF75E08C2F0E94AE1881E090E075
:1068C000CF910895EF92FF920F931F93182F7B01A2
:1068D000042F80E00E94030D402FB701812F0E94FA
:1068E000373499271F910F91FF90EF900895EF9201
:1068F000FF920F931F93182F7B01042F83E00E94B8
:10690000030D402FB701812F0E94373499271F9123
:106910000F91FF90EF9008956FEF75E00E94AE1811
:1069200082E00E94030D80E090E008950F931F9392
:10693000CF93C82F762F642F00E010E0A801872F97
:106940000E94EC338C01892B21F462E08C2F0E9491
:106950008933C801CF911F910F9108957F928F9233
:106960009F92AF92BF92CF92DF92EF92FF920F93DE
:106970001F93CF93DF93882E942E2FEF37E260E0A2
:106980000E9496345C01009719F481E090E062C1A6
:106990000E944B246C01892B69F421E0291510F029
:1069A0006AE012C0C5010E9473246C01892B11F4A6
:1069B0006BE00AC031E0391508F0D6C00E94BB195F
:1069C000782E882331F068E0882D0E94893399273A
:1069D00041C1F601C481D58110EFE12E1FE7F12EF0
:1069E000EC22FD228D2F992787FD90958827990FFE
:1069F000881F99278C0121E030E040E050E0692DAC
:106A000082E00E94EC33892B21F020E030E8E22A7A
:106A1000F32ACE01817090708C0121E030E040E0DB
:106A200050E0692D84E00E94EC33892B21F081E055
:106A300090E0E82AF92ACE019695879581709070AA
:106A40008C0121E030E040E050E0692D85E00E94BB
:106A5000EC33892B21F0E2E0F0E0EE2AFF2ACE01B0
:106A60009695879596958795817090708C0121E019
:106A700030E040E050E0692D86E00E94EC33892B45
:106A800021F024E030E0E22AF32AE3E0D695C7952E
:106A9000EA95E1F7C170D0708E0121E030E040E06E
:106AA00050E0692D87E00E94EC33892B21F088E0CB
:106AB00090E0E82AF92A472DB701C5010E941E2758
:106AC000F601608586810E94122E99278C012FE79E
:106AD00030E040E050E0692D81E00E94EC33C82FA7
:106AE00080913404863411F411E015C0823511F41C
:106AF000172D11C000E010E0F601868187FF02C06B
:106B000001E010E021E030E040E050E0692D83E05A
:106B10000E94EC33182FC13029F4C0E0C5010E9457
:106B2000B41A06C0F60160858C2F0E94442EC82F2F
:106B30001111C0682C2F332720783070F601668140
:106B4000862F9927807890702817390729F0607868
:106B500040E0C5010E949B2640E06C2FC5010E94C9
:106B60009B26C5010E9488270E94420D823011F4A5
:106B700061E405C00E94420D833021F062E4882D5B
:106B80000E948933F6018481958183FF03C081E3EC
:106B900090E002C080E390E09F938F93F6018481A0
:106BA000958182FF03C081E390E002C080E390E022
:106BB0009F938F93F6018481958181FF03C081E3C8
:106BC00090E002C080E390E09F938F93F601848170
:106BD000958180FF03C081E390E002C080E390E0F4
:106BE0009F938F93F601868187FF03C086E690E02E
:106BF00002C082E790E09F938F93F6018581282F52
:106C0000332727FD3095209530952227330F221FFB
:106C1000332781E390E0821B930B9F938F936085D2
:106C200086810E94122E99279F938F93BF92AF92D5
:106C300089E096E09F938F938F920E94041981E0E0
:106C400090E02DB73EB72D5E3F4F0FB6F8943EBF94
:106C50000FBE2DBFDF91CF911F910F91FF90EF904D
:106C6000DF90CF90BF90AF909F908F907F900895CE
:106C7000CF93C82F2FEF37E260E08C2F0E9496341D
:106C8000009719F10E944B24FC01892B19F463E24F
:106C900076E018C0808599278370907082309105C6
:106CA00061F0833091051CF4019721F00EC0039729
:106CB00039F00BC06AE276E005C067E376E002C017
:106CC00064E476E08C2F0E94AE1881E090E0CF91D2
:106CD00008957F928F929F92AF92BF92CF92DF9250
:106CE000EF92FF920F931F93CF93DF93A82EB42EB2
:106CF0002FEF37E260E00E9496344C01009719F4C0
:106D000081E090E021C10E944B246C01892B69F441
:106D100021E02B1510F06AE012C0C4010E94732418
:106D20006C01892B11F46BE00AC031E03B1508F0CF
:106D30008FC00E94BB19782E882331F068E08A2D1D
:106D40000E948933992700C1F601E480F580E701AC
:106D5000C070C701817090708C0121E030E040E08C
:106D600050E06B2D81E00E94EC33892B09F0C1606B
:106D7000C70196958795817090708C0121E030E075
:106D800040E050E06B2D82E00E94EC33892B09F04B
:106D9000C260C7019695879596958795817090708A
:106DA0008C0121E030E040E050E06B2D83E00E9458
:106DB000EC33892B09F0C46003E0F694E7940A955C
:106DC000E1F7F1E0EF22FF24870121E030E040E02D
:106DD00050E06B2D84E00E94EC33892B09F0C860F1
:106DE000870121E030E040E050E06B2D85E00E941B
:106DF000EC33892B09F0C061870121E030E040E0ED
:106E000050E06B2D86E00E94EC33892B09F0C062C4
:106E1000870121E030E040E050E06B2D87E00E94E8
:106E2000EC33892B09F0C064870121E030E040E0B9
:106E300050E06B2D88E00E94EC33892B09F0C0688C
:106E4000472DBE01C4010E941E27C4010E9488274D
:106E50000E94420D882321F462E48A2D0E94893326
:106E6000F6018481958187FF03C081E390E002C031
:106E700080E390E09F938F93F6018481958186FF54
:106E800003C081E390E002C080E390E09F938F9382
:106E9000F6018481958185FF03C081E390E002C003
:106EA00080E390E09F938F93F6018481958184FF26
:106EB00003C081E390E002C080E390E09F938F9352
:106EC000F6018481958183FF03C081E390E002C0D5
:106ED00080E390E09F938F93F6018481958182FFF8
:106EE00003C081E390E002C080E390E09F938F9322
:106EF000F6018481958181FF03C081E390E002C0A7
:106F000080E390E09F938F93F6018481958180FFC9
:106F100003C081E390E002C080E390E09F938F93F1
:106F20009F928F9288E496E09F938F93AF920E94F6
:106F3000041981E090E02DB73EB72B5E3F4F0FB6AE
:106F4000F8943EBF0FBE2DBFDF91CF911F910F91DF
:106F5000FF90EF90DF90CF90BF90AF909F908F9079
:106F60007F9008957F928F929F92AF92BF92CF921F
:106F7000DF92EF92FF920F931F93CF93DF93A82E90
:106F8000B42E2FEF37E260E00E9496344C01009758
:106F900019F481E090E02EC10E944B246C01892BF2
:106FA00069F421E02B1510F06AE012C0C4010E94C0
:106FB00073246C01892B11F46BE00AC031E03B159E
:106FC00008F09DC00E94BB19782E882331F068E03C
:106FD0008A2D0E94893399270DC1F601C481D5817C
:106FE0004FEFE42E40ECF42EEC22FD228D2F99275A
:106FF000817090708C0121E030E040E050E06B2D1A
:1070000081E00E94EC33892B21F020E031E0E22A7C
:10701000F32ACE01892F99278695817090708C0173
:1070200021E030E040E050E06B2D82E00E94EC3344
:10703000892B21F080E092E0E82AF92ACE01892FFD
:10704000992786958695817090708C0121E030E0BB
:1070500040E050E06B2D83E00E94EC33892B21F05F
:10706000E0E0F4E0EE2AFF2ACE01892F99278695E9
:1070700086958695817090708C0121E030E040E02B
:1070800050E06B2D84E00E94EC33892B21F020E04E
:1070900038E0E22AF32ACE01892F992782958F7052
:1070A000817090708C0121E030E040E050E06B2D69
:1070B00085E00E94EC33892B21F080E090E1E82A02
:1070C000F92ACD2FDD27C295C695C770C170D07043
:1070D0008E0121E030E040E050E06B2D86E00E9420
:1070E000EC33892B21F0E0E0F0E2EE2AFF2A472D75
:1070F000B701C4010E941E27C4010E9488270E9474
:10710000420D882321F462E48A2D0E948933F6011E
:1071100084819581892F992782958695877080FF34
:1071200003C081E390E002C080E390E09F938F93DF
:10713000F60184819581892F992782958F7080FF30
:1071400003C081E390E002C080E390E09F938F93BF
:10715000F60184819581892F992786958695869554
:1071600080FF03C081E390E002C080E390E09F9342
:107170008F93F60184819581892F9927869586952D
:1071800080FF03C081E390E002C080E390E09F9322
:107190008F93F60184819581892F9927869580FFA9
:1071A00003C081E390E002C080E390E09F938F935F
:1071B000F60184819581892F992780FF03C081E39F
:1071C00090E002C080E390E09F938F939F928F9214
:1071D00085E696E09F938F93AF920E94041981E019
:1071E00090E02DB73EB72F5E3F4F0FB6F8943EBFED
:1071F0000FBE2DBFDF91CF911F910F91FF90EF90A8
:10720000DF90CF90BF90AF909F908F907F90089528
:10721000AF92BF92CF92DF92EF92FF920F931F93A4
:10722000CF93DF93A82EC42F0E94420D882311F420
:1072300066E05BC028EF37E04C2F60E08A2D0E94AB
:1072400096346C01892B19F021E02A1518F481E09D
:1072500090E081C088E4A89EC00111248B589C4F07
:10726000C23008F44CC075E4E72EF12CE80EF91E8C
:10727000F70180819181FFEF8F3F9F0741F060E030
:107280000E94F05F8FEF9FEFF701808391838091E1
:107290001604873411F4BB2410C0823519F461E060
:1072A000B62E0BC002E010E021E030E040E050E0FC
:1072B0006C2F81E00E94EC33B82E00E010E021E05A
:1072C00030E0A8016C2F82E00E94EC33EC018601D3
:1072D00001501040000F111F0B0D111D682FC80128
:1072E0000E94F05F882331F467E08A2D0E94893381
:1072F000992731C0CC2319F0F70100831183C6010F
:1073000001970E94B85FC0E0D0E0082F112707FD69
:107310001095C8010E94F467892B11F0C1E0D0E0FC
:10732000DF93CF93C8010E9407689F938F93DF92EA
:10733000CF928DE796E09F938F93AF920E940419AE
:1073400081E090E02DB73EB7275F3F4F0FB6F8942E
:107350003EBF0FBE2DBFDF91CF911F910F91FF90C8
:10736000EF90DF90CF90BF90AF9008951F93182FAC
:1073700068E876E00E94AE1865E976E0812F0E9409
:10738000AE180E94F74FDC01CB01BF93AF939F93E0
:107390008F938BE996E09F938F931F930E9404191C
:1073A0008DB79EB707960FB6F8949EBF0FBE8DBFE0
:1073B00081E090E01F910895EF92FF920F931F9349
:1073C000CF93DF93E82EF42E0E94BA4FEC01FF20FA
:1073D000E1F08B8599278C0124E130E040E050E01A
:1073E0006F2D80E00E94EC338B878C859927880F66
:1073F000991F8C012EEF31E042E050E06F2D81E0CB
:107400000E94EC33969587958C878C859927880FF9
:10741000991F9F938F938B8599279F938F9388EACA
:1074200096E09F938F93EF920E9404198DB79EB7B9
:1074300007960FB6F8949EBF0FBE8DBF81E090E017
:10744000DF91CF911F910F91FF90EF9008950F93CF
:107450001F93CF93C82F642F442379F080918A0A19
:107460009927817090708C0121E030E040E050E07D
:1074700080E00E94EC330E94305980918A0A99275B
:10748000817090709F938F9381EB96E09F938F9381
:10749000CF930E9404190F900F900F900F900F90B0
:1074A00081E090E0CF911F910F910895DF92EF92CC
:1074B000FF920F931F93CF93E82E842F00E010E0EC
:1074C00020E230E041E050E0682F80E00E94EC33A1
:1074D000C82F882309F447C099279F938F9387EB80
:1074E00096E09F938F93EF920E940419DC2EDA941A
:1074F00060E08D2D0E942059082F1127A1E0FA2E5F
:107500000F900F900F900F900F90C7E08F2D99273D
:1075100080239123892B11F061E301C060E38E2D5C
:107520000E947E18C150FF0CC7FFF0CF60E28E2D85
:107530000E947E1861E08D2D0E942059082F11278E
:10754000F1E0FF2EC7E08F2D992780239123892B0F
:1075500011F061E301C060E38E2D0E947E18C150DE
:10756000FF0CC7FFF0CF81E090E0CF911F910F910A
:10757000FF90EF90DF900895FF920F931F93F82EE6
:10758000642F8091890A9927880F991F8C0120E424
:1075900030E040E050E080E00E94EC338F5F869561
:1075A0008093890A9927880F991F9F938F938AED5B
:1075B00096E09F938F93FF920E9404190F900F9073
:1075C0000F900F900F9081E090E01F910F91FF902E
:1075D0000895CF93C82F4423C9F4C13031F460EE2D
:1075E00076E08C2F0E94AE1813C00E94CC0F9F93A0
:1075F0008F9386EE96E09F938F93CF930E9404190A
:107600000F900F900F900F900F9002C0C13019F49F
:1076100081E090E00DC069EE76E08C2F0E94AE18FC
:1076200080910504909106040E948C0F80E090E008
:10763000CF9108950F931F93CF93C82F842F0FEFEF
:107640001FEF27EE33E040E050E0682F80E00E941B
:10765000EC330E947B2E97FF06C062E08C2F0E94C5
:107660008933992711C090709F938F938CEE96E089
:107670009F938F93CF930E94041981E090E00F9025
:107680000F900F900F900F90CF911F910F91089531
:10769000EF92FF920F931F93982F642F4423C9F00A
:1076A00088E4989F7001112485E793E0E80EF91EA5
:1076B00000E010E021E030E0A80180E00E94EC331F
:1076C000F701E95BFF4F892B19F081E0808301C04E
:1076D000108281E090E01F910F91FF90EF9008954C
:1076E000DF92EF92FF920F931F93CF93DF93082FB8
:1076F000EB01D42E823008F00CC188E4089F900181
:1077000011242B583C4F4881142F1F71642F772769
:10771000CB01807E90708034910509F4A1C0813442
:10772000910534F40097A9F0809709F463C0F1C083
:107730008038910509F4BDC0813891052CF480365C
:10774000910509F4AEC0E5C0803C910509F4CAC0BA
:10775000E0C021E02D1508F0DEC08981C82FDD27AB
:10776000CE010E947324FC01892B09F4D2C0E4806D
:10777000F58014FF05C080E090E8E82AF92A04C0EB
:107780008FEF9FE7E822F9221F70068100781F30F3
:1077900019F460E8602729C080851F7011F01F3040
:1077A00019F460E070E020C00E940328282F3327DE
:1077B0002C31310571F02D31310524F42B31310597
:1077C00029F010C02E37310531F00CC0110F1150C7
:1077D00009C0110F07C089E0189F802D1124682F60
:1077E000772702C0612F7727602B40E0CE010E94EF
:1077F0009B264EC0437F488345E4E42EF12CE20EE5
:10780000F31EF70180819181FFEF8F3F9F0741F0C9
:1078100060E00E94F05F8FEF9FEFF701808391831C
:107820002881203209F475C0233209F472C0F1E0D6
:10783000FD15C8F46981213231F4C62FDD27219767
:10784000CC0FDD1F05C0C62FDD27CC0FDD1F219714
:1078500061E0CE010E94F05FF701C083D18359C07F
:10786000F1E0FD1518F080E090E055C08981C82F47
:10787000DD27CE010E94A32500EFE02E0FEFF02EB2
:10788000E822F922812F99278F709070E82AF92A2F
:1078900040E0B701CE010E941E27CE010E9488273A
:1078A00038C060FF02C080E001C083E00E94030D89
:1078B00030C0112311F4812F18C0C0E0C11748F562
:1078C00060E08C2F0E940F59682F802F0E947E1835
:1078D00061E08C2F0E940F59682F802F0E947E1824
:1078E000CF5FECCF112321F481E00E94305911C009
:1078F000115060E0812F0E940F59682F802F0E9445
:107900007E1861E0812F0E940F59682F802F0E94FE
:107910007E1881E090E0DF91CF911F910F91FF9051
:10792000EF90DF9008959B012F5F3F4F42E0B90138
:107930000E94703B8FEF90E008959B012F5F3F4FB7
:1079400041E0B9010E94703B8FEF90E008958230D2
:10795000C0F4282F332788E490E0289FF001299F66
:10796000F00D389FF00D1124EB58FC4FEC5BFF4FEE
:107970001082339610828FEF9FEF929382930E9432
:107980002E62089508952F923F924F925F926F92C8
:107990007F928F929F92AF92BF92CF92DF92EF929F
:1079A000FF920F931F93CF93DF93CDB7DEB7259749
:1079B0000FB6F894DEBF0FBECDBF8B83B62E8230DC
:1079C00008F0DFC188E49B81989F800111240B5847
:1079D0001C4FE4E4CE2ED12CC00ED11ED6018C91CA
:1079E0008823B1F0F80180819181A281B38188530D
:1079F0009F4FAF4FBF4FBC01CD010E945E13882344
:107A000039F0C8010E94C82D882311F4D6018C9347
:107A10008091F2069091F306A091F406B091F506DC
:107A2000F80180839183A283B383D6018C91803443
:107A300008F01C92C8010E94E62D882391F0B8E05E
:107A4000BB1641F4F6018081882309F49AC1815064
:107A5000808397C1BB2009F494C1FDE0BF1609F4EF
:107A6000BB24D601FC90F801EF0DF11DB482F39414
:107A7000FC92C8010E94C82DA82E882309F476C163
:107A8000C8010E94E62D882309F43CC1BB2009F0FF
:107A900078C1F601B08286E491E08C839D8374E026
:107AA000472E512C400E511E095B1F4FD8018C915F
:107AB00007541040882329F465E0462E512C400ECF
:107AC000511EF2018081882309F416C143E050E081
:107AD0006FEE76E0C2010E94F262892B19F4C201B6
:107AE000039601C0C2010E94506449825A82EE246A
:107AF00086E9E5E0F4E011928A95E9F705C008947B
:107B0000211C311C29823A8229803A80D1019C9122
:107B1000992391F09C3281F0943271F0953261F0AA
:107B2000892F80538A3040F0892F992787FD9095BF
:107B30000E94FE67892B19F3F1018081882309F4E3
:107B4000A8C004C00F5F1F4F09831A8309811A81DF
:107B5000D801FC908F2D992787FD90950E94FE6794
:107B6000892B81F7FF2009F496C0BCE2FB1609F4CB
:107B700082C08FE0E89E60011124E5E0F4E0CE0EC3
:107B8000DF1E480152E0A52EB12CAC0CBD1C6624B2
:107B9000772409C00894811C911CD501FD925D01D8
:107BA0000894611C711CBBE06B1671047CF4F40139
:107BB000F080FF2059F0FCE2FF1641F08F2D99274D
:107BC00087FD90950E94FE67892B21F3D5011C92B9
:107BD000F8018081843239F4C801019689839A833F
:107BE00040E150E008C0853251F4C8010196898314
:107BF0009A8342E050E0BE016F5F7F4F06C04AE0CB
:107C000050E0BE016F5F7F4FC8010E940063DC013E
:107C1000CB01F6018083918381E0F601868704C061
:107C20000F5F1F4F09831A8309811A81D801FC90C5
:107C3000FF2081F08F2D992787FD90950E94FE6788
:107C4000892B41F4BCE2FB1659F704C00F5F1F4FAC
:107C500009831A8309811A81F801F080FF2041F01D
:107C60008F2D992787FD90950E94FE67892B71F7CC
:107C7000FCE2FF1621F40F5F1F4F09831A83E39480
:107C8000E981FA818081882321F089E08E1508F04E
:107C90005DCFD1011C924E2D5527142F80914601A6
:107CA00090914701892BD1F0EC81FD816081718138
:107CB000C2010E94D362892B41F4EC81FD812281B3
:107CC00033812115310581F417C08C819D81049683
:107CD0008C839D83DC018D919C91E4CF63EF76E0F2
:107CE0008B810E94AE1808C0412FB2018B81F9012F
:107CF0000995882309F445C063E077E08B810E94F1
:107D0000AE183FC0EEEAF1E0A8014C5F5F4F2F2DA7
:107D1000095B1F4FD8018C9107541040882321F430
:107D2000A8014B5F5F4F21508091AE01882349F13C
:107D30009081DA018C919817A1F48181281708F1BC
:107D40000280F381E02D309749F0BA018B810995CB
:107D5000682F8F3F19F08B810E947E18F6011082E8
:107D600010C034968081882319F70BC00C5F1F4F19
:107D70004F2DB8018B810E94703B882311F0D601F2
:107D8000AC9225960FB6F894DEBF0FBECDBFDF9143
:107D9000CF911F910F91FF90EF90DF90CF90BF9008
:107DA000AF909F908F907F906F905F904F903F909B
:107DB0002F900895FB0121E057FF04C020E050956B
:107DC00041955F4F8330910549F18430910534F43A
:107DD0008130910591F0029729F12AC084309105F4
:107DE00019F0059761F024C081818F5F8183992705
:107DF00084179507ECF0222359F0118219C0818174
:107E00008150818399278417950794F0222321F0CC
:107E1000842F815081830CC021830AC01282138277
:107E2000168A06C090E08281882309F491E092834B
:107E300080E090E008950F931F93CF93DF938C0120
:107E40000E940F28EC01009731F461EF7FE082E09F
:107E50000E94AE180FC09F938F9387EF9FE09F9370
:107E60008F9382E08F930E9404190F900F900F90D0
:107E70000F900F900115110521F0B80182E00E94CA
:107E8000AE18CE01DF91CF911F910F9108950F93FE
:107E90001F93CF93DF93EC018B01009731F097FD97
:107EA00035C00297029790F52BC060E081E00E94F8
:107EB0002617F8018281882359F46BEF7FE082E076
:107EC0000E94AE1864E070E182E00E94AE1818C013
:107ED0000E94F74FDC01CB01BF93AF939F938F9329
:107EE0008AE090E19F938F9382E08F930E94041920
:107EF0008DB79EB707960FB6F8949EBF0FBE8DBF85
:107F000040E050E0B801CE010E94DA3E80E090E00F
:107F1000DF91CF911F910F9108958230910541F02B
:107F20008330910541F440E050E00E94DA3E03C006
:107F30008FEF9FEF089580E090E008950895CF922D
:107F4000DF92EF92FF920F931F93CF93DF93EC0199
:107F50007B010E940C288C01C230D10509F453C06A
:107F6000C330D1052CF42097D1F0219731F090C087
:107F7000C630D1050CF08CC02AC0FC016785262FC5
:107F8000269526952370637009F461E083E0689F6D
:107F9000C0011124280F2350F701218379C060E02C
:107FA00081E00E94261786E190E10E941B3F892B09
:107FB00009F46EC0F70191818AE0989FC0011124F5
:107FC000895A984FBC0182E00E94AE1861C049E016
:107FD00050E0B701CE010E94DA3EF8018081918124
:107FE0008F3F910509F008F453C0F7018181882380
:107FF00011F486E08183F7018181863008F048C062
:1080000088E0818345C0FC0182819381892B09F03E
:108010003FC0F7018281882399F1F801C081D181A5
:108020002097B1F1F7013181832F63E00E94C1678E
:10803000282F2F5F832F0E94C167892F9927880FD0
:10804000991F880F991F282BF801C288D388622FA7
:10805000CE010E94AD25CE010E948F250E941129DC
:10806000C114D10469F0C80144969C01F801478508
:1080700060817181C6010E94FB5AF801828B938B4B
:1080800090E0F7018281882309F491E0F70192835F
:1080900080E090E0DF91CF911F910F91FF90EF90E2
:1080A000DF90CF900895482F30E0832F992787FDE8
:1080B0009095FC01EA5DF84F2491241729F03F5F69
:1080C000222399F78FEF9FEF08950895EF92FF9283
:1080D0000F931F93CF93DF93EB018230910509F447
:1080E00086C08330910534F4009709F43EC00197AF
:1080F00069F0BAC08430910509F443C08430910519
:108100000CF470C0059709F456C0AEC00E940C284C
:108110008C01FC0180819181892B09F4A5C044E187
:10812000E42EF12CE00EF11E8E01065F1F4F6596C6
:108130000C171D07B8F4F7018081882339F00E94DD
:10814000534087FD03C0F701808101C080E2F80140
:1081500081938F01F7018081882351F30894E11CFA
:10816000F11CE6CFF80110827FC00E941B3F60E047
:1081700081E00E9426172A96BE0182E00E94C41860
:1081800073C08981FB01E80FF11DEF012A968285FA
:108190000E9453408F5FE82FFF27E7FDF095EA5DCF
:1081A000F84F8491882319F4E6E2F7E08491992747
:1081B00087FD909515C08981FB01E80FF11DEF0146
:1081C0002A9682850E945340181614F08FE201C04F
:1081D0008150E82FFF27E7FDF095EA5DF84F849185
:1081E000888342C049E050E00E94DA3E3DC00E94D0
:1081F0000C288C01FC0182819381892BA9F59A813D
:10820000992349F489E08B8381E0888F99839F8B40
:108210008A838E8B29C089818F5F89838F8B8B3076
:1082200018F11B821A821E8A8CE098012C5E3F4F47
:10823000D901FE013A9601900D928A95E1F7F80175
:1082400082899389009731F04785608171810E940E
:10825000FB5A07C0A901F8016785808191810E94BE
:10826000B35BF801828B938B80E090E0DF91CF913C
:108270001F910F91FF90EF900895AF92BF92CF9210
:10828000DF92EF92FF920F931F93CF93DF93CDB7BF
:10829000DEB721970FB6F894DEBF0FBECDBF9C01AD
:1082A0008B018230910509F455C0833091052CF47F
:1082B0000097C1F0019759F0A3C084309105D9F11E
:1082C000843091050CF441C00597C9F199C04BE089
:1082D00050E060E270E0C8010A960E949B62F801DB
:1082E000158A8EC0FB018281882309F489C08181AF
:1082F000882309F485C0065F1F4FA801B90199279B
:108300000E94BB5B9F938F9389E190E19F938F9332
:1083100062E0F62EFF920E94041960E081E00E9464
:108320002617B8018F2D0E94C4180F900F900F9040
:108330000F900F9065C0FB018181992721C0FB013F
:10834000818199270E942D5C1DC049E050E00E9468
:10835000DA3E56C090E0FB018281882309F491E067
:10836000F80192830E940C287C01F8018281882305
:1083700061F0F70182899389009711F0828902C028
:108380000E94FB5BF80181833BC05AE0A52EB12C13
:10839000A00EB11EF8018181A501BE016F5F7F4F64
:1083A00099270E94BB5B6C01F70112821382108235
:1083B0001182BC018FEF0E942551F70180819181CC
:1083C000892B59F06981C6010E94AD25C6010E9422
:1083D0008F250E9411290E941E28F701808191811A
:1083E000892B59F0B501C70144960E94DD62F8015E
:1083F00081819927F701828B938B8FEF9FEF02C0CA
:1084000080E090E021960FB6F894DEBF0FBECDBF9E
:10841000DF91CF911F910F91FF90EF90DF90CF9060
:10842000BF90AF9008950F931F93CF93DF93EC010C
:108430000E940C288C01209719F02297C9F03DC0AA
:10844000CE010E941B3F892BC1F160E081E00E94B8
:108450002617F80182899389892B11F081E001C0E8
:1084600082E00E94A84EBC0182E00E94AE1825C0A6
:10847000FC01C281D381209701F580819181892BF4
:10848000E1F082899389892BC1F060E081E00E944C
:10849000261783E00E94A84EBC0182E00E94AE181D
:1084A00084EF91E00E949515F801828993890E94DA
:1084B000F85AF801C28BD38B148A80E090E0DF91E8
:1084C000CF911F910F9108951F93CF93DF93EB01ED
:1084D0008230910509F440C0833091052CF4009757
:1084E00089F0019731F04CC0863091050CF048C0FE
:1084F0002EC00E94BA4FFC01848163E00E94C167D4
:1085000089833EC060E081E00E942617898113E0E4
:10851000819F802D11240E94791882E090E00E94B2
:10852000951581B7612F0E94C167898399279F9311
:108530008F938DE190E19F938F9382E08F930E94C0
:1085400004190F900F900F900F900F9019C04FEEDD
:108550005FEF0E94DA3E14C08A81882359F00E949E
:10856000BA4F398123E0329F90011124FC0124830A
:108570000E94414F90E08A81882309F491E09A8318
:1085800080E090E0DF91CF911F9108951F93CF93EA
:10859000DF93EC018A81882309F45CC060E081E00C
:1085A0000E9426178C819D819F938F9381E290E199
:1085B0009F938F9312E01F930E9404198B810F9059
:1085C0000F900F900F900F90843059F487E290E154
:1085D0009F938F931F930E9404190F900F900F90F9
:1085E00010C0888599279F938F938BE290E19F938A
:1085F0008F931F930E9404190F900F900F900F906C
:108600000F90898D9A8D97FD03C06FE270E10AC0CB
:108610008E5F9F4F19F467E370E104C084E00E940D
:10862000A84EBC0182E00E94AE1881E0888F8E8B3C
:108630008B8199278130910564F08330910524F076
:108640000497029730F402C083E001C088E08F8B6A
:1086500001C01E8ADF91CF911F9108950F931F9340
:10866000CF93DF938C01FC018281882311F581E097
:108670008383643019F488E090E003C080E094E0E4
:10868000F80186839783F80124813581868197815B
:108690008217930724F481E090E08483958381E03E
:1086A000F8018283683009F410C180E00E94030D54
:1086B0000CC1F801848195819093A5048093A40452
:1086C000C62FDD27C430D10561F1C530D10594F442
:1086D000C130D10509F4C2C0C230D1051CF42097C5
:1086E00001F1F3C0C230D10509F4BAC0239709F4EF
:1086F000E9C0EBC0C730D10509F4B0C0C830D1051E
:1087000044F4C530D10509F4A9C0C630D10549F0FB
:10871000DCC0C830D10509F47EC0299709F49EC099
:10872000D4C0F801838181508230E0F58EEF9FEF55
:10873000818F928FC8010E94C6426AE081E00E9448
:10874000261789E00E94A84EBC0182E00E94AE1864
:10875000C430D10581F0C530D1051CF4CD2B21F0FA
:1087600019C0269771F016C0F80184819581019790
:108770000E94E2580CC0F801848181500E94F9588F
:1087800006C0F8018481958101970E940859F8017B
:10879000818F928FF801818D928D97FD5DC0818DC3
:1087A00080875AC06AE081E00E9426178AE00E9412
:1087B000A84EBC0182E00E94AE18C430D10589F0F9
:1087C000C530D1051CF4CD2B21F046C02697C1F051
:1087D00043C0F80184819581608501970E94DB5830
:1087E00016C0F8018481958109971CF08FEF9FEFE7
:1087F0000FC0F8018481608581500E94F15807C044
:10880000F80184819581608501970E940159F801E2
:10881000818F928F21C00E940C28FC012081318120
:1088200021153105C9F087859927837090700397CA
:1088300099F4F801648175816115710569F083818E
:108840008150823048F0615070404085C9010E94DB
:10885000F027F801138239C081E035C084E033C0CD
:10886000F80183818150823010F481E02DC06AE0EC
:1088700081E00E942617F8018381863079F489E02F
:108880000E94A84EBC0182E00E94AE18F8018481CB
:108890009581618501970E94D4580FC08AE00E949B
:1088A000A84EBC0182E00E94AE18F8018481958137
:1088B000418D618501970E94CD58F801818F928F7B
:1088C00086E001C087E0F8018383DF91CF911F919B
:1088D0000F9108959C01FB018130910561F0823078
:1088E00091051CF4892BD1F024C083309105E9F067
:1088F0000597C1F01EC08EEF9FEF818F928F409140
:10890000A4045091A504CA0101978050944018F422
:10891000448355830EC0248335830BC0CB010E9452
:10892000C64207C081E0838304C040E050E00E945B
:10893000DA3E80E090E008950F931F93CF93DF938A
:108940008C01EB010E940C28FC0180819181892B14
:1089500031F08785992783709070039761F060E00C
:1089600081E00E94261785E00E94A84EBC0182E0AB
:108970000E94AE181BC00230110541F004301105F1
:1089800089F469E0CE010E942E4310C068E0CE0158
:108990000E942E438B81882349F40E9435178FEF64
:1089A0009FEF06C0BE01C8010E946A4480E090E0CB
:1089B000DF91CF911F910F910895CF93DF93EB013A
:1089C0008230910509F481C08330910534F4009719
:1089D000A1F08130910569F07CC08430910509F4E3
:1089E00062C0843091050CF46BC0059709F460C037
:1089F00070C00E946A4419866CC08A81882309F479
:108A000068C060E081E00E9426178B81882331F4E2
:108A10006FE370E182E00E94AE1818C08985992743
:108A20009F938F938C819D819F938F938FE490E18F
:108A30009F938F9382E08F930E9404198DB79EB706
:108A400007960FB6F8949EBF0FBE8DBF898D9A8D85
:108A500097FD0BC0823091051CF0029721F005C0F4
:108A6000898D805D03C08FE301C085E40E94EE160E
:108A700081E0888F8E8B8B8199278630910561F0FC
:108A80008730910524F40197029758F403C00797A3
:108A900029F007C086E003C08CE001C08EE08F8B18
:108AA00018C01E8A16C08B81863039F463E00EC070
:108AB0008B81863011F481E001C086E08B8309C090
:108AC00040E050E00E94DA3E04C062E0CE010E9425
:108AD0002E4380E090E0DF91CF9108959B0182309A
:108AE000910529F08430910539F461E001C060E01E
:108AF000C9010E942E4302C00E946A4480E090E0B7
:108B000008959B018230910529F08430910539F454
:108B100065E001C064E0C9010E942E4302C00E94CA
:108B20006A4480E090E008959B018230910529F02D
:108B30008430910539F467E001C066E0C9010E9404
:108B40002E4302C00E946A4480E090E008951F9383
:108B5000182F60E081E00E942617812F992781302D
:108B6000910571F0823091051CF4892B39F013C006
:108B70008230910539F0039739F00DC08BE005C0C4
:108B80008CE003C08DE001C08EE00E94A84EBC01C5
:108B900082E00E94AE181F910895CF93C82F181637
:108BA000B4F480E00E94A7456C2F80E090E00E9422
:108BB000DB58892B39F440E065E08CE190E00E94BD
:108BC000CD5807C08C2F0E94E958892B11F082E004
:108BD00001C083E00E94A74584EF91E00E949515B3
:108BE000CF910895CF93DF93EB0182309105E1F1AE
:108BF000833091051CF4892B29F04EC083309105F8
:108C000071F14AC08A81882309F446C060E081E09E
:108C10000E9426178C819D8197FF0CC08EE590E104
:108C20009F938F9382E08F930E9404190F900F906F
:108C30000F900FC09F938F9383E690E19F938F9344
:108C400082E08F930E9404190F900F900F900F9065
:108C50000F9083E08F8B81E0888F8E8B1DC040E06A
:108C600050E00E94DA3E18C08A81882321F08C816E
:108C70000E94CD4505C081E00E94A74581E08A831E
:108C800080E090E00E94E2588C839D8381E08B839A
:108C90008FE790E08E839F8380E090E0DF91CF911B
:108CA00008950F931F93CF93DF938B01813091052C
:108CB00071F0823091051CF4892B79F0B4C08230B8
:108CC000910509F43FC083309105B9F1ACC08FEF35
:108CD0009FEFFB0184839583A6C0FB0182818823DB
:108CE00009F4A1C060E081E00E942617F8018481A8
:108CF000958197FF0CC087E690E19F938F9382E068
:108D00008F930E9404190F900F900F900FC09F93A4
:108D10008F938EE690E19F938F9382E08F930E94D2
:108D200004190F900F900F900F900F9085E0F801AD
:108D3000878B81E0808F868B76C040E050E00E9478
:108D4000DA3E71C0FB018281882389F1C481D5811B
:108D5000C038D10520F48C2F0E94CD452EC0F8E2FA
:108D6000C030DF07A0F480E00E94A7458D2F99272F
:108D7000806C682F80E190E00E94DB58009729F416
:108D80006C2F81E190E00E94DB58892B11F082E08A
:108D900007C041E065E08CE190E00E94CD5883E09F
:108DA0000E94A74584EF91E00E94951506C081E0DE
:108DB0000E94A74581E0F8018283F80184819581B2
:108DC00001978F37910540F480E090E00E94E258CF
:108DD000F8018483958315C080E190E00E94E258F9
:108DE000982F8827F8018483958381E190E00E9481
:108DF000E258F80124813581282B392B3F732483D5
:108E00003583F80184819581805098422CF08FEF52
:108E10009FEFF8018483958381E0F80183838FEFCE
:108E200097E28683978380E090E0DF91CF911F9156
:108E30000F9108951F93CF93DF93EB01122F823090
:108E4000910519F1833091052CF4009761F0019799
:108E500029F02EC0863091055CF512C0842F0E9447
:108E6000DB4F898325C060E081E00E94261789815D
:108E7000810F0E94004FBC0182E00E94AE1818C012
:108E800042E050E00E94DA3E13C08A81882351F00C
:108E90008981882321F0842F0E94E54F03C0842F0D
:108EA0000E94ED4F90E08A81882309F491E09A8333
:108EB00080E090E0DF91CF911F91089522E0422F52
:108EC0000E941A47089522E048E00E941A47089538
:108ED00020E041E00E941A4708950F931F93CF931B
:108EE000DF938C01EB0124E0422F0E941A470230ED
:108EF000110529F48A81882311F40E94781D80E0ED
:108F000090E0DF91CF911F910F910895FF920F9301
:108F10001F93CF93DF93EC018B01F42E0E94BA4F85
:108F2000FC01C230D10509F471C0C330D1052CF465
:108F30002097C9F0219771F07DC0C430D10509F4A4
:108F40004DC0C430D1050CF44DC0C530D10509F475
:108F500049C070C0FF2019F08485E80155C08385A1
:108F6000F801818367C060E081E00E942617E80174
:108F70009981FF20F9F0892F6AE00E94C167892F4B
:108F800099279F938F9389810E94C16799279F9307
:108F90008F9382E790E19F938F9382E08F930E945B
:108FA0000419EDB7FEB737960FB6F894FEBF0FBEA3
:108FB000EDBF40C082E3989FC00111249F938F931F
:108FC0008AE790E19F938F9382E08F930E94041928
:108FD0000F900F900F900F900F902CC0F80181818F
:108FE0008F3F41F1FF2019F040E05FEF02C04BEEF0
:108FF0005FEFB801CE010E94DA3EFF20D9F0E80110
:1090000089818823B9F481E0898314C0E8018A81C9
:10901000882341F09981FF2011F0948701C0938744
:109020000E94414F90E0F8018281882309F491E089
:10903000E8019A8380E090E0DF91CF911F910F913A
:10904000FF90089540E00E948647089541E00E9405
:1090500086470895CF93DF93EB018230910559F154
:10906000833091052CF4009759F0019729F02FC017
:109070008630910564F51AC00E94C24F898327C0CB
:1090800060E081E00E94261789819927880F991F47
:10909000880F991F8A5F984FBC0182E00E94AE182A
:1090A00060E870E182E00E94AE1811C048E050E034
:1090B0000E94DA3E0CC08A81882319F089810E94BF
:1090C000C64F90E08A81882309F491E09A8380E07A
:1090D00090E0DF91CF910895CF93DF93EB01823041
:1090E000910561F18330910534F4009749F08130A6
:1090F0009105F1F04BC0863091050CF047C018C0C7
:109100008A81882309F442C060E081E00E9426172A
:109110006981623020F082E10E94A84E04C0862F4F
:109120008A5F0E94004FBC0182E00E94AE182EC0F0
:1091300042E050E0BE010E94DA3E28C08A818823C6
:1091400019F18981823018F48E5F89831FC060E035
:1091500081E00E9426178981833051F48FE00E94BC
:10916000A84EBC0182E00E94AE180E94675D09C053
:1091700080E10E94A84EBC0182E00E94AE180E94CD
:109180002F5E8FEF9FEF04C081E08A8380E090E044
:10919000DF91CF910895CF9380919B04803178F037
:1091A00010929B0410929C0461E0862F0E94261767
:1091B000CEE085EA0E94EE16C150C7FFFACF60915B
:1091C0009B0481E00E94261780919C04992781309E
:1091D000910559F0823091051CF4892B21F014C0BF
:1091E000029739F011C085E001C084E00E94EE16BC
:1091F0000BC080E20E94EE1685E00E94EE16809180
:109200009B048F5F80939B0480919C048F5F80936D
:109210009C04833010F010929C04CF910895CF935A
:10922000DF93EB018230910509F1833091051CF445
:10923000892B31F049C0863091050CF045C011C032
:1092400060E081E00E9426178A81882311F081E185
:1092500001C083E10E94A84EBC0182E00E94AE18CA
:1092600033C040E050E00E94DA3E2EC08A8188235D
:1092700029F10E94361D64E971E084E00E945518CE
:109280006CE871E085E00E94551868EC70E08BECAA
:1092900098E40E945F1760E0862F0E94261783E003
:1092A0000E94A84EBC0182E00E94AE180E941B24BE
:1092B0000E94565C0E94634F0E94B55190E08A81E3
:1092C000882309F491E09A8380E090E0DF91CF91C8
:1092D0000895CF92DF92EF92FF920F931F93CF9357
:1092E000DF93029709F0CEC060E0862F0E94261718
:1092F00080E20E94EE1660E081E00E94261780E086
:109300000E94030D68E870E182E00E94AE1821E03F
:109310004EE468E086E00E94740E6D9880E00E9442
:109320007D1080E00E941712CC24DD248EEF0E9475
:10933000861280E00E9430198F5F9F4FD1F781E045
:109340000E9430198F5F9F4FD1F7A8950E94D316C6
:109350008331910509F488C08B30910509F484C0EC
:109360000A9701F581C0CF3FD10551F0209741F018
:109370006C2F80E00E947E186C2F81E00E947E1886
:10938000CF33D10519F0CB32D10519F4B4E8CB2E87
:10939000D12CC332D10511F0AA9721F4A6E0CA2E30
:1093A000A1E0DA2E0E94B312EC018F5F9F4FD9F635
:1093B000C114D10409F4BACFE090F206F090F3069C
:1093C0000091F4061091F50688EC90E0A0E0B0E082
:1093D000E80EF91E0A1F1B1F3BC0A8950E943019FA
:1093E000EC019FEFCF3FD90721F481E00E943019B3
:1093F000EC01AFEFCF3FDA0721F18C2F0E948612EC
:109400000894C108D108E090F206F090F3060091AC
:10941000F4061091F50688EC90E0A0E0B0E0E80ECC
:10942000F91E0A1F1B1F0DC0CF3FD10551F0209719
:1094300041F06C2F80E00E947E186C2F81E00E942A
:109440007E180E94B312EC019FEFCF3FD90761F75E
:10945000C114D10409F468CFC801B7010E945E139A
:10946000882309F4BACF60CF81E00E947D1081E0AB
:109470000E9417126D9A0E94C24F21E04EE468E0EC
:109480000E94740E80E090E0DF91CF911F910F91C8
:10949000FF90EF90DF90CF900895CF93DF93EB0193
:1094A0008230910509F440C0833091052CF4009777
:1094B00071F0019731F048C0863091050CF044C03E
:1094C0002EC00E94BA4FFC01868189833DC060E0B6
:1094D00081E00E9426176981662369F484E10E9475
:1094E000A84E9F938F9382E08F930E9404190F9050
:1094F0000F900F9029C085E0689FC00111249F93B1
:109500008F9385E990E19F938F9382E08F930E94E0
:1095100004190F900F900F900F900F9015C049EC09
:1095200050E00E94DA3E10C08A81882339F00E9400
:10953000BA4F2981FC0126830E94414F90E08A8125
:10954000882309F491E09A8380E090E0DF91CF9145
:109550000895CF93DF93EB018130910569F082305C
:1095600091051CF4892B81F049C08230910539F1B5
:1095700083309105F9F042C00E94BA4FFC0180850A
:1095800099278C839D833AC060E081E00E94261772
:109590008C819D819F938F938BE990E19F938F9313
:1095A00082E08F930E9404190F900F900F900F90FC
:1095B0000F9024C040E050E00E94DA3E1FC08A8134
:1095C000882361F483E08B8380E290E08E839F8325
:1095D00091E0988F82E08F8B9E8B0AC01E8A0E943A
:1095E000BA4F2C81FC0120872093890A0E94414FA9
:1095F00090E08A81882309F491E09A8380E090E0EA
:10960000DF91CF910895EF92FF920F931F93CF9325
:10961000DF938C01EB010E94BA4F7C0102301105EF
:1096200009F463C00330110544F40115110571F00C
:109630000130110509F446C072C00330110509F468
:109640003DC0063011050CF06AC03CC08A818823F9
:1096500009F465C0F7018085882309F460C060E0E3
:1096600081E00E9426178C819D819F938F9380EAD1
:1096700090E19F938F9382E08F930E94041960E0A2
:1096800089810E940F59082F61E089810E940F593A
:10969000182FC0E80F900F900F900F900F9094E04C
:1096A000802F8C2309F096E0812F8C2309F09F5F97
:1096B000892F0E94EE16C69591F731C01E8A81E06F
:1096C0000E943059F70180859927AC01BE01C8017D
:1096D0000E94DA3E8981992701968C839D838B8134
:1096E0008230E9F488E08B831AC02A81222391F426
:1096F00081E090E08C839D83F701808599278E839C
:109700009F8311E01A83822F0E943059188F85E0C1
:109710008F8B1E8B88E08B838C818150898380E0C6
:1097200090E0DF91CF911F910F91FF90EF900895FE
:10973000CF92DF92EF92FF920F931F93CF93DF931D
:109740008C01C62F0E944D180E94BA4F6C01C23284
:1097500008F05CC0DD277E01EE0CFF1CEE0CFF1C48
:1097600082E292E0E80EF91EF8018281882311F06E
:1097700080E001C082E00E94EE16F6018581992703
:1097800081309105A1F0823091051CF4892B39F0CC
:1097900029C08230910599F00397C9F023C034E0C5
:1097A000CC0FDD1F3A95E1F7CF51D24F17C024E01F
:1097B000CC0FDD1F2A95E1F7CF52D44F0FC094E0B4
:1097C000CC0FDD1F9A95E1F7CF53D64F07C084E049
:1097D000CC0FDD1F8A95E1F7CF54D84FBE0182E050
:1097E0000E94AE18E701EA81FB81309721F0B801B1
:1097F00080E090E00995F8018689882329F067893F
:10980000808D0E942F1702C00E943517DF91CF91E3
:109810001F910F91FF90EF90DF90CF90089560E03F
:10982000E2E2F2E0482F552747FD509520E030E076
:10983000808199278417950711F4C90108956F5FF6
:109840002F5F3F4F3496613298F38FEF9FEF08956B
:109850000895BF92CF92DF92EF92FF920F931F93E2
:10986000CF93DF93CDB7DEB76B970FB6F894DEBF1B
:109870000FBECDBFB82E20E2281718F480E090E08C
:10988000FDC16E010894C11CD11C8BE1F60111923F
:109890008A95E9F7A895EB2DFF27EE0FFF1FEE0F36
:1098A000FF1FEE5DFD4F0280F381E02D309721F028
:1098B000B60181E090E009956B2DC6010E94984B9E
:1098C0000E94460DEB2CFF24EE0CFF1CEE0CFF1C3F
:1098D00082E292E0E80EF91E0E94D316AC018A30B3
:1098E000910509F4E7C08B30910564F4009709F401
:1098F00008C1181619060CF41CC14F5F5F4F09F41C
:10990000ACC1DECF8331910509F48CC0843191055F
:1099100044F48B30910509F485C0419709F499C14D
:10992000CFCF8431910519F0459741F1C9CFF601A8
:109930008281882381F0F70122813381211531054D
:1099400031F0BE016F5F7F4F84E090E07FC1F60190
:1099500081818F5F26C0F7019081FFE1FB1534F014
:10996000F7018481891711F4B3942FC0892F0E94C5
:109970000F4C682F772767FD70953EC0F6018281F6
:10998000882389F0F701228133812115310531F0D7
:10999000BE016F5F7F4F85E090E058C1F601818185
:1099A0008150818367C16B2DF7019081BB2091F0BD
:1099B0002CEF3FEFE20EF31EF701808124E030E050
:1099C000E20EF31E891731F4BA946B2D772767FDE9
:1099D000709512C03FE13B1564F0D7011496F70172
:1099E0008481891731F46F5F60321CF414968C9176
:1099F000F8CF772767FD7095B62EE62FFF27EE0F7D
:109A0000FF1FEE0FFF1FEE5DFD4F0280F381E02D83
:109A1000309709F42FC1BE016F5F7F4F81E090E066
:109A2000099528C1F7019181992361F1092F112727
:109A300003561B4FF801808118162CF0892F0E94C5
:109A40000F4CF8018083F7018181E82FFF27E3564F
:109A5000FB4F80810E94294C282F332727FD30950A
:109A6000F7018181E82FFF27E356FB4FC90137FF3C
:109A700004C088279927821B930B808337FFFAC085
:109A8000B1943AC0F701228133812115310551F09B
:109A9000BE016F5F7F4F82E090E0F9010995992345
:109AA0007CF319C0F6018281882309F491E0F60164
:109AB0009283E0C0F60182818823F1F0F7012281D0
:109AC000338121153105A9F0BE016F5F7F4F83E01F
:109AD00090E0F9010995F6018281882309F0CAC056
:109AE000F70122813381BE016F5F7F4F81E090E0FB
:109AF000ADC0F6011282BEC08B2D992787FD9095CF
:109B0000BDC0F6018381813009F4DACE883089F452
:109B100081E00E94305960E0F60181810E940F5976
:109B200061E0F60181810E940F5980E00E94305966
:109B3000A1C0F601838199278530910509F454C0AD
:109B40008630910584F48230910581F1833091054E
:109B50001CF40197B9F08EC08330910599F00497F9
:109B600009F43EC087C08730910509F456C087309C
:109B700091050CF44CC08830910521F0099709F447
:109B800053C078C0F60186819781892B21F48FEF2D
:109B90009FE786839783F6018681978184179507CF
:109BA0000CF468C01482158282E08383F6018481FC
:109BB00095819C0163E0220F331F6A95E1F7280F1E
:109BC000391F280F391F240F351F37FD53C08681D9
:109BD0009781821793070CF44DC0248335834AC0C4
:109BE000F601108685E08383F60190858AE0989FD0
:109BF00090011124240F351F2F3F310509F008F47F
:109C000020878EEF9FEFF601818F928F33C048300F
:109C1000510584F5F60141872DC04230510554F5B8
:109C2000F601418F528F26C0F6018181E80FF11DA8
:109C3000842F805D8287F7012281338121153105D0
:109C4000C9F0BE016F5F7F4F82E090E0F901099596
:109C500011C080E00E94030D0DC0F60183818830A1
:109C600009F02ECEBE016F5F7F4F80E090E00E9432
:109C7000034B26CE6B2DCE01019620CE6B960FB6F0
:109C8000F894DEBF0FBECDBFDF91CF911F910F9132
:109C9000FF90EF90DF90CF90BF900895CF93C82FA3
:109CA0006CE571E080E00E94551864E671E082E0A6
:109CB0000E94551864E871E084E00E9455186CE732
:109CC00071E085E00E94551864E771E086E00E942B
:109CD00055186CE671E087E00E94551880919D044C
:109CE000813210F010929D04C7FD04C08C2F0E9499
:109CF000294C0EC080919D040E94294C992787FD14
:109D0000909597FF03C0909581959F4F80939D04F8
:109D10006CE372E080E00E9455186CE172E082E032
:109D20000E94551864EF71E084E00E9455186CEEB3
:109D300071E085E00E94551864EE71E086E00E94B3
:109D400055186CED71E087E00E945518CF91089589
:109D5000CF93C82F893118F082E999E12CC00E9475
:109D6000BA4FFC01858199278230910581F08330BB
:109D700091051CF4019721F018C0039779F015C0E4
:109D800081E1C89FC00111248751984E14C081E120
:109D9000C89FC0011124805C994E0DC081E1C89F0D
:109DA000C001112489569B4E06C081E1C89FC001A5
:109DB000112482519D4ECF910895882319F08FE987
:109DC00099E108950E94BA4FFC018581992782305C
:109DD000910561F0833091051CF4019721F00CC0CE
:109DE000039739F009C08DED92E108958CEC92E172
:109DF00008958BEB92E108958AEA92E1089508951F
:109E0000CF93C82F883018F08FEA99E138C00E94AC
:109E1000BA4FFC01858199278230910599F08330F2
:109E200091051CF4019721F021C00397A9F01EC0F1
:109E30008C2F992754E0880F991F5A95E1F7865D7A
:109E40009D4E1DC08C2F992744E0880F991F4A957D
:109E5000E1F786559E4E13C08C2F992734E0880F6A
:109E6000991F3A95E1F7865D9E4E09C08C2F992780
:109E700024E0880F991F2A95E1F786559F4ECF91D0
:109E80000895EF92FF921F93CF93DF9386EAE82E17
:109E900084E0F82EC0E0D0E01FE1CE010E946262B3
:109EA000F70161917F01861719F0CE010E947B6254
:109EB000A8951150219617FFF0CFDF91CF911F91F8
:109EC000FF90EF9008959091AB04943008F091E0EA
:109ED0008FE0E6EAF4E011928A95E9F788E1809351
:109EE000AA049093AB0481E08093A70484E180935B
:109EF000AC0482E08093B10482E38093B2040E94B8
:109F0000414F089540E250E060E070E086EA94E05E
:109F10000E946A628091A8049091A9048F5F9F4F6C
:109F200011F40E94634F8091A704883018F081E0FB
:109F30008093A7048091B3049091B404885F974004
:109F400020F01092B4041092B3048091AB048430DA
:109F500010F01092AB048AEF9FEFA1E0B0E0ABBF2E
:109F6000FC0187918F3F21F0882311F080936F00CF
:109F70000895089586EA94E008958093AB040E94C2
:109F8000414F08958091A70499270895CF93C82F32
:109F9000883008F0C7E08091A704C81751F0C0933B
:109FA000A7040E94414F21E04EE468E08C2F0E94FC
:109FB000740ECF91089520E030E09091A60498238C
:109FC00011F021E030E0C90108959091A604982B8A
:109FD0009093A6040E94414F0895982F90958091E8
:109FE000A60489238093A6040E94414F08958CEF14
:109FF0009FEFA1E0B0E0ABBFFC0187919791A791E3
:10A00000B691B070BC01CD0108958FEF9FEFA1E034
:10A01000B0E0ABBFFC018791992708950E944B24C3
:10A02000FC01892BB9F0A6ECB4E043E02D913C9102
:10A030001197808191812817390729F082819381B6
:10A040002817390719F41D921C9211974150139645
:10A0500047FFECCF089508959F92AF92BF92CF92A1
:10A06000DF92EF92FF920F931F93CF93DF93CDB7C1
:10A07000DEB726970FB6F894DEBF0FBECDBFC82E51
:10A080007B01942ECE0101960E94E751DD2496ECCF
:10A09000A92E94E0B92EF501808191818E159F053E
:10A0A00009F08AC082818F5F8283843008F4B9C04E
:10A0B000C7010E9473248C01009709F4B4C0FFEF1C
:10A0C000CF1619F5992029F0FC0164817581C7012B
:10A0D00017C0FC01448155816681C7010E94B028E8
:10A0E000F80180850E941129F801828193810097EF
:10A0F00049F00E947324FC01648175818081918103
:10A100000E94FA280E941E2851C0992049F0FC01A3
:10A110004481558160E0CE0101960E94CA5139C048
:10A12000FC01448155816681CE0101960E94CA518D
:10A13000AE014F5F5F4F67E08C2D0E946A52F801BD
:10A1400080858F778B830E9480528823E1F3AE0154
:10A150004F5F5F4F69E08C2D0E946A52F801828147
:10A1600093810E944B248C010097D1F0FC01608107
:10A170007181CE0101960E94E751F8014481558119
:10A1800060E0CE0101960E94CA510E94805288234D
:10A19000E1F3AE014F5F5F4F68E08C2D0E946A5281
:10A1A00040E050E06DE08C2D0E946A52F501108273
:10A1B000118281E090E037C0D39483E090E0A80E54
:10A1C000B91E93E09D1508F066CFDD2406EC14E07F
:10A1D000F80180819181892BA1F40E940F288E15AE
:10A1E0009F0519F40E94242807C0AE014F5F5F4FFE
:10A1F00065E08FEF0E946A52F801E082F1821282DC
:10A2000006C0D3940D5F1F4FF3E0FD1508F783E000
:10A210008D1538F4AE014F5F5F4F66E08FEF0E94FF
:10A220006A5280E090E026960FB6F894DEBF0FBE2B
:10A23000CDBFDF91CF911F910F91FF90EF90DF90F5
:10A24000CF90BF90AF909F9008950F931F93CF939F
:10A25000DF93082FEB01672B79F010E040E0BE019F
:10A26000802F0E942C50882339F40E94805288232A
:10A27000E1F31F5F143190F3DF91CF911F910F91A4
:10A2800008958F929F92BF92CF92DF92EF92FF92AA
:10A290000F931F93CF93DF93CDB7DEB726970FB6FB
:10A2A000F894DEBF0FBECDBFB82E4B016A01CB01C3
:10A2B0000E9473248C01892B09F445C0C6010E94B9
:10A2C00073247C01892B09F43EC0F80180850E942B
:10A2D00003288C01F70180850E940328081B190BB5
:10A2E000C80117FF03C0909581959F4F0297E4F036
:10A2F000FFEFBF1621F481E00E94702924C086E0A0
:10A30000FE01319611928A95E9F781E08983AE01C9
:10A310004F5F5F4F61E28B2D0E946A5214C0B601FD
:10A32000C4010E9459270FC010E041E0B6018B2DF7
:10A330000E942C50882399F70E9480528823E1F3D1
:10A340001F5F143190F326960FB6F894DEBF0FBE50
:10A35000CDBFDF91CF911F910F91FF90EF90DF90D4
:10A36000CF90BF909F908F9008950E94361DF894D3
:10A37000FFCF682790E027E0862F86959F5F60FFDC
:10A3800003C0682F622701C0682F9830A8F3862F7A
:10A3900099270895FC01262F862F8F778283269593
:10A3A0002074CA01892F9927869586958F73822BF1
:10A3B0008383CA0123E0969587952A95E1F78F77E5
:10A3C0008483842F8295807F8F7785830895FC0115
:10A3D000CB01262F2F772083880F892F881F990B79
:10A3E00091958F7781830895803480F4E82FFF273B
:10A3F000662329F0E75FFA4F8AE080830895E75FDC
:10A40000FA4F8081882311F0815080830895089548
:10A41000EF92FF920F931F93CF93DF93782FC62F66
:10A420007A01A8958091F604282F33278091F704AC
:10A43000992701972817390741F08091F604833056
:10A4400039F48091F704882319F480E090E03BC050
:10A450009091F60489E0989F800111240E521B4FC1
:10A46000872F8068F8018083682F80E00E94B951AF
:10A47000F801C1836C2F0E94B951982FE8012296F0
:10A4800005E0E114F10431F0F70181917F018F774C
:10A49000888301C018826991892F0E94B951982F31
:10A4A000015007FFEECF87FD909598838091F604C9
:10A4B0008F5F8093F6048091F604843010F0109240
:10A4C000F60481E090E0DF91CF911F910F91FF9012
:10A4D000EF9008950F931F93CF93DF93082F162FBC
:10A4E000EA0102C00E94460DAE01612F802F0E943A
:10A4F00008528823B9F3DF91CF911F910F910895EE
:10A500009F92AF92BF92CF92DF92EF92FF920F9302
:10A510001F93CF93DF93CDB7DEB76C970FB6F89448
:10A52000DEBF0FBECDBF99245EC227FF05C01092CB
:10A53000FF048FEF809301058091FF04893040F480
:10A54000E82FFF27E050FB4F20838F5F8093FF04AD
:10A550008091FF04893009F046C28091000587FF91
:10A5600042C2E0E0EE2EE5E0FE2E90E017E0F701BB
:10A5700081917F01682F892F0E94B951982F115026
:10A5800017FFF5CF87FD909580910805981709F082
:10A5900025C2FF248091000588230CF01FC27FE7AD
:10A5A000B72EB82230910205C32EDD244091030559
:10A5B000842F99279695982F882797958795C82A4D
:10A5C000D92A20910105822F9927AA27BB27FC01B0
:10A5D0003197E334F10508F001C2EA5BFF4FEE0F5B
:10A5E000FF1F0590F491E02D0994109104058091CE
:10A5F0000505282F332726FD1068322F2227330F19
:10A60000330F8091060599278F77907043E0880F6C
:10A61000991F4A95E1F7282B392B80910705992737
:10A620008077907004E0959587950A95E1F7282B3F
:10A63000392B41E0B901C6010E941E2741E0612F7C
:10A64000C6010E949B26C6010E940E50C3C1809184
:10A650000405992790E4899F902D88271124C82A02
:10A66000D92A60910505662351F061E0C6010E9478
:10A67000F05FC601969587950E940562ABC1C60141
:10A680000E94F05FA7C180910405682F7727809111
:10A690000505282F3327C901877090709695982F4C
:10A6A000882797958795682B792B20743070220F17
:10A6B000331F80910605822B482FC6010E94F02788
:10A6C00089C180910405E82EFF240027112780917D
:10A6D000050599279695982F882797958795AA27F6
:10A6E00097FDA095BA2FE82AF92A0A2B1B2B8091F7
:10A6F0000605992790E4899F902D88271124AA2781
:10A7000097FDA095BA2FE82AF92A0A2B1B2B209136
:10A710000705822F9927AA27BB2787709070A07002
:10A72000B07035E1880F991FAA1FBB1F3A95D1F76A
:10A73000E82AF92A0A2B1B2B269526952695D8015F
:10A74000C7010197A109B1098F5F9F4FAF4FB0407B
:10A7500008F040C1A601C801B7010E94115D3AC1CD
:10A760000E94420D843009F435C1809102050E9497
:10A77000030D882309F42EC184E00E94FF612AC1E1
:10A78000C114D10409F426C1B6018B2D0E942551B4
:10A7900021C160910405C6010E94AD25809102058A
:10A7A0008A87809103058B87C6010E948F258C873D
:10A7B000AE01465F5F4F69E0A7C01AE0E12EF12CC1
:10A7C000EC0EFD1EAE01405F5F4FBE01645F7F4F28
:10A7D000C6010E94BB5B6C018F778A87CC0CCD2CA5
:10A7E000CC1CDD08D1948C2D8F778B8788898D8741
:10A7F00089898E871F86A70161E18B2D0E946A528D
:10A800008E010F5F1F4FF80194E08189818791507D
:10A81000319697FFFACFA70162E18B2D0E946A5211
:10A82000F80193E0868981879150319697FFFACF9E
:10A83000A70163E169C0A3E0FA2E33E0F30E83E0E1
:10A84000F80E8601243199F480910405C82EDD2488
:10A850008091050599279695982F88279795879534
:10A86000C82AD92A809106058C8F188A23C0AE0188
:10A87000405F5F4FBE01645E7F4FC6010E94BB5BBD
:10A880006C0194E0EAE0EF1588F0DE01AF0DB11D38
:10A890005096E92FFF27E050FB4F80818D939F5FFB
:10A8A000F394973018F4FAE0FF1598F7FE01EF0DD6
:10A8B000F11D108A9E01205F3F4F4C8DB601C801EB
:10A8C0000E94FB5A8C018F778A87000F012F001F8F
:10A8D000110B1195802F12C0213121F4C6010E9465
:10A8E000FB5B03C0C6010E942D5C6C018F778A87D9
:10A8F000CC0CCD2CCC1CDD08D1948C2D8F778B8784
:10A90000AE01465F5F4F60E18B2D0E946A5262C0CC
:10A91000C6010E94F85A5EC080910405282F332793
:10A920008091050599279695982F88279795879563
:10A93000282B392BA901B6018B2D0E9441514AC009
:10A94000C6010E94792746C0BB24E9E0F5E0819169
:10A95000882369F442E055E064E08B2D0E946A523E
:10A960008091F9048B1538F4B092F90404C0B394C3
:10A970003FE33B1560F782E08093FA042BC080919F
:10A98000FA04833038F583E08093FA043093FB04B3
:10A990004093FC04809104058093FD041092FE0412
:10A9A00019C08091FA048230A8F482E08093FA04FE
:10A9B0003093FB044093FC041092FD040BC0909173
:10A9C000FA04992339F481E08093FA043093FB046C
:10A9D0009093FC0461E08B2D0E94F4511092FF04CF
:10A9E0008FEF809301050E94B3129C018FEF2F3FE0
:10A9F000380709F09ACD0E9475120A970CF421C10C
:10AA00009091F6048091F704981711F19091F70452
:10AA100089E0989F70011124E2EDF4E0EE0EFF1E34
:10AA200008E010E0F70181917F010E948612015039
:10AA3000104017FFF7CF8091F7048F5F8093F704E2
:10AA40008091F704843008F4FCC01092F704F9C038
:10AA50007E010894E11CF11C57018091F8048034B8
:10AA600029F06091FA04662309F475C08FEF898399
:10AA70000894E11CF11C8091FA049927813091051A
:10AA8000C9F0823091051CF4892B39F059C082300D
:10AA9000910519F10397C1F153C080E4F701819347
:10AAA0008091FB04982F97708F5F8093FB049193A4
:10AAB0007F0148C081E4F70181938091FB04877096
:10AAC00081938091FC04982F9F778F5F8093FC0483
:10AAD00091937F018091FC0431C082E4F70181935E
:10AAE0008091FB04877081938091FC048F77819320
:10AAF0008091FD04982F9F778F5F8093FD04919341
:10AB00007F018091FD041AC083E4F7018193809155
:10AB1000FB04877081938091FC048F7781938091EF
:10AB2000FD048F7781938091FE04982F9F778F5F2C
:10AB30008093FE0491937F018091FE0487FF02C001
:10AB40001092FA048091FA04882309F059C0809188
:10AB5000F8048F5F53C08134A1F58FEF8983089487
:10AB6000E11CF11C83E0F70181937F018F010894C0
:10AB7000E11CF11C0E94420D8F77F80180838091C7
:10AB8000F8048F5F8093F8040E940C288C01FC016C
:10AB9000868581FF13C0808191810E940E5041E023
:10ABA000F8016089808191810E949B2641E0F80133
:10ABB00064817581808191810E941E2751E0952ECC
:10ABC0001FC0803410F06093F8048091F80480680E
:10ABD00089830894E11CF11C82E0F70181937F01D5
:10ABE0008091F8040E94F4518091F8048F5F809363
:10ABF000F8049091F904981718F480E48093F8040D
:10AC0000CE010996E816F90620F4F70111927F01AA
:10AC1000F9CFDD24750107E010E0F70160818D2D8B
:10AC20000E94B951D82EF70181917F010E948612AE
:10AC30000150104017FFF1CFD7FCD0948D2D0E940A
:10AC40008612A895892D99276C960FB6F894DEBFC9
:10AC50000FBECDBFDF91CF911F910F91FF90EF906D
:10AC6000DF90CF90BF90AF909F900895CF93DF93E8
:10AC7000CDB7DEB726970FB6F894DEBF0FBECDBFB7
:10AC800036E0FE01319611923A95E9F74983AE011B
:10AC90004F5F5F4F0E946A5226960FB6F894DEBF50
:10ACA0000FBECDBFDF91CF9108951F93CF93DF9358
:10ACB000EC0110E001C0A8950E94961D8823D9F3ED
:10ACC00010C0A89504C081E090E00E9495150E94F4
:10ACD000961D8823C1F361E080E090E00E94BB1BD9
:10ACE00021970E94A61D882311F4209751F70E94F6
:10ACF000A61D811111E0C5E00EC063E080E090E088
:10AD00000E94BB1B0E94AA1D01C0A8950E94961D0F
:10AD10008823D9F3C1500E94A61D882311F0CC23AB
:10AD200061F7CC2309F41C2F812F9927DF91CF9154
:10AD30001F910895EF92FF921F93CF93DF937C01B1
:10AD4000CFEFDFEF10E0612FC7010E94341C80E0DD
:10AD500090E00E945556882311F0C12FDD271F3F38
:10AD600049F483E090E00E945556882331F0CFEFFC
:10AD7000D0E005C01F5FD7FDE6CFD7FD14C01C2F64
:10AD8000CFEFDFEF612FC7010E94341C83E090E01A
:10AD90000E945556882311F0C12FDD27112319F089
:10ADA0001150D7FDEFCFCE01DF91CF911F91FF90D2
:10ADB000EF9008955F926F927F928F929F92AF92E1
:10ADC000BF92CF92DF92EF92FF920F931F93CF9398
:10ADD000DF93CDB7DEB726970FB6F894DEBF0FBE70
:10ADE000CDBF782E6B01A42E522E8091620082601E
:10ADF0008093620080E00E94791886E0FE0131961F
:10AE000011928A95E9F7AE014F5F5F4F62E28FEFD3
:10AE10000E946A520E94B71D83EC87B98FEE86B9F3
:10AE20006FEF862E962E662480E00E94030D82E34B
:10AE300090E00E94951584E00E94030D84E690E066
:10AE40000E949515E090F206F090F3060091F4064A
:10AE50001091F50680ED97E0A0E0B0E0E80EF91E55
:10AE60000A1F1B1FBB2410924A05109249052BC0D4
:10AE70000E94B21DAC012091490530914A05C901DB
:10AE8000885A9D4F8417950734F0C9018855924020
:10AE90004817590744F450934A0540934905BB208D
:10AEA00059F0BA9409C0240F351F35952795309372
:10AEB0004A0520934905B39494E09B1550F08AE02D
:10AEC00090E00E949515C801B7010E945E13882387
:10AED00079F28091490590914A0544975CF584E3A5
:10AEE00093E00E94AD1D83E090E00E94555610E073
:10AEF000412F612F80E090E00E94FB1B83E090E0F7
:10AF00000E945556811111E041E060E080E090E040
:10AF10000E94FB1B83E090E00E94555681111F5F49
:10AF2000113041F484E190E090934A058093490503
:10AF300045E0B42E8091490590914A054497855A81
:10AF40009B4018F4B4E0BB15D0F060E081E00E94B3
:10AF500026178091490590914A05449714F485E19C
:10AF600001C087E10E94A84EBC0182E00E94AE1899
:10AF700080E00E94030D88EE93E00E949515809179
:10AF8000490590914A05805E9C4F0E94AD1D86E95F
:10AF900090E00E9495150E94420D843009F0CFC0C8
:10AFA000072D11270330110509F447C0043011059E
:10AFB0004CF40130110539F102301105FCF4012B7C
:10AFC00071F0ACC0053011050CF4A8C007301105B4
:10AFD0000CF453C0093011050CF0A0C06FC0452D12
:10AFE0006A2DC6010E94DB1B8FE090E00E9455563F
:10AFF000882309F496C0852C992493C06A2DC60134
:10B000000E944D1C4CC040E06A2DC6010E94FB1BF3
:10B0100083E090E00E945556882309F046C041E045
:10B020006A2DC6010E94FB1B83E090E00E945556EA
:10B03000882309F476C0480174C010E0012F1695EA
:10B0400040E0602FC6010E94FB1B83E090E00E945D
:10B050005556882309F410680F5F083080F3612F7C
:10B06000C6010E94661C83E090E00E94555688232A
:10B0700009F457C0812E992454C061E085E090E026
:10B080000E941B1C8FE090E00E945556C6018770FD
:10B090009070E5E07E1661F46A2D0E941B1C8FE023
:10B0A00090E00E9455568823E1F18824992439C004
:10B0B0000E949A564C0133E0632E33C0C601969528
:10B0C000879596958795682F6F5F85E090E00E9441
:10B0D0001B1C8FE090E00E945556C6018370907053
:10B0E000F7E07F1661F46A2D0E941B1C8FE090E050
:10B0F0000E945556882341F08824992405C00E9457
:10B100009A564C0193E0692E61E085E090E00E9440
:10B110001B1C8FE090E00E94555603C08FEF882ED5
:10B12000982E80E00E94030D97FE09C08CE291E00A
:10B130000E949515639422E0261508F075CE16B886
:10B1400086B187B90E94BA4FFC0184810E947918A8
:10B1500081E08983AE014F5F5F4F62E28FEF0E9413
:10B160006A52809162008D7F80936200C4012696AE
:10B170000FB6F894DEBF0FBECDBFDF91CF911F9108
:10B180000F91FF90EF90DF90CF90BF90AF909F9086
:10B190008F907F906F905F900895242F462FBC0171
:10B1A00080E00E94DA56089520E0462FBC0181E03D
:10B1B0000E94DA56089520E0462FBC0182E00E94EA
:10B1C000DA56089520E0422FBC0183E00E94DA564F
:10B1D000089520E0482F60E070E085E00E94DA5694
:10B1E0000895992720E0462FBC0185E00E94DA5699
:10B1F0000895992720E0422FBC0186E00E94DA568C
:10B20000089520E0462FBC0187E00E94DA56089599
:10B2100020E0422FBC0188E00E94DA560895880F92
:10B2200061118F5FF894E82FFF27E553F54F908168
:10B2300080918A0A80FD10827894892F9927089539
:10B24000880F61118F5FF894E82FFF27DF01A55F5A
:10B25000B44F8C91E557F54F8083789499270895E2
:10B2600090918A0A882311F0916001C09E7F90938B
:10B270008A0A0895089580E4EBE8FAE011928A952D
:10B28000E9F7089584E0809374001092710082E2DF
:10B290008093700008951F920F920FB60F921124A1
:10B2A0008F939F93EF93FF93809171009927887FED
:10B2B00090708032910509F487C0813291056CF459
:10B2C00080319105D9F0813191051CF40897D1F0B6
:10B2D0007DC0489709F43FC079C080349105A9F139
:10B2E0008134910524F4889709F441C06FC08035FA
:10B2F0009105D9F08835910561F068C080914B05C2
:10B3000087FF02C080EA01C081EA8093730085E86C
:10B3100061C0E0915105F0915205809173008193D5
:10B32000F0935205E093510548C0E0915105F0912A
:10B330005205809173008193F0935205E09351057B
:10B3400080914C05815080934C0580914C05823052
:10B35000F4F285EC3FC080914F0590915005892F04
:10B360009927809373008FEF80934B05D0CF809106
:10B370004B0587FF09C080914F0590915005809340
:10B38000730010924B05C3CF80914D058823E1F0E7
:10B3900080914C05882389F0E0915105F091520588
:10B3A0008191F0935205E093510580937300809151
:10B3B0004C05815080934C05AACF84E9809374009A
:10B3C00081E080934E0508C085EA04C08FEF80932A
:10B3D0004E0584E980937400FF91EF919F918F91C6
:10B3E0000F900FBE0F901F901895809174009927B1
:10B3F00087709070009711F081E090E008950895B3
:10B4000060934C059093500580934F0520934D0514
:10B4100050935205409351058EEF80934B05109247
:10B420004E0585EA80937400089580914E05992712
:10B4300087FD909508950E94005A01C0A8950E942A
:10B44000155A892BD9F380914E05992787FD909540
:10B450000895AB0120E060E134E0880F991F3A9530
:10B46000E1F70E941B5A0895AB0121E060E174E00E
:10B47000880F991F7A95E1F70E941B5A089520E0E2
:10B48000AC0164E080E090E00E941B5A089521E046
:10B49000AC0164E080E090E00E941B5A0895EF92B6
:10B4A000FF920F931F93CF93DF93CDB7DEB7229711
:10B4B0000FB6F894DEBF0FBECDBF7C0119821A8291
:10B4C00009811A8120E0AE014F5F5F4F62E0C80141
:10B4D000E4E0880F991FEA95E1F70E941B5AA895AE
:10B4E00089819A81009719F08E159F0549F7C80147
:10B4F00022960FB6F894DEBF0FBECDBFDF91CF917D
:10B500001F910F91FF90EF9008950F931F93CF938A
:10B51000DF93CDB7DEB722970FB6F894DEBF0FBE2C
:10B52000CDBF8C0101978F5F9340E0F420E0AE0126
:10B530004F5F5F4F62E0C801A4E0880F991FAA9592
:10B54000E1F70E941B5AC8010E944F5A21E0AE0148
:10B550004F5F5F4F62E0F4E0880F991FFA95E1F7C3
:10B560000E941B5A22960FB6F894DEBF0FBECDBFC5
:10B57000DF91CF911F910F9108950F931F93CF9358
:10B58000DF93CDB7DEB764970FB6F894DEBF0FBE7A
:10B59000CDBF8C0101978F5F9340F8F4C8010E94E2
:10B5A000855ACE0141960E943F5A40E150E06FEF2C
:10B5B00070E0CE0101960E949B628B899C898983F1
:10B5C0009A83BE016F5F7F4FC8010E94345A0B8B74
:10B5D0001C8BCE0141960E94475A64960FB6F89490
:10B5E000DEBF0FBECDBFDF91CF911F910F910895A8
:10B5F0000E94BD5A08957F928F929F92AF92BF9200
:10B60000CF92DF92EF92FF920F931F93CF93DF932E
:10B61000CDB7DEB7AA970FB6F894DEBF0FBECDBF89
:10B620007C014B01742E5901232B79F1672B69F1B1
:10B6300080E0E81684E0F80640F5E114F10421F01A
:10B64000C7010E94855A1EC0CE0181960E943F5AB2
:10B650000BA11CA10115110511F4C70112C020E0B6
:10B66000AE014D5D5F4F62E0C80134E0880F991F65
:10B670003A95E1F70E941B5ACE0181960E94475AE3
:10B68000C8017C01E114F10411F4C70158C06E0136
:10B690000894C11CD11CF5018B829C827D82DE0145
:10B6A00016962081222351F0CE014196A817B907A2
:10B6B00028F431962D9320812223C1F7C6014096AC
:10B6C000A817B90708F41C92E9A6FAA6CE01859638
:10B6D0000E943F5AEE24FF240DA11EA10115110561
:10B6E000B1F0A895BE016F5E7F4FC8010E94295A34
:10B6F000C60105964BE050E0BC01CE0146960E9483
:10B70000E462992324F4780109891A89E7CFF601C4
:10B7100000831183A895B60189A59AA50E94345A81
:10B7200021E0AE01475D5F4F62E0C701B4E0880FE2
:10B73000991FBA95E1F70E941B5A89A59AA5AA9666
:10B740000FB6F894DEBF0FBECDBFDF91CF911F9132
:10B750000F91FF90EF90DF90CF90BF90AF909F90B0
:10B760008F907F9008959A01462FBC0180E090E071
:10B770000E94FB5A0895EF92FF920F931F93CF936D
:10B78000DF93CDB7DEB760970FB6F894DEBF0FBE7C
:10B79000CDBF9C017B018A0101978F5F934018F018
:10B7A00080E090E01BC0BE016F5F7F4FC9010E9427
:10B7B000295AE114F10419F08D81F70180830115F4
:10B7C000110551F08BE0F801DE0116960D90019203
:10B7D0008A95E1F7F80113868B819C8160960FB6FC
:10B7E000F894DEBF0FBECDBFDF91CF911F910F91B7
:10B7F000FF90EF9008950F931F93CF93DF93CDB7F2
:10B80000DEB764970FB6F894DEBF0FBECDBF8C01D4
:10B8100084E00130180718F080E090E013C0CE01FA
:10B8200041960E943F5A0115110551F0BE016F5F0C
:10B830007F4FC8010E94295A89819A81009711F48B
:10B8400089899A8964960FB6F894DEBF0FBECDBF82
:10B85000DF91CF911F910F910895CF93DF93CDB7D3
:10B86000DEB724970FB6F894DEBF0FBECDBF24E03D
:10B870008130920718F080E090E00FC0009739F413
:10B88000CE0101960E943F5A89819A8106C00E948A
:10B890004F5A009711F40E944F5A24960FB6F8940D
:10B8A000DEBF0FBECDBFDF91CF910895EF92FF9223
:10B8B0000F931F93CF93DF93CDB7DEB764970FB687
:10B8C000F894DEBF0FBECDBF198A1A8A01E010E0DE
:10B8D0000B8B1C8BA895CE0141960E94475A40E1E4
:10B8E00050E06FEF70E0CE01800F911F0E949B62CD
:10B8F00040E1E42EF12C83E00F3F18073CF40F5F8A
:10B900001F4F09831A830150104002C019821A8206
:10B910000E94460D21E0AE014F5F5F4F60E1C7011D
:10B920000E941B5A0F5F1F4F80E190E0E80EF91E46
:10B9300094E000301907FCF264960FB6F894DEBF6D
:10B940000FBECDBFDF91CF911F910F91FF90EF9070
:10B9500008950F931F93CF93DF93CDB7DEB764970E
:10B960000FB6F894DEBF0FBECDBFCE0141960E9448
:10B970003F5A89E00E941116882329F08EE00E9428
:10B980001116882351F48B899C898F5F9F4F21F575
:10B9900089899A898F5F9F4FF9F464E971E084E0A7
:10B9A0000E9455186CE871E085E00E94551868EC1B
:10B9B00070E08BEC98E40E945F1760E0862F0E9495
:10B9C000261783E00E94A84EBC0182E00E94AE18B8
:10B9D0000E94565C0E94B55109891A89011511050A
:10B9E000A9F0BE016F5F7F4FC8010E94295A8B8169
:10B9F0009C8101978F5F974218F0C8010E94BD5A41
:10BA000009811A81A8950115110559F764960FB699
:10BA1000F894DEBF0FBECDBFDF91CF911F910F9184
:10BA20000895EF92FF920F931F93CF93DF93CDB7BB
:10BA3000DEB728970FB6F894DEBF0FBECDBF7B01EF
:10BA40008C01FA018091530590915405892B91F155
:10BA5000E982FA820B831C831F821886022F11272A
:10BA600000FF09C04F83588740E050E0BA01CF0182
:10BA70000E94BB5BFC0101FF05C08F819885906827
:10BA80008F839887ED83FE83EF2BA1F021E0AE0139
:10BA90004F5F5F4F68E080915305909154050E947D
:10BAA0001B5A809153059091540508969093540524
:10BAB0008093530528960FB6F894DEBF0FBECDBF16
:10BAC000DF91CF911F910F91FF90EF900895CF924A
:10BAD000DF92EF92FF921F93CF93DF93CDB7DEB744
:10BAE00028970FB6F894DEBF0FBECDBF10E0C12C73
:10BAF00030E4D32E8091880A181798F5812F992762
:10BB0000FC0123E0EE0FFF1F2A95E1F7E80FF91F74
:10BB1000E80FF91FE85FF74F8081918189839A834D
:10BB2000828193818B839C83848195818D839E8385
:10BB30008085282F33272F833887868187FD03C090
:10BB400031602F83388721E0AE014F5F5F4F68E09F
:10BB5000C6010E941B5A1F5F88E090E0C80ED91EE4
:10BB6000C9CF0E94BA4F2FEF3FEF29833A83FC01E0
:10BB7000858596858B839C8321E0AE014F5F5F4F67
:10BB800068E0C6010E941B5A88E090E0C80ED91EEA
:10BB90000E940C28FC01D0925405C0925305828962
:10BBA00093892685892B41F020FF02C023E001C044
:10BBB00021E04289538907C020FF02C022E001C072
:10BBC00020E04081518160E070E080E090E00E94E0
:10BBD000115D10E040E050E06BE0812F0E946A525E
:10BBE0001F5F1034B8F310E00E9480528823E1F305
:10BBF0001F5F1630C8F310E0212F4FEF5FEF6FEF9C
:10BC00007FEF8FEF9FEF0E94115DC0905305D090A2
:10BC1000540510925405109253058BE4E82E8BE0E6
:10BC2000F82E1FE121E0A70168E0C6010E941B5A1F
:10BC30001150E8E0F0E0EE0EFF1ECE0EDF1E17FF03
:10BC4000F1CF28960FB6F894DEBF0FBECDBFDF91BF
:10BC5000CF911F91FF90EF90DF90CF9008957F924A
:10BC60008F929F92AF92BF92CF92DF92EF92FF920C
:10BC70000F931F93CF93DF93CDB7DEB76C970FB6BB
:10BC8000F894DEBF0FBECDBF0E94420D782E80E03B
:10BC90000E94030D40E050E060E0CA010E94B0281D
:10BCA00086E08E010F5E1F4FF80111928A95E9F729
:10BCB000FF24A80167E08F2D0E946A5284E190E082
:10BCC0000E949515F3942FE32F1598F70E940324F3
:10BCD00019821A82A12C00E4B02E20E0AE014F5F41
:10BCE0005F4F68E0C5010E941B5A89819A81EFEF7E
:10BCF0008F3F9E07E1F00E9473248C01892BB9F0DD
:10BD00008F818F70682FF801808191810E94AD250D
:10BD10008B819C81F801828393838D819E818483B2
:10BD200095838F819885892F992780FD168288E0D9
:10BD300090E0A80EB91E89819A818F5F9F4F69F6A6
:10BD400019861A861B861C86B9E08B2E912C8C0EC8
:10BD50009D1E20E0A40168E0C5010E941B5A898550
:10BD60009A85AB85BC8580509040A040B14008F0DA
:10BD7000A8C08D859E85009709F4A3C028E2803075
:10BD8000920708F09EC0FF242F85388937FF02C034
:10BD9000A2E0FA2E8C012115310589F089011F7767
:10BDA00040E050E0BA01C8010E94BB5B2D853E8592
:10BDB0002817390719F481E0F82A01C08901F40134
:10BDC0002081318142815381CF2CDD242115310521
:10BDD00041055105C1F50E940C287C01C0FE08C038
:10BDE0004496AC0160E070E0C8010E94BB5B8C012E
:10BDF000C8010E944B248C010097D1F0FC014481C2
:10BE000055816681808191810E94B028F8018085EA
:10BE10000E941129F801828193810E944B2400978E
:10BE200039F0FC0164817581808191810E94FA283A
:10BE3000C1FE04C0F701868581608687F70186858B
:10BE4000826086873EC0802F8F778F8B000F012FF7
:10BE5000001F110B1195802F8F77888FF40180813F
:10BE60008F77898FE7E05695479537952795EA951F
:10BE7000D1F7822F8F778A8F77E056954795379540
:10BE800027957A95D1F7822F8F778B8F67E056951C
:10BE90004795379527956A95D1F7822F877053E09C
:10BEA000CC0CDD1C5A95E1F78C298C8FAE01495ED4
:10BEB0005F4F6CE08FEF0E946A520E94805288238D
:10BEC000E1F388E090E0A80EB91E89859A85AB85DC
:10BED000BC8580509040A040B14008F435CF0BE4C1
:10BEE0001BE04FE1F42E20E0A80168E0C5010E94AC
:10BEF0001B5AFA94085F1F4F88E090E0A80EB91E05
:10BF0000F7FEF1CF83E00E94030D84E690E00E94EB
:10BF100095158B819C810E940861872D0E94030DDD
:10BF20006C960FB6F894DEBF0FBECDBFDF91CF91F8
:10BF30001F910F91FF90EF90DF90CF90BF90AF9047
:10BF40009F908F907F9008956FEF7FEF80E090E05B
:10BF50009C014FE1FC01E20FF31FEB5AFA4F6083A3
:10BF6000718341502F5F3F4F099647FFF3CF0895EC
:10BF7000AC01FC0123E0F695E7952A95E1F7E55B36
:10BF8000F44F808199279A012770307002C09595EF
:10BF900087952A95E2F7440F551F382F317080FF9F
:10BFA00002C04F5F5F4F20E0E5E5F5E080819181C1
:10BFB0008417950741F4332319F082E590E0089542
:10BFC00087E490E008952F5F3A96203278F3332388
:10BFD00019F082E790E0089587E690E008950895CB
:10BFE000DF92EF92FF920F931F93CF93DF937C0129
:10BFF000D62E805F9F40B0F080E090E0C8C0E08225
:10C00000F1828091F2069091F306A091F406B0912E
:10C01000F50686839783A087B18782839383A48361
:10C02000B5831BC020E0E5E5F5E0808191818E15A8
:10C030009F0599F02F5F3A962032B8F320E0E5E5AE
:10C04000F5E0808191818F5F9F4FC9F22F5F3A9613
:10C050002032B8F3C0E0D0E003C0EF01EF2B11F4C1
:10C06000CE0195C00E94BA4F8C01DD2009F473C047
:10C07000FC0183859927AA27BB27BC01CD0122E3B8
:10C0800030E040E050E00E94A2679B01AC0180914B
:10C09000F2069091F306A091F406B091F506820F96
:10C0A000931FA41FB51F8E839F83A887B987F801AC
:10C0B00084859927AA27BB27BC01CD0124E630E05F
:10C0C00040E050E00E94A2679B01AC018091F20623
:10C0D0009091F306A091F406B091F506820F931F9C
:10C0E000A41FB51F8A839B83AC83BD8361E08881D5
:10C0F00099810E94A61BC70144E0969587954A95B1
:10C10000E1F7482FB701769567959B01277030704E
:10C1100081E090E002C0880F991F2A95E2F7982FDE
:10C120005527E0FE06C0FA01E55BF44F8081892BBC
:10C1300006C0FA01E55BF44F9095808189238083E6
:10C14000F8018585968586179707F8F465877687C1
:10C150000E94414F1AC06E817F81888599850E9417
:10C160005E13882349F48E819F81A885B9858A83CF
:10C170009B83AC83BD8309C06D2D888199810E940A
:10C18000A61B8FEF9FEF8883998381E090E0DF917A
:10C19000CF911F910F91FF90EF90DF9008951F9323
:10C1A000CF93DF93C5E5D5E01FE1888199818F5F4B
:10C1B0009F4F31F16A817B818C819D810E945E134A
:10C1C000882351F060E0888199810E94A61B8FEF3F
:10C1D0009FEF8883998314C06E817F8188859985BC
:10C1E0000E945E13882361F08091F2069091F3061D
:10C1F000A091F406B091F5068E839F83A887B98736
:10C2000011502A9617FFD1CFDF91CF911F9108953A
:10C210009F92AF92BF92CF92DF92EF92FF920F93D5
:10C220001F93CF93DF937C0188EFE81687E0F80631
:10C2300008F074C00E94BA4F5C01FC01E586F686E6
:10C240000E94414FCC24DD249924092D1127E016AA
:10C25000F10608F44EC0C80163E0969587956A958B
:10C26000E1F7482F98012770307081E090E002C01C
:10C27000880F991F2A95E2F7982FE801CC0FDD1F50
:10C28000E42FFF27E55BF44F8081892309F0219695
:10C2900061E0CE010E94F05F60E0CE010E94F05F9D
:10C2A00060E081E00E9426170894E11CF11CFF92D7
:10C2B000EF920894E108F1080894C11CD11CDF92A8
:10C2C000CF9288E10E94A84E9F938F9382E08F9334
:10C2D0000E94041984E690E00E9495158DB79EB7E0
:10C2E00007960FB6F8949EBF0FBE8DBF0C5F1F4F11
:10C2F000AECFF501838599270E9495159394F3E0BD
:10C30000F91508F0A2CF84E690E00E94951502C0CE
:10C310000E94460D0E94961D8823D1F3DF91CF9194
:10C320001F910F91FF90EF90DF90CF90BF90AF9053
:10C330009F900895EF92FF920F931F93CF93DF93F7
:10C3400080919506682F772710929506EBE4FCE024
:10C350008191882311F0706805C08DE0EA34F807F8
:10C36000B9F3B4F340E050E08091880A9927481768
:10C3700059079CF4DC019A01F901E40FF51FE85F0D
:10C38000F74F878180FF02C0706407C04F5F5F4F27
:10C39000275F3F4F4A175B077CF340E050E08091F6
:10C3A000890A9927880F991F4817590704F57C01B6
:10C3B000EBECFAE00BE81AE0CBE0DBE09991D80176
:10C3C0008D918D01981759F48081282F3327892F5B
:10C3D00099278095909528233923232B11F070629B
:10C3E00006C04F5F5F4F31964E155F053CF3CB01A2
:10C3F000DF91CF911F910F91FF90EF900895909151
:10C400009506982B9093950608959C0187E0283F08
:10C410003807A0F4F90183E0F695E7958A95E1F7EE
:10C42000E55BF34F2770307081E090E002C0880F29
:10C43000991F2A95E2F72081282B208308950895DB
:10C4400028E28030920740F40E944B24FC01892BA3
:10C4500019F087818160878308950895CF93DF93D2
:10C460001092950680E091E0EBE4FCE011920197D8
:10C47000E9F7CBE8DAE0ABE0BBE0EBECFAE0809187
:10C48000890A9927880F991F009741F09C018D9187
:10C490009191892B899321503040C9F7E8E0F8E069
:10C4A0008091880A9927009751F09C0187818E7F9F
:10C4B0008783215030403A9621153105B9F7DF9135
:10C4C000CF910895E199FECF9FBB8EBBE09A99274B
:10C4D0008DB308954115510569F0DC01E199FECF56
:10C4E0007FBB6EBBE09A6F5F7F4F0DB20D924150E4
:10C4F0005040B1F70895E199FECF9FBB8EBB6DBB55
:10C500000FB6F894E29AE19A0FBE089541155105CD
:10C5100089F0DC018FB7E199FECF7FBB6EBB0D9038
:10C520000DBAF894E29AE19A8FBF6F5F7F4F415046
:10C53000504089F70895DC0101C06D93415050408F
:10C54000E0F708950F931F93CF93DF93CDB7DEB736
:10C550002C970FB6F894DEBF0FBECDBF0B891C8998
:10C56000ED89FE893EE03C8309831A834FEF5FE744
:10C570004D835E83AE01495E5F4FBF01CE010196E0
:10C580000E945D642F813885020F131FD8011C9211
:10C590002C960FB6F894DEBF0FBECDBFDF91CF91C2
:10C5A0001F910F910895FB01DC018D91019080197D
:10C5B00011F40020D1F7990B0895FB01DC010190E3
:10C5C0000D920020E1F70895FB01DC01415050403D
:10C5D00030F08D910190801919F40020B9F7881B73
:10C5E000990B0895FB01DC014150504030F08D91D2
:10C5F0000590801919F40020B9F7881B990B08954C
:10C600002F923F924F925F926F927F929F92AF9242
:10C61000BF92CF92DF92EF92FF920F931F93CF932F
:10C62000DF93CDB7DEB76E970FB6F894DEBF0FBEBF
:10C63000CDBF898B9A8B6B8B7C8B4D8B5E8B3C013A
:10C640001F8A188EF30191903F01892D99270E942E
:10C650001C68892BB9F70DE2901609F4FFC01BE2A4
:10C66000911609F4F7C02D893E892115310509F489
:10C67000DAC02031310509F4D6C0ED89FE89EF2BEF
:10C6800041F430E3931609F4C9C04AE050E04D8B01
:10C690005E8B8D899E89AA2797FDA095BA2F898FD9
:10C6A0009A8FAB8FBC8F8F89988D892B09F4B1C07D
:10C6B00060E070E080E090E8298D3A8D4B8D5C8DD4
:10C6C0000E944D6829873A874B875C876D877E87F4
:10C6D0008F87988B58E0DE011196FE013996019004
:10C6E0000D925A95E1F7CC24DD247601AA24BB24CF
:10C6F00029803A804B805C802D813E812D8F3E8F3A
:10C70000092D1127C8010E941068892BC9F1C801A1
:10C710000E941568892B09F46BC070ED970E892D66
:10C7200099276D897E898617970754F5B7FC24C031
:10C730002C143D044E045F04F8F0C214D304E40446
:10C74000F504A9F021E0A22EB12CC701B601298D74
:10C750003A8D4B8D5C8D0E94A2676B017C01C90CE8
:10C76000D11CE11CF11CD3019D903D01C9CFAD8CC2
:10C77000BE8CA816B90634F73FEFA32EB32EF3CF25
:10C78000B7FE29C0EF89F88DEF2BE1F0C12CD12C39
:10C79000E12C90E8F92E02E210E010934C0D00938A
:10C7A0004B0D8B899C89892B09F460C0AB2839F02B
:10C7B000C3010197AB89BC898D939C9357C089892C
:10C7C0009A89F8CF8FEFC82E8FEFD82E8FEFE82EF3
:10C7D0008FE7F82EE0CFAF89B88DAB2B11F3F09433
:10C7E000E094D094C094C11CD11CE11CF11CD9CFA1
:10C7F000C8010E94F667892B19F2C8010E94F467EC
:10C80000892B21F0802F8753982E89CF802F875531
:10C81000FBCF6FEF7FEF8FEF9FE74ECF08E010E089
:10C820000D8B1E8B36CF40E3941609F026CFF30113
:10C830008081883719F0883509F01FCFD301119610
:10C840009C9082E090E0680E791E60E170E06D8B54
:10C850007E8B13CFD3019D903D0105CF21E030E0C9
:10C860002F8B388FF30191903F01FDCEC701B601A8
:10C870006E960FB6F894DEBF0FBECDBFDF91CF919D
:10C880001F910F91FF90EF90DF90CF90BF90AF90EE
:10C890009F907F906F905F904F903F902F90089562
:10C8A000DC015C91552341F05F7D51341CF05B3518
:10C8B0000CF45C931196F5CF08952F923F924F920E
:10C8C0005F926F927F928F929F92AF92BF92CF9220
:10C8D000DF92EF92FF920F931F93CF93DF93CDB729
:10C8E000DEB762970FB6F894DEBF0FBECDBFAA24A5
:10C8F000BB2465014C016D877E874F87588B44248C
:10C900005524FC0146825782838181FD5BC28FEFF3
:10C910009FEF6FC240FE44C2862D80538A30E0F400
:10C92000F0E36F1641F42A89222329F4772019F4C1
:10C9300080E091E08BC08AE09A89989F902D112425
:10C94000892F860D80538A8B882314F4EFE7EA8BB6
:10C9500043FC38C27A8836C243FE05C0FA89FF23F9
:10C9600011F421E02A8B862D992787FD9095883632
:10C97000910554F5853691050CF06BC0883591050D
:10C9800009F4D3C089359105B4F48B32910509F4CB
:10C9900042C08C32910544F48032910509F43FC0C5
:10C9A000839709F442C0F2C18D329105D9F18E9777
:10C9B00009F440C0EBC18336910509F454C08436B4
:10C9C000910509F478C0E2C18037910509F4A5C04A
:10C9D0008137910584F48C369105B1F18D3691053E
:10C9E0002CF48936910509F466C0D0C18F369105C3
:10C9F00009F490C0CBC18537910509F498C08637FA
:10CA0000910524F483379105B9F1C0C188379105A8
:10CA100009F48BC0BBC180E190E0482A592AE0E2CA
:10CA2000F0E005C080E890E011C0E0E4F0E04E2ABC
:10CA30005F2AC8C188E090E0482A592AEFEFFEEF4C
:10CA40004E225F221A8ABEC184E090E0482A592A09
:10CA5000B9C10F2EFFE3AF2EF02D7A940F2EF3E61F
:10CA60006F2EF02D3AC1EF85F889CF0102968F879E
:10CA7000988BA0807A9431C1EF85F889CF01029616
:10CA80008F87988BA080B18043FE0BC0EA898E2FE0
:10CA9000992787FD9095BC01C5010E949767898BF6
:10CAA00007C0F50101900020E9F73197EA19E98BF9
:10CAB000F9897F1A12C142FE0BC0EF85F889CF01B8
:10CAC00004968F87988B20813181428153810DC0DC
:10CAD000EF85F889CF0102968F87988B80819181AD
:10CAE0009C01442737FD4095542F59016A01552375
:10CAF00064F4E2E0F0E04E2A5F2AD094C094B0944F
:10CB0000A094A11CB11CC11CD11C8FEB9FEF48222B
:10CB100059222BC098E0998B0AC0E0E4F0E04E2A3D
:10CB20005F2A0F2EF8E76F2EF02DF0E1F98B42FE11
:10CB30000BC0EF85F889CF0104968F87988B2081F1
:10CB40003181428153810BC0EF85F889CF01029674
:10CB50008F87988B808191819C01442755275901AB
:10CB60006A01EFECFFEF4E225F221E010894211CA8
:10CB7000311CF989EF2EFF2400271127C601B501CA
:10CB8000A80197010E942B68DC01CB01F101808391
:10CB90008A301CF0860D815203C0F1018081805DD6
:10CBA000F10181931F01C601B501A80197010E94FF
:10CBB0002B6859016A012115310541055105F1F62E
:10CBC000CE010196A22CA81AC20182739070892B03
:10CBD00009F07A9446FE0FC0872D992787FD90951E
:10CBE000F989F03131F40F2EFEEF7F2EF02D780E03
:10CBF00002C0782E7A9443FE12C08A89282F3327E8
:10CC000027FD30958A2D9927821793072CF0E7EF9F
:10CC1000FFEF4E225F2203C0FA89FA19FA8B43FE16
:10CC200003C02A89721A01C07A18C20180789170F3
:10CC3000892B69F4872D7A9418164CF4B40180E29C
:10CC400090E00E946467872D7A941816BCF341FE29
:10CC500004C0B4018DE290E00BC044FE04C0B401F6
:10CC60008BE290E005C045FE05C0B40180E290E093
:10CC70000E94646746FE0FC0B40180E390E00E940A
:10CC800064678989803139F4862D992787FD9095CD
:10CC9000B4010E94646750FE0DC0872D7A94181667
:10CCA0004CF4B40180E390E00E946467872D7A948D
:10CCB0001816BCF343FE11C08A89982F91509A8BA5
:10CCC00018165CF4B40180E390E00E9464678A89DE
:10CCD000E82FE150EA8B1816ACF3842D807869F4C4
:10CCE000872D7A9418164CF4B40180E290E00E94EB
:10CCF0006467872D7A941816BCF3F3E66F1641F437
:10CD00008A2D992787FD9095B4010E9464672DC0F4
:10CD100023E76216B1F489898150898B8F3F29F10D
:10CD2000F5018081992787FD90950894A11CB11C7D
:10CD3000B4010E94646799899150998B9F3F81F754
:10CD400014C0CE0101962816390679F08E010F5FC6
:10CD50001F4FF10182911F01992787FD9095B40122
:10CD60000E94646720163106A1F7842D8078A9F00F
:10CD7000872D7A9418168CF4B40180E290E00E941A
:10CD80006467872D7A941816BCF307C0862D9927FF
:10CD900087FD9095B4010E9464674424552412C015
:10CDA000F5E26F1641F44424552443941A8A7A8894
:10CDB0002AE0298B07C0862D992787FD9095B4011D
:10CDC0000E946467F401838183FF08C0ED85FE85BE
:10CDD000CF0101968D879E87649005C0ED85FE8505
:10CDE0006190ED87FE87662009F094CDF40186817D
:10CDF000978162960FB6F894DEBF0FBECDBFDF916C
:10CE0000CF911F910F91FF90EF90DF90CF90BF9047
:10CE1000AF909F908F907F906F905F904F903F90DA
:10CE20002F9008950F931F93CF93DF93CDB7DEB765
:10CE30002C970FB6F894DEBF0FBECDBF8C0136E045
:10CE40003C8389839A832FEF3FE72D833E83CE0176
:10CE500001960E945D64AF81B885A00FB11F1C923E
:10CE60002C960FB6F894DEBF0FBECDBFDF91CF91E9
:10CE70001F910F9108950F931F93CF93DF93CDB719
:10CE8000DEB72C970FB6F894DEBF0FBECDBF8C0176
:10CE90003EE03C8389839A832FEF3FE72D833E83D7
:10CEA000CE0101960E945D64AF81B885A00FB11FCD
:10CEB0001C922C960FB6F894DEBF0FBECDBFDF914B
:10CEC000CF911F910F9108950F931F93CF93DF93ED
:10CED0008C01EB018B81992781FF22C082FF14C056
:10CEE0002E813F814C815D81241735073CF4A88158
:10CEF000B9810D93A883B9832E813F812F5F3F4F66
:10CF00002E833F83C8010EC0E885F985802F0995DF
:10CF1000892B31F4EE81FF813196EE83FF83F2CFCE
:10CF20008FEF9FEFDF91CF911F910F910895FC013B
:10CF30006150704001900110D8F7809590958E0F48
:10CF40009F1F0895629FD001739FF001829FE00DA3
:10CF5000F11D649FE00DF11D929FF00D839FF00D78
:10CF6000749FF00D659FF00D9927729FB00DE11D24
:10CF7000F91F639FB00DE11DF91FBD01CF01112401
:10CF80000895991B79E004C0991F961708F0961B25
:10CF9000881F7A95C9F78095089597FB092E072673
:10CFA0000AD077FD04D00CD006D000201AF470957A
:10CFB00061957F4F0895F6F7909581959F4F08955D
:10CFC000AA1BBB1B51E107C0AA1FBB1FA617B707AF
:10CFD00010F0A61BB70B881F991F5A95A9F78095CB
:10CFE0009095BC01CD01089585FD17C080629923FD
:10CFF000A1F4813694F08B3784F40895992369F471
:10D00000803269F0893059F08B3039F408958F936C
:10D01000EDDF8F9109F080620895992788270895A0
:10D020009923D9F78095807808959923B1F78033B3
:10D03000A4F38A3394F70895992379F7803279F32A
:10D040008A3069F38C3059F38D3049F3893039F3E4
:10D050008B3019F70895A1E21A2EAA1BBB1BFD0104
:10D060000DC0AA1FBB1FEE1FFF1FA217B307E407C7
:10D07000F50720F0A21BB30BE40BF50B661F771F1F
:10D08000881F991F1A9469F76095709580959095FF
:10D090009B01AC01BD01CF01089597FB092E052628
:10D0A0000ED057FD04D0D7DF0AD0001C38F45095BD
:10D0B0004095309521953F4F4F4F5F4F0895F6F7BC
:10D0C00090958095709561957F4F8F4F9F4F0895F4
:10D0D0005A7A41003F004800484C004854004846F6
:10D0E000002E0053544F50002100474F0048414C40
:10D0F00054004C004C430046004658005400590070
:10D1000056004D54005352005353005345004040C5
:10D11000004200534F000001483B04012334060144
:10D12000233408010E340B0115340E011C34110197
:10D13000623413016234180177341A0177341D0107
:10D140008C342201AE342401383627016936290196
:10D15000B2372C0108392E0137343001B63932018B
:10D16000DC393501273A3801563A3B01BC3A3E01D9
:10D17000B5514101E93A43011A3B00000000800526
:10D180003C2F8105412F8403462F85036F2F880490
:10D19000992F8904C02F8C03EB2F8D03043090034B
:10D1A000223094039C309502DB309802F7309901CD
:10D1B0001A319C021F319D034231A0016931A20145
:10D1C000C631A403DD31A5010132A6010A32A7014F
:10D1D0001032C4011632C6029D3CC703933CC801FD
:10D1E0001932C9015632CA019832CB0117330000F7
:10D1F0000000000100000002000000006C48000375
:10D20000000000006949000064420000473F000040
:10D210008D3F01003D4101009F3F0100664001003C
:10D22000134202006E450200DD440200F245020096
:10D230005146020081450200944502009C440304CB
:10D24000000003000F490305000003002A480306FD
:10D25000000003006347030068470400A94A040074
:10D26000034B05006D4705004D4A06005E4706006A
:06D27000224806002648DA
:00000001FF
